:020000040000fa
:080000000002040000000000f2
:020000040000fa
:100400000f242100007f240000018800000000006c
:100410000a00070011000700000020000000e000b3
:10042000020032000000020000000000f062020042
:10043000000000000040da000000fe004440a90077
:10044000e0c720000000e0000300320000002000b0
:10045000a00188004440a8000000060020072700f3
:10046000010020001500370062004000e0804800d5
:10047000910188009001ba0062004000e0804800cd
:10048000910188009002ba0062004000e0804800bc
:100490000002eb006028e10004003a000059eb0084
:1004a0008301e900fdff3e00040037006128e10000
:1004b000010032000082eb00050007009101880076
:1004c0001001ba000200e000e7ff3a00000005005a
:1004d000910188008002780062004000e0804800be
:1004e0003559ba008301e900080032002559ba00e5
:1004f0008301e900050032000400e000f4ff32004f
:1005000015d9ba008301e900f1ff3a0000000600a6
:100510006c7d0400000000002e7f0400000000003d
:100520000c60040000000000826104000000000074
:1005300086610400000000009a62040000000000d0
:10054000d88c040000000000ce7e040000000000f3
:10055000fe7e04000000000004780400000000009b
:100560006e7a0400000000008e7a04000000000093
:100570008a7a0400000000008c7a04000000000069
:10058000d27b040000000000da7b040000000000c1
:10059000fa7b040000000000547c0400000000000e
:1005a000c67c040000000000067d0400000000007e
:1005b000907a040000000000987a04000000000017
:1005c000b87a040000000000127b04000000000064
:1005d000847b040000000000c47b040000000000d5
:1005e000c68a040000000000ea8b0400000000003e
:1005f000288b040000000000288c0400000000008c
:100600000403040000000000881f78000204780042
:10061000ba000700080040004f0478000000060000
:100620000000fa00881f7800000478003fb99700a6
:10063000ea8157008000780040302000b6000700b3
:10064000800078000000e000020035000040eb0070
:1006500000f47800010078004f0478000080fa0070
:100660000000060080007800010037000000e8006c
:100670001004e000fdff3a000100500000000600f9
:100680008001eb0002003700817178008301e800ef
:10069000828f5100fcff3a0000000600889fbe00d8
:1006a000e30440000900a100808f54004a00360096
:1006b000e38f540001003e00490020006281800069
:1006c0000200e00002003200820078000c003700d7
:1006d000e102210003003700908f54002300360010
:1006e0008080e800110078000000e000faff3a0086
:1006f0000f003700908f54001c0036008080e80007
:10070000110078000000e000faff3a0012017800c2
:10071000e102210003003700908f540013003600df
:100720008080e80011007800820f5000faff3a0044
:1007300058818000890f54000100310009047800bd
:10074000080078002d0107000000e00004003a00d6
:10075000890f5400200032000804d100f5ff370053
:100760000818780031000700d4ff37001101780025
:100770009201780064805100890f5000030031001d
:10078000120090008008780007003700090041003f
:100790008008780092019000130098001100780002
:1007a0001288140009097800910078000100e00027
:1007b00005003200110090000000e000020032004d
:1007c0000180e800010037000000eb006081880034
:1007d0000280e800010037000000eb004f04be007b
:1007e0000000060000047800060037008200410087
:1007f00090818000e10078000200e800808188009c
:100800000100010082818000a0818000800f5100e2
:10081000f6ff390000f520009081880020022000ba
:10082000a081880008007800d80307000000e000dd
:10083000310032008080e90091027800e38f52009d
:100840002d0036000508a3002b003a0072818000bd
:100850000200e00002003200828f500004003100ec
:1008600002087800718188001600370003017800c3
:10087000920190000300e00002003200818f5100dd
:10088000faff39001202780004004100808f500006
:1008900019003900810f500003003a000509420099
:1008a00082007800070037000300e00003003200f8
:1008b00005804000808f51000f00390093009800a0
:1008c00011019800110190000200e0000a003200be
:1008d00011804000820f500007003a00c002210042
:1008e0000008eb0011009000110178009008410011
:1008f0001000900090009800000006008001eb00be
:100900000200370061f079008301e800828f510016
:10091000fcff3a00000006006200fa00889fbe005b
:100920008a9fbe000004be000205780083007800a4
:1009300060f92f000f004000b700070088979f0064
:1009400099979f000000eb00a09f9f009a457800b8
:100950000b80fb000000ea00cf04de0050c2b300b1
:1009600080cf5500020032000904780001003700f2
:100970000904e9000800e0000b0034001f90970014
:10098000080178008a0078008f9197000300010029
:1009900090979f000000e000930032002f9897008e
:1009a00000004400a09f9f000905450050c2b3000d
:1009b00080cf5500040032000b04e000e3ff3a0052
:1009c0002f989700890037000000eb00809f9f0060
:1009d000f0979f00e0979f00d0979f00c0979f00df
:1009e000b0979f00c09f9f0009003700e0002100e2
:1009f000008050000000400021002100e10078004c
:100a00004f98970001007000c09f9f000a05e80002
:100a10001a4478008800fb00e000210083000700f2
:100a2000800078000000e000f0ff3a00a0c2b300b0
:100a3000804f54000e003a00bf8897000180e90003
:100a4000b08f9f0010007800b09f9f000000e00072
:100a500005003d000000ea00b09f9f004f989700fe
:100a60000020a000c09f9f000a05e800100037008a
:100a7000b19f9f0009003700bf989700f0ff270043
:100a8000808f5000040032006a08b9000000410065
:100a900003004000b09f9f000a05e8001a01fb0018
:100aa00003fd2f0003004100e90f5000f2ff360064
:100ab000e0c2b3009a4f1000040032000080eb0047
:100ac000909f9f008a0478001c0037008a04e80089
:100ad000a0c2b300994f100007003a00bf889700ea
:100ae0000180e900b08f9f0010007800909f9f0068
:100af0008a84e800110037000000eb00909f9f00ff
:100b0000090037009f989700f0ff2700808f500062
:100b1000040032006a08b9000000410003004000f0
:100b2000909f9f008904e8001901fb0003fd2f003e
:100b300003004100e90f5000f2ff3600194478002d
:100b40008800fb00c0012100380007000000e00021
:100b500002003a0000447800010037008904e800f0
:100b6000a87f9f0080c6b300804f540004003a0065
:100b7000994f14000a003a00664050000600370002
:100b8000c0c6b300804f540005003a00994f1400ce
:100b900003003a0065404000a07f9f008904e80000
:100ba0000905e800cbfb2f008f8545001901fb00ec
:100bb00060f92f000f0040000084e8008b017800ee
:100bc0008000780008007800210007000000e000a5
:100bd00005003a008b007800080078005f010700ec
:100be0000000e00059ff3d000080eb004f05be0013
:100bf0004f04be000080fa00000006000000e00084
:100c000003003400e9020700e10f400001003a0050
:100c10000000eb00000006000200fa00f1bf9f0098
:100c2000010878000080fa00000006000400370088
:100c30000204e00001003a00000005000000e800a6
:100c400010417800814f5100f9ff3a000000060082
:100c5000889fbe008a1f7800000478000102780097
:100c60008244780003057800e0c6b300804f51004d
:100c7000d200320015003c006b405000804f510004
:100c8000240032000a003c0070405000804f5100a8
:100c90000f01320065404000804f51007400320067
:100ca00050c2b300804f510020013a001c013700b0
:100cb00040c6b300804f51001b0032006540400029
:100cc000804f510019013a001700370030c7b300b8
:100cd000804f5100fe00320007003c00644050008d
:100ce000804f5100620032000040e800804f510008
:100cf0000e013a00e700370050c7b300804f5100a3
:100d00005b00320063404000804f510007013a0011
:100d1000570037009180e900010a780078009000c0
:100d20009171780007013700a8609000c0c6b30039
:100d300080cf50000a003a00940078006480500090
:100d4000000a78001000be004f89de00cf91de005f
:100d50000002be000203780082037800130037000f
:100d600010c7b30080cf500003003200a0c6b3000c
:100d700080cf500006003a00940078006880500050
:100d8000000a78003002be002003be0007003700d2
:100d90001480e900000a7800100078000002780052
:100da000cfa2de000503780086037800049cbe0015
:100db0000694be00a860900080c6b30080cf5000ab
:100dc0000e00320020c6b30080cf500005003a006c
:100dd0000400fb00cf80de00010178008201780072
:100de0000a00370040c7b30080cf50000300320034
:100df0006640400080cf500006003a0004007800b2
:100e0000cf80de000101780082017800009cbe00e6
:100e10000294be003800be002801be00e00f500062
:100e2000e08f5800e00f5900e08f590003003d00ab
:100e300078009000d1c2b3000a003700081090007b
:100e40000018a3000300320078009000b1c2b30084
:100e5000040037000008a30053003200780090001f
:100e600001c2b300017578000000e8004d003700b2
:100e7000a8609000c0c6b30080cf500006003a00c2
:100e80009400780064805000000a78001002be00d0
:100e90006033b8001300370010c7b30080cf500094
:100ea00003003200a0c6b30080cf500006003a0015
:100eb0009400780068805000000a78003002be007c
:100ec0002003be00070037001480e900000a780004
:100ed00010007800000278000500200006002000c5
:100ee00007002000049cbe000694be00a86090008d
:100ef00080c6b30080cf50000e00320020c6b30081
:100f000080cf500005003a000480fb000100200063
:100f100002002000030020000a00370040c7b30091
:100f200080cf5000030032006640400080cf500068
:100f300006003a00040078000100200002002000b2
:100f400003002000009cbe000294be000810900028
:100f50000038a300140032003800be002801be0093
:100f6000e00f5000e08f5800e00f5900e08f59006b
:100f70000d00320080c7b30080cf54000300320060
:100f800080c5b30080cf540007003a00780090007d
:100f900001c3b300017578008000e80009f578000e
:100fa0000080e80070049800780090000000450080
:100fb000600498008940780042003700a8609000e3
:100fc000c0c6b30080cf5000250032000a003c00ac
:100fd0006440500080cf50002800320000c0e8007c
:100fe00080cf5000140032006840500080cf500085
:100ff00022003a000a00370040c7b30080cf5000fb
:101000001e0032006640400080cf50001b003200be
:101010006940500080cf500018003a0006003700a9
:101020001480e900000a780010007800485c900005
:1010300008487800450037001480e900000a78006d
:101040001002780068089000cf80de00010178006f
:1010500082017800009abe000292be003b00370079
:101060001480e900000a78001001780068089000f8
:10107000cf80de000089be00340037001480e90014
:10108000000a780010007800680c900008087800ca
:101090002e0037001180e9008008780010007800e9
:1010a000cf80de000101780082017800009cbe0044
:1010b0000294be0078009000000045006004980093
:1010c00081c7b30008007800ee0007001f0037005a
:1010d0001480e900000a780010007800600498008d
:1010e000580990000200e00002003d005dfd07008d
:1010f000090037008000eb009a01070080007800ab
:101100000000e00003003200680090000080500002
:101110000100370058089000100c98000b003700b1
:101120007800900002757800060037007800900083
:10113000800045000904e00001003a0059c2b300f4
:10114000894878000000e800700498000000eb0077
:101150004f0578004f04be00000006000400fa00ae
:10116000889fbe008a9fbe008c1f78000004780014
:101170000106780070089000f8009000010050000f
:10118000880890000100500098089000010050006d
:10119000a808900001005000b8089000010050001d
:1011a000c8089000810550000002220090bf9f00f7
:1011b00000032300a0bf9f00081090000028a30098
:1011c00018003a000b00e000160034008b04780091
:1011d00009057800e28f5400020036002a00200042
:1011e000020037000900e0000b00340058009000b6
:1011f000c80190000a017800ee805700030001004a
:10120000500498000000e00096003200680890004a
:1012100000004500600c98008a8454004240a900f8
:10122000ebff3c00780190000200e0000b0034006e
:1012300058009000c80190008c0078000300010065
:10124000500498000000e00086003200680890001a
:10125000f800900001004000600c9800880c90009d
:101260000900e0001500340009057800e28f540001
:10127000020036002a002000020037000900e000ca
:101280000b00340058009000c80190000a0178005b
:10129000ec80570003000100500498000000e000bb
:1012a000700032006808900000004500600c980053
:1012b0008a8454004240a900ebff3c0018099000ca
:1012c0000200e0000b003400e8009000580090009d
:1012d000c801900003000100500498000000e000e5
:1012e00060003200680890009808900001004000fb
:1012f000600c9800a80c90000900e0001500340074
:1013000009057800e28f5400020036002a00200010
:10131000020037000900e0000b0034005800900084
:10132000c80190000a017800ec805700030001001a
:10133000500498000000e0004a0032006808900065
:1013400000004500600c98008a8454004240a900c7
:10135000ebff3c00380990000200e0000d00340073
:10136000e80090001808900080804000580090002d
:10137000c801900003000100500498000000e00044
:101380003800320068089000b80890000100400062
:10139000600c9800c80c90000900e00015003400b3
:1013a00009057800e28f5400020036002a00200070
:1013b000020037000900e0000b00340058009000e4
:1013c000c80190000a017800ec805700030001007a
:1013d000500498000000e0002200320068089000ed
:1013e00000004500600c98008a8454004240a90027
:1013f000ebff3c00081090000028a3001b00320007
:101400000b00e000190034008b0478000905780017
:10141000e28f5400020036002a002000020037004c
:101420000900e0000b00340058009000c801900053
:101430000a017800ee805700030001005004980074
:101440000000e0000700320068089000000045003e
:10145000600c98008a8454004240a90003003400c4
:10146000eaff37000080eb00010037000000eb00ce
:101470004f0678004f05be004f04be000080fa0002
:1014800000000600ef02b000889fbe008a9fbe00e9
:101490008c9fbe008e1f780000067800f0fd2000b3
:1014a000c0b79f0080c5b30080cf50000800320055
:1014b000e2fc2000c2b79f007740400080cf500080
:1014c00003003a0083002000b3b79f000a003700f2
:1014d00080c7b30080cf500005003200a400200078
:1014e000b4b79f0080c5b30080cf500002003a001f
:1014f00000012000b0b79f003c04be002c05be00d8
:1015000040c6b30080cf5000030032006540400069
:1015100080cf50000b003a00e00f5400e08f5c00d9
:10152000e00f5d00e08f5d0006003d006000b80048
:101530006011b80008045000898458000a05590059
:101540008b855900e00f5400e08f5c00e00f5d00d8
:10155000e08f5d0004003a005c0890008d012000df
:101560000000e0000c003200bfb0970001027800dc
:10157000cfa2de0005037800860378000800be00d5
:101580000a01be006e0207004fb297006440780067
:10159000d0df9f007d0120003fb09700000278005f
:1015a000cfa2de0005037800860378000800be00a5
:1015b0000a01be005b020700009ebe000296be004c
:1015c0000d00e90061fc2f008f8040000087400083
:1015d0001e0037003fb1970002047800cfc4de0040
:1015e000090578008a0578000802be000a03be00db
:1015f0007fa897008fb097001fb19700afb19700f9
:1016000053020700d0b79f00e1b79f00f2b79f00d9
:1016100083bf9f008d06e9000802be000a03be00da
:10162000d10207007faa970000005200cfb09700b8
:10163000615778005fb09700efb097007fb19700d7
:101640008fb99700009ebe000296be003c00be000f
:101650002c01be00f0af9f0081b79f0092b79f00a2
:10166000a3b79f00e00f5000e08f5800e00f590033
:10167000e08f5900020034000d00e000d5ff3c006f
:10168000bfb09700e88f500010003a000c10900097
:101690000038a3000d003200f78f560006003e0010
:1016a00062fc2f000f0141008d00410000c3b30018
:1016b000914f1000050032008d06e90000c3b30011
:1016c00063fc2f008f81410080f17e00788116003d
:1016d000120e98006c00900063fc2f008f81410077
:1016e0008d80410085fc07001c0990005c0890007b
:1016f000800f510006003d0002005000000e9800cf
:101700000c1090000040a100001698000f00370058
:101710000000e0000d003d000c109000740060001f
:10172000f00f500009003a007c089000fc00900087
:10173000010050008c089000010050000200500091
:101740004240a90001003400000e98004f077800c5
:101750004f06be004f05be004f04be00ef02b100b1
:10176000000006008001eb00040037008301e80060
:1017700090cf1000040032000000e800828f51007a
:10178000faff3a000000eb00000006002002e20031
:1017900004003d002342ab00020032002302ab00f4
:1017a000feff32000040da00feff3700889fbe00d7
:1017b00080047800d20ce20004003a000000eb0044
:1017c000100007000000e0000a003500906680006d
:1017d0000900e00002003a0000047800060037002b
:1017e0000004780009004000060007000000e00047
:1017f00001003d000084eb00080078004f04be00ab
:1018000000000600800078000000e00004003a00bc
:10181000000421009066880001017800060037006e
:101820000081eb0000242100808f500002003e0068
:10183000916688000001eb000200780000000600bd
:10184000889fbe008a9fbe00010578000100e0006d
:101850000400350008003c000000e00020003200d9
:101860000500370060001000e080180002003b0017
:1018700001f02c001a0037000004be006011b8000f
:101880006b0920000982cf00020039000882cf00d6
:101890000441b000694252000e00320008003b00d3
:1018a00082817100610164008904d1000884d30041
:1018b0008b05e8000442e800f9ff3a000500370014
:1018c0000804440089844c008b05e9000442e900c7
:1018d000fbff3a00520207000af0a70001f0a00047
:1018e0004f05be004f04be000000060003f0a2003a
:1018f000889fbe008a9fbe008c1f78006e02070082
:10190000750233006450e1004f0032006420e100b2
:101910005200320003826c0007003b000905d00032
:101920000306d000820f54000c065d00020039004f
:101930000200320089017800030678008582550094
:1019400004003d000003fd008103fd008502ea0064
:101950008b854200840f720002003b006000100083
:10196000e08018006011b8000005eb007a28e10063
:101970000a00390006007800c75ddd00f707b200f5
:10198000878075002d003700828171000a01780080
:10199000610560008180d1000080d3008502e900ec
:1019a000f9ff3b00060440008784480002003b002a
:1019b00060041400e0841c000988a30007003200c2
:1019c0008a81710082817100610164008904d10003
:1019d0000884d3008b05e800170037000978a300be
:1019e00013003a000b00e000130034008b05e900ff
:1019f0000804440089844c000a4474000978a30058
:101a00000d003a000b00e000070034008b05e900f0
:101a10000804440089844c0001003a000b002000b7
:101a20000978a300f7ff32000001eb000200370045
:101a3000828171000a017800f90107000cf0a7000b
:101a400001f0a0002d0237006420e10002003a00fe
:101a5000838f6c002d0233000801be000200be001f
:101a600026023700889fbe008a9fbe008c1f780028
:101a7000110207001802330003866c006450e10075
:101a80002e0032006420e100330032006150e1009a
:101a90002f0032006120e1003100320085855500c1
:101aa000eb07b00009002000080420000500370003
:101ab0000804440089844c000a00310006034300f6
:101ac00087834b000001530081815b00f8ff3300e6
:101ad0000203be000800a0000804440089844c00f2
:101ae000f6ff3900c639dd008301730001003200c2
:101af000130020008904d1000884d3000998a300b2
:101b0000050032000800a7000300a0008904d100ee
:101b10000884d3008b05e8008904d1000884d30031
:101b20000001eb000281d200bd01070001f0a1001d
:101b30000cf0a70001f0a000f00137006420e100e4
:101b4000f20132000801be000200be00f7ff3700bc
:101b50006120e100ed0132006000b800f3ff3700c2
:101b60000000200001f82700f0ff3700889fbe002a
:101b70008a9fbe008c1f7800cf010700d60133007a
:101b800003866c006450e100240032006420e10010
:101b9000270032006150e100220032006120e100a4
:101ba000210032008b854200eb07b1000134b80000
:101bb000003ab8000804420089844a00013ab8009b
:101bc0000030b8008880400009014a00040033005a
:101bd0000000400081804800020149008b05e900b7
:101be000c909dd00830170000100320013002000ec
:101bf000c814de004814dd004709de001200b20000
:101c0000c808de00088470008501070001f0a1000b
:101c10000cf0a70001f0a000b80137006120e1003e
:101c2000ba0132000801be000200be00f7ff370013
:101c30006150e100fcff3a00b40137000001be0032
:101c4000b50107000470a70003f0a1006509b10009
:101c5000160032000d0035006828e100060035004e
:101c6000f0ff2f00f1ff27000300e00013003b000e
:101c700001002800000005000000400081804800ad
:101c80008502e900fcff3a0008003700f88f4200a7
:101c900002003c008000eb00000005008100d10044
:101ca0000080d3008502e800fcff3a000300e0005a
:101cb00002003b0060001000e080180000000600f9
:101cc000f4ff2f00a901370014002000a7013700fe
:101cd0000001be00900107000470a70003f0a100fe
:101ce00003f8a30013003a006509b10010003200a8
:101cf000090035006928e1000200350001002800d4
:101d00000000050000004000818048008502e900d5
:101d1000fcff3a0000000600f88f42000500350085
:101d20008100d1000080d3008502e800fcff3a006a
:101d3000000006008000eb0000000500881f78000e
:101d4000000478005001be004000be0004004000c6
:101d5000858048000601490087814900009cbe003b
:101d60000294be000400e1000588e1000690e10055
:101d70000798e10002003100680044001008e80004
:101d80004f04780000000600f4874700889fbe00db
:101d90008a9fbe008c9fbe008e1f78000205be0089
:101da0000004be00d4b79f00e5b79f00f6b79f00c0
:101db00087bf9f000000eb00c0b79f00b0b79f0037
:101dc000a0b79f0090b79f0080b79f000d04200030
:101dd000bfb097004fb09700000140000000e00046
:101de0000f003d004f08de0000007100c0b79f00eb
:101df0009e00070001003d0012002000a100070026
:101e000001003d0012002000a6000700b1000700fd
:101e1000b60007000f004000c8ff0700220037008f
:101e20004f08de0000067100ccb79f008f0007004e
:101e300001003d00120020009200070001003d005b
:101e40001200200097000700a20007000fb29700c1
:101e50009fb297002fb39700bfb39700a900070068
:101e60000000520081805a0002015b0083815b0008
:101e700080b79f0091b79f00a2b79f00b3b79f00a4
:101e80000007eb009f0007000020e10001a8e1002f
:101e900002b0e10003b8e100010031001e002000a3
:101ea0000e005600c0b79f004fb297000400e0003c
:101eb0000700350010002000010020006011b8006c
:101ec00008047000898470000a0571008b85710018
:101ed0008d06e900beff3a000400e00003003d006b
:101ee000820007000f00400094ff07004fa89700f2
:101ef0000000e00004003a000fb497009fb4970080
:101f00002fb59700bfb59700940007004f077800e2
:101f10004f06be004f05be004f04be004f01b1008a
:101f200000000600881f780018002000881f780035
:101f300095ff07008f87e9004f0478000000060036
:101f4000801feb0090ff07008f87e900000006006c
:101f5000889fbe008a9fbe008c1f78006e0007001d
:101f600007003d0073000700e00f5b00e08f5b009f
:101f700007003d00320007000006eb0004003700b8
:101f80003400070002003d002a0007001c0020006a
:101f900072000700e3ff07000203be000002be005c
:101fa0000c00e00001003200220007000400be0027
:101fb0000601be004f0678004f05be004f04be006c
:101fc00000000600889fbe008a9fbe008c1f78001c
:101fd0005100070005003d0056000700e00f5b00c0
:101fe000e08f5b0006003d00040037001900070089
:101ff00003003d006000b8006011b8001000070049
:1020000056000700ceff07000203be000002be001c
:102010000c00e00001003200060007000400be00d2
:102020000601be004f0678004f05be004f04be00fb
:10203000000006006000b8006011b8000000370022
:102040000402500085825800060359008783590016
:10205000000006000006eb00e00f5200e08f5a007f
:10206000e00f5b00e08f5b00000006000180400095
:1020700090b79f000001eb008fb097000100e000d7
:10208000000006000200700090b79f000180400031
:1020900080b79f000001eb00ffa897000100e0005f
:1020a000000006000200700080b79f000180400021
:1020b0006faa9700cf20de0001007000f0af9f00f4
:1020c00004024200250007004f18de0000027200e3
:1020d00000000600e4af9f000804440089844c001f
:1020e0000a054d008b854d00000006003fb29700a9
:1020f000cfb297005fb39700efb3970000fe2f00b9
:10210000000006003fb09700cfb097005fb1970086
:10211000efb19700000006000205be000004be00fb
:10212000e00f5000e08f5800e00f5900e08f590099
:10213000000006006000b8006011b80008045000fc
:10214000898458000a0559008b8559001c0020001d
:10215000e00f5200e08f5a00000006000800be00a9
:102160000a01be0000000600889fbe008a9fbe00d4
:102170008c1f78000205be000004be000006eb00c4
:10218000e00f5000e08f5800e00f5900e08f590039
:1021900007003d006000b8006011b800080450005e
:1021a000898458000a0559008b8559001c002000bd
:1021b000e00f5200e08f5a00e00f5b00e08f5b0001
:1021c00002003d000f0007000c00a2000800be0046
:1021d0000a01be00800007000203be000002be002c
:1021e0000c00e00001003200060007000400be0001
:1021f0000601be004f0678004f05be004f04be002a
:10220000000006006000b8006011b8000402500031
:102210008582580006035900878359000000060094
:1022200081002000618055000b003d000b00200064
:1022300061fe2f000100e1001d0034008281710069
:10224000610164008904d1000884d3000000e80023
:10225000faff3a0071002000610064000300700082
:10226000020060000900320061044400e0844c0078
:102270000988a500050032008b05e8006808e10028
:1022800002003a008904d1000884d300f20f200034
:102290000258e10005003d00c75ddd00f907b2000e
:1022a0008980750008007800000006000bf8270000
:1022b0008b007800000005000004be001600070037
:1022c0000003be000405be000200be0012000700ad
:1022d000844f7500000006000200be006450e1005b
:1022e000050036006420e100020036000968a30002
:1022f00001003a000800be000160a0004f0678000f
:102300004f05be004f04be0000000600f0ff2f0086
:10231000f1ff2700f9ff3700c70ade00f107b2001e
:10232000f50fb20008003200e1cf42000200320097
:102330000170a00024000500810f70000100320030
:102340000408050044000500810f700002003a00f7
:10235000140005008502e9000000400081c048002b
:10236000fcff3b000170a00024000500889fbe0018
:102370008a9fbe00841f7800cfff07004f007800bf
:1023800011003300f0ff2f00838f6c0006003b002c
:10239000040565000a00a7000800370009f0a60040
:1023a0001000200008003700820f5400838f5c006b
:1023b000030039001000200001003e000000200052
:1023c00009f0a7000000ea004f05be004f04be0060
:1023d0000000e00000000600889fbe008a9fbe004b
:1023e0008c9fbe000404b8000506b80089044600ae
:1023f00060854e000606b8000a054600e0854e00de
:102400000706b8008b054600040eb8008904460094
:102410000a854e00e0854d00050eb8000a0546000d
:102420008b854e00060eb8008b0546000416b800da
:102430000a0546008b854e000516b8008b05460040
:10244000041eb8008b0546000800be000a01be004d
:102450004f06be004f05be004f04be000000060040
:102460000000fa0023c2bf000004a2000000fb002d
:10247000610060000080fa00000006000000fa0021
:1024800033c2bf000004a2000000fb006100600036
:102490000080fa00000006000000fa0021e2a90016
:1024a0009560a9009580a9008560a9008580a90094
:1024b0000080fa00000006000000fa0031e2a900e6
:1024c00097c0a90097e0a90087c0a90087e0a900ec
:1024d0000080fa00000006000200fa00000f7800f9
:1024e0008560a9008580a9001e0078006740600013
:1024f0006740600067406000674060004401dd00a5
:10250000910a200091407800f0c8b30000c060003c
:1025100002407000a9e0b700000720001e00600024
:102520004400de006740600067416000a10a2000af
:102530009140780080cfb30000c06000024070007e
:10254000aae0b7009e007800688060004300de00cb
:1025500061406000614060004301dd0051092000de
:102560009140780070cfb30000c06000024070005e
:1025700095e0b700000820001e0060004700de0064
:1025800061406000614060004401dd0051092000ad
:1025900091407800f0ceb30000c0600002407000af
:1025a00095e0b7000080fa00000006000200fa0083
:1025b000000f780087c0a90087e0a9001e007800fe
:1025c00067406000674060006740600067416000ee
:1025d000310b20009140780080cfb30000c0600034
:1025e00002407000b3e0b700000720001e0060004a
:1025f0004400de0067406000674060004401dd0089
:10260000310b200091407800f0c8b30000c060009a
:1026100002407000b3e0b7009e0078006880600060
:102620004300de0061406000614060004601dd0063
:102630007109200091407800f0cbb30000c0600029
:102640000240700097e0b700000820001e00600004
:102650004700de0061406000c700dd0097c0bf009a
:102660000074a1000140700097e0b7000080fa00fc
:10267000000006000000fa0022c2bf0061406000b6
:102680000080fb000080fa00000006000000fa0055
:1026900032c2bf00614060000080fb000080fa0091
:1026a000000006000c00fa0020079800310798008f
:1026b000420798000000eb00100798003e009000d1
:1026c000000f7800230037009e0090004e0090001d
:1026d000808f5000040031001e0090000000e800d0
:1026e00010079800030037002e0090005007980054
:1026f0001d003700dfff07000004e000f2ff32009a
:102700000000eb001007980020c2bf006640600088
:10271000e64f500007003a00311180003e00900063
:10272000010878003e0090000080e8003007980023
:102730000500370030118000804078001e007800ce
:10274000014878001e0fe8002e0090000000e9000c
:10275000200798002e0090000000e000e5ff3a00fe
:102760002e009000500798005e0090000080fa0054
:10277000000006000c00fa002007980031079800be
:10278000420798000000eb00100798003e00900000
:10279000000f7800230037009e0090004e0090004c
:1027a000808f5000040031001e0090000000e800ff
:1027b00010079800030037002e0090005007980083
:1027c0001d003700b1ff07000004e000f2ff3200f7
:1027d0000000eb001007980030c2bf0066406000a8
:1027e000e64f500007003a00b11180003e00900013
:1027f000010878003e0090000080e8003007980053
:1028000005003700b0118000804078001e0078007d
:10281000014878001e0fe8002e0090000000e9003b
:10282000200798002e0090000000e000e5ff3a002d
:102830002e009000500798005e0090000080fa0083
:10284000000006000600fa00000f7800110798004b
:10285000220798002e009000401188001e0078008a
:10286000001188001e009000101188000080fa00fe
:10287000000006000600fa00000f7800110798001b
:10288000220798002e009000c01188001e007800da
:10289000801188001e009000901188000080fa00ce
:1028a000000006000400fa00100798001e009000c7
:1028b000000f780023c2bf00624060000004e00007
:1028c000fcff3a0020c2bf0066406000e64f5000a7
:1028d00019003a000a0037001e009000100078002e
:1028e000201188001e0090000080e800100798006a
:1028f00023c2bf00624060000004e000fcff3a0019
:102900001e009000100078000000e000f2ff3a0086
:102910000d0037001e007800104078000000fb001a
:10292000201188001e0fe80023c2bf006240600033
:102930000004e000fcff3a001e0078001040780020
:102940000004e000f3ff3a000080fa0000000600f7
:102950000400fa00100798001e009000000f780095
:1029600033c2bf00624060000004e000fcff3a0098
:1029700030c2bf0066406000e64f500019003a00c8
:102980000a0037001e00900010007800a011880097
:102990001e0090000080e8001007980033c2bf00be
:1029a000624060000004e000fcff3a001e0090005e
:1029b000100078000000e000f2ff3a000d00370040
:1029c0001e007800104078000000fb00a011880075
:1029d0001e0fe80033c2bf00624060000004e00048
:1029e000fcff3a001e007800104078000004e00070
:1029f000f3ff3a000080fa00000006000200fa002f
:102a000020c2bf0066406000e64f500003003a005d
:102a100030118000000f7800040037003111800071
:102a2000f00f200080806000010f78001e00780009
:102a30000080fa00000006000200fa0030c2bf0069
:102a400066406000e64f500003003a00b01180007d
:102a5000000f780004003700b1118000f00f200053
:102a600080806000010f78001e0078000080fa006e
:102a7000000006000200fa00000f780023c2bf0029
:102a8000624060000004e000fcff3a0020c2bf008a
:102a900066406000e64f500003003a001e007800d8
:102aa0002011880003003700f00f20001e00600096
:102ab000201188000080fa00000006000200fa00e1
:102ac000000f780033c2bf00624060000004e000e5
:102ad000fcff3a0030c2bf0066406000e64f500085
:102ae00003003a001e007800a011880003003700a0
:102af000f00f20001e006000a01188000080fa0086
:042b000000000600cb
:020000040000fa
:0200000401f009
:04000000ffff0000fe
:020000040000fa
:0200000401f009
:04000400ffff0000fa
:020000040000fa
:0200000401f009
:04000c00faff0000f7
:020000040000fa
:0200000401f009
:040010007eff00006f
:020000040000fa
:0200000401f009
:040014007fff00006a
:020000040000fa
:0200000401f009
:04001800ffff0000e6
:020000040000fa
:10000800e48c000078640000da6400003c650000bd
:100018009e650000e48c0000e48c0000e48c000085
:10002800e48c0000e48c0000e48c0000384a0000f6
:10003800e48c0000e48c0000e48c000008810000df
:1000480026860000e48c0000e48c0000ea8b0000a7
:10005800c68a0000e48c0000e48c0000e48c0000f8
:10006800e48c0000aa770000e48c0000e48c000017
:10007800e48c0000e48c0000e48c0000e48c0000b8
:10008800e48c0000e48c0000e48c00008240000056
:10009800e48c0000e48c0000288c0000288b000011
:1000a800e48c0000e48c0000e48c0000e48c000088
:1000b800e48c0000e48c0000e48c0000e48c000078
:1000c800e48c0000e48c0000e48c0000e48c000068
:1000d800e48c0000e48c0000e48c0000e48c000058
:1000e800e48c0000e48c0000e48c0000e48c000048
:1000f800e48c0000e48c0000e48c0000e48c000038
:10010800e48c0000e48c0000e48c0000e48c000027
:10011800e48c0000e48c0000e48c0000e48c000017
:10012800e48c0000e48c0000e48c0000e48c000007
:10013800e48c0000e48c0000e48c0000e48c0000f7
:10014800e48c0000e48c0000e48c0000e48c0000e7
:10015800e48c0000e48c0000e48c0000e48c0000d7
:10016800e48c0000e48c0000e48c0000e48c0000c7
:10017800e48c0000e48c0000e48c0000e48c0000b7
:10018800e48c0000e48c0000e48c0000e48c0000a7
:10019800e48c0000e48c0000e48c0000e48c000097
:1001a800e48c0000e48c0000e48c0000e48c000087
:1001b800e48c0000e48c0000e48c0000e48c000077
:1001c800e48c0000e48c0000e48c0000e48c000067
:1001d800e48c0000e48c0000e48c0000e48c000057
:1001e800e48c0000e48c0000e48c0000e48c000047
:0801f800e48c0000e48c00001f
:020000040000fa
:10020800e48c000078640000da6400003c650000bb
:100218009e650000e48c0000e48c0000e48c000083
:10022800e48c0000e48c0000e48c0000384a0000f4
:10023800e48c0000e48c0000e48c000008810000dd
:1002480026860000e48c0000e48c0000ea8b0000a5
:10025800c68a0000e48c0000e48c0000e48c0000f6
:10026800e48c0000aa770000e48c0000e48c000015
:10027800e48c0000e48c0000e48c0000e48c0000b6
:10028800e48c0000e48c0000e48c00008240000054
:10029800e48c0000e48c0000288c0000288b00000f
:1002a800e48c0000e48c0000e48c0000e48c000086
:1002b800e48c0000e48c0000e48c0000e48c000076
:1002c800e48c0000e48c0000e48c0000e48c000066
:1002d800e48c0000e48c0000e48c0000e48c000056
:1002e800e48c0000e48c0000e48c0000e48c000046
:1002f800e48c0000e48c0000e48c0000e48c000036
:10030800e48c0000e48c0000e48c0000e48c000025
:10031800e48c0000e48c0000e48c0000e48c000015
:10032800e48c0000e48c0000e48c0000e48c000005
:10033800e48c0000e48c0000e48c0000e48c0000f5
:10034800e48c0000e48c0000e48c0000e48c0000e5
:10035800e48c0000e48c0000e48c0000e48c0000d5
:10036800e48c0000e48c0000e48c0000e48c0000c5
:10037800e48c0000e48c0000e48c0000e48c0000b5
:10038800e48c0000e48c0000e48c0000e48c0000a5
:10039800e48c0000e48c0000e48c0000e48c000095
:1003a800e48c0000e48c0000e48c0000e48c000085
:1003b800e48c0000e48c0000e48c0000e48c000075
:1003c800e48c0000e48c0000e48c0000e48c000065
:1003d800e48c0000e48c0000e48c0000e48c000055
:1003e800e48c0000e48c0000e48c0000e48c000045
:0803f800e48c0000e48c00001d
:020000040000fa
:102b0400436f00006d6d0000206c00006f6f0000cb
:102b140070200000697300002073000074610000dd
:102b240072740000656400000a000000497300002c
:102b340020740000686500007265000020610000d8
:102b4400206d00006573000073610000676500007c
:102b5400206600006f720000206d0000653f0000d9
:102b64000a00000025730000202d00003e20000014
:102b7400257300000a00000053300000002a000002
:102b8400005300003100000054680000657200002a
:102b94006520000069730000206400006174000077
:102ba4006120000055410000525400000a0000005a
:102bb40046610000696c0000656400002074000038
:102bc4006f2000007265000061640000206d000049
:102bd4006573000073610000676500000a0000006f
:102be40049200000676f0000742000007468000032
:102bf400652000006d6500007373000061670000cc
:102c0400650a000000540000686500007265000059
:102c140020690000732000006461000074610000fa
:102c2400206f00006e200000425400000a000000e3
:102c34005b25000030320000585d000000430000b6
:102c4400464700005f4300004f4d00004d4c00001c
:102c54004f4f0000503a0000207300006243000010
:102c640066670000436f00006d6d00004c6f00004c
:102c74006f70000044650000636f0000646500002d
:102c84000a0000005365000074200000436f000038
:102c94006d6d00004c6f00006f7000002056000046
:102ca40065720000626f00007369000074790000af
:102cb4000a000000537400006f700000706500008b
:102cc40064200000436f00006d6d00004c6f000035
:102cd4006f7000002056000065720000626f0000f3
:102ce40073690000747900000a0000004346000084
:102cf400475f0000434f00004d4d00004c4f000063
:102d04004f5000003a20000073620000426100004e
:102d14007369000063520000657000006c79000064
:102d2400456e0000636f0000646500000a00000047
:102d340043460000475f0000434f00004d4d000034
:102d44004c4f00004f5000003a2000007362000016
:102d5400536500006e6400004d650000737300004d
:102d640061670000650000004b450000455000000d
:102d74005f4100004c490000564500003a20000025
:102d84007362000042610000736900006352000036
:102d9400657000006c790000456e0000636f0000f0
:102da40064650000004b000045450000505f0000d2
:102db400414c000049560000453a000020730000d1
:102dc40062530000656e0000644d000065730000ee
:102dd4007361000067650000004b0000656500003a
:102de40070200000416c000069760000650a000054
:102df40000430000464700005f4300004f4d0000c1
:102e04004d3a000020730000624300006667000032
:102e1400436f00006d6d000044650000636f0000a7
:102e240064650000005300007461000072740000c7
:102e340065640000206300006f6e00007469000088
:102e44006e7500006f75000073200000636f000052
:102e54006d6d0000756e0000696300006174000010
:102e6400696f00006e0a00000053000074610000e6
:102e74007274000065640000206f00006e2d000075
:102e8400646500006d6100006e6400002063000052
:102e94006f6d00006d7500006e69000063610000d5
:102ea400746900006f6e00000a00000043460000d1
:102eb400475f0000434f00004d4d00003a200000e2
:102ec40073620000426100007369000063520000f5
:102ed400657000006c790000456e0000636f0000af
:102ee4006465000000430000464700005f430000a3
:102ef4004f4d00004d3a0000207300006253000063
:102f0400656e0000644d000065730000736100008d
:102f14006765000000530000544100005445000060
:102f24003a200000736200005265000071530000f3
:102f3400746100007465000044650000636f000064
:102f44006465000000530000544100005445000033
:102f54003a20000046610000696c000065640000ce
:102f6400207400006f200000656e0000636f000095
:102f74006465000020680000656c000069200000a2
:102f84007374000061740000650a000000530000bf
:102f940054410000544500003a20000073620000d0
:102fa400536500006e6400004d65000073730000fb
:102fb4006167000065000000416300006365000074
:102fc40070740000656400002073000074610000e8
:102fd40074650000207200006571000075650000d2
:102fe40073740000202500003034000058200000d5
:102ff40025300000345800000a0000004745000056
:10300400545f00005645000052530000494f000031
:103014004e3a000020730000625600006572000002
:10302400736900006f6e00004d7300006745000077
:103034006e6300006f640000650a00000047000032
:10304400455400005f5600004552000053490000fb
:103054004f4e00003a2000007362000053650000e8
:103064006e6400004d65000073730000616700002a
:103074006500000052650000636500006976000089
:10308400656400002076000065720000736900002a
:103094006f6e00002072000065710000756500000d
:1030a400737400000a000000534500004e530000f2
:1030b4004f5200004c490000535400003a200000d5
:1030c40073620000536500006e7300006f720000ad
:1030d4004c69000073740000456e0000636f0000cb
:1030e400646500000a000000534500004e530000d0
:1030f4004f5200004c490000535400003a20000095
:1031040073620000536500006e6400004d650000aa
:1031140073730000616700006500000052650000e1
:103124006365000069760000656400002073000098
:10313400656e0000736f0000722000006c6900006f
:103144007374000020720000657100007565000052
:10315400737400000a000000436f00006e6e0000ec
:1031640065630000746900006f6e00002061000058
:10317400636300006570000074650000640a000069
:10318400004300004f4e00004e4500004354000031
:103194003a2000007362000042610000736900007d
:1031a40063520000657000006c790000456e0000f9
:1031b400636f0000646500000a000000434f0000d4
:1031c4004e4e000045430000543a000020730000b6
:1031d40062530000656e0000644d000065730000da
:1031e400736100006765000000440000495300005b
:1031f400434f00004e4e000045430000543a000087
:1032040020730000624200006173000069630000e3
:1032140052650000706c0000794500006e63000088
:103224006f640000650a0000004400004953000078
:10323400434f00004e4e000045430000543a000046
:103244002073000062530000656e0000644d0000ae
:1032540065730000736100006765000000440000ae
:1032640069730000636f00006e6e00006563000008
:10327400746900006f6e0000206100006363000049
:103284006570000074650000640a000000520000cc
:1032940045530000455400003a20000073620000ca
:1032a4004261000073690000635200006570000011
:1032b4006c790000456e0000636f000064650000d7
:1032c4000a0000005245000053450000542000004d
:1032d40052650000636500006976000065640000c3
:1032e4000a00000043460000475f00004f41000011
:1032f400564f0000494400003a2000007362000069
:1033040043660000674f000041440000656300000d
:103314006f640000650a0000004300004647000097
:103324005f4f0000415600004f490000443a00003e
:1033340020730000624200006173000069630000b2
:1033440052650000706c0000794500006e63000057
:103354006f640000650a0000004300004647000057
:103364005f4f0000415600004f490000443a0000fe
:103374002073000062530000656e0000644d00007d
:10338400657300007361000067650000004300007e
:103394006f6e0000666900006775000072650000ca
:1033a400642000004f620000737400006163000039
:1033b4006c65000020410000766f00006964000025
:1033c400616e0000636500000a00000043460000cf
:1033d400475f0000544900004d4500004f55000070
:1033e400543a000020730000624300006667000046
:1033f400546900006d6500006f750000744400009e
:10340400656300006f640000650a0000004300006b
:103414006f6e000066690000677500007265000049
:1034240064200000546900006d6500006f750000a1
:10343400743a0000202500006420000026200000cb
:10344400256400000a00000043460000475f0000b6
:10345400544900004d4500004f550000543a000007
:103464002073000062420000617300006963000081
:1034740052650000706c0000794500006e63000026
:103484006f640000650a0000004300004647000026
:103494005f540000494d0000454f000055540000a2
:1034a4003a20000073620000536500006e6400005f
:1034b4004d65000073730000616700006500000043
:1034c400496700006e6f0000726500006420000010
:1034d40054720000696d0000204d00006f6400000c
:1034e40065200000284e00006f2000006861000085
:1034f4006e6400006c650000722900000a00000080
:1035040054520000494d00005f4d00004f4400003c
:10351400453a000020730000625400007269000004
:103524006d4d00006f640000654500006e6300008f
:103534006f640000650a0000005400005249000056
:103544004d5f00004d4f0000444500003a2000004c
:1035540073620000536500006e6400004d65000056
:10356400737300006167000065000000545200009e
:10357400494d00005f4d00004f440000453a0000f3
:103584002073000062540000726900006d4d000059
:103594006f64000065440000656300006f64000010
:1035a400650a000000490000676e00006f720000a9
:1035b4006564000020540000726900006d20000062
:1035c4004d6f0000646500000a000000436f0000b6
:1035d4006e66000069670000757200006564000093
:1035e40020540000726900006d2000004d6f00003f
:1035f400646500000a00000054520000494d0000b8
:103604005f4d00004f440000453a00002073000065
:1036140062420000617300006963000052650000ab
:10362400706c0000794500006e6300006f64000058
:10363400650a000000490000676e00006f72000018
:1036440065640000204300006f6e00007472000087
:103654006f6c00002050000061720000616d00007a
:10366400657400006572000073200000284e00009d
:103674006f200000686100006e6400006c6500004b
:10368400722900000a00000043540000524c00005c
:103694005f500000415200004d3a000020730000ca
:1036a40062540000726900006d4d00006f640000f8
:1036b400654500006e6300006f640000650a000049
:1036c40000430000545200004c5f000050410000d1
:1036d400524d00003a200000736200005365000060
:1036e4006e6400004d6500007373000061670000a4
:1036f4006500000043540000524c00005f5000007d
:10370400415200004d3a0000207300006243000063
:10371400747200006c50000061720000616d000062
:103724006574000065720000734400006563000066
:103734006f640000650a000000490000676e000025
:103744006f72000065640000204300006f6e00008b
:10375400747200006f6c0000205000006172000061
:10376400616d00006574000065720000730a00005a
:10377400004300006f6e000066690000677500007a
:103784007265000064200000436f00006e74000046
:10379400726f00006c200000506100007261000034
:1037a4006d65000074650000727300000a0000007b
:1037b40043540000524c00005f500000415200008e
:1037c4004d3a000020730000624200006173000063
:1037d4006963000052650000706c000079450000c8
:1037e4006e6300006f640000650a0000004300007f
:1037f400464700005f520000415700005f4300004d
:103804004d4400003a20000073620000436600004b
:103814006752000061770000436f00006e7400007f
:10382400726f00006c440000656300006f64000068
:10383400650a0000004300006f6e00006669000026
:10384400677500007265000064200000526100008a
:1038540077200000436f00006d6d0000616e000072
:10386400640a000000430000464700005f52000065
:10387400415700005f4300004d4400003a2000001f
:10388400736200004261000073690000635200002b
:10389400657000006c790000456e0000636f0000e5
:1038a400646500000a00000043460000475f000012
:1038b40052410000575f0000434d0000443a0000ad
:1038c4002073000062530000656e0000644d000028
:1038d4006573000073610000676500000043000029
:1038e400464700005f4300004f4e00005452000062
:1038f4004f4c00003a200000736200004366000051
:10390400674300006f6e0000747200006f6c00006b
:1039140044650000636f0000646500000a00000055
:10392400436f00006e660000696700007572000056
:1039340065640000204300006f6e00007472000094
:103944006f6c0000204300006f6d00006d6100008b
:103954006e6400000a00000043460000475f000058
:10396400434f00004e540000524f00004c3a0000f8
:10397400207300006242000061730000696300006c
:1039840052650000706c0000794500006e63000011
:103994006f640000650a0000004300004647000011
:1039a4005f4300004f4e0000545200004f4c000093
:1039b4003a20000073620000536500006e6400004a
:1039c4004d6500007373000061670000650000002e
:1039d40053450000545f0000434f00004e54000064
:1039e400524f00004c3a0000207300006253000064
:1039f40065740000436f00006e740000726f000075
:103a04006c440000656300006f640000650a0000f8
:103a140000410000636300006570000074650000ed
:103a240064200000436f00006e740000726f000099
:103a34006c200000436f00006d6d0000616e00009b
:103a4400640a000000530000455400005f43000076
:103a54004f4e0000545200004f4c00003a2000002a
:103a64007362000042610000736900006352000049
:103a7400657000006c790000456e0000636f000003
:103a8400646500000a00000053450000545f000014
:103a9400434f00004e540000524f00004c3a0000c7
:103aa4002073000062530000656e0000644d000046
:103ab4006573000073610000676500000053000037
:103ac400455400005f4300004f4e00005452000074
:103ad4004f4c00003a200000736200005365000060
:103ae400744300006f6e0000747200006f6c00007d
:103af4005769000074680000546900006d65000097
:103b040073740000616d0000704400006563000080
:103b14006f640000650a0000005200004157000075
:103b24005f4300004f4d00004d4100004e44000033
:103b34003a200000736200005261000077430000e5
:103b44006f6e0000747200006f6c0000446500002a
:103b5400636f0000646500000a0000004163000018
:103b6400636500007074000065640000205200006a
:103b740061770000204300006f6d00006d6100005c
:103b84006e6400000a00000052410000575f00000c
:103b9400434f00004d4d0000414e0000443a0000e8
:103ba400207300006242000061730000696300003a
:103bb40052650000706c0000794500006e630000df
:103bc4006f640000650a00000052000041570000c5
:103bd4005f4300004f4d00004d4100004e44000083
:103be4003a20000073620000536500006e64000018
:103bf4004d650000737300006167000065000000fc
:103c040053450000545f00004e410000564d000033
:103c14004f440000453a0000207300006253000046
:103c2400657400004e610000764400006563000086
:103c34006f640000650a0000005300004554000052
:103c44005f4e0000415600004d4f00004445000007
:103c54003a200000736200004261000073690000b2
:103c640063520000657000006c790000456e00002e
:103c7400636f0000646500000a0000005345000003
:103c8400545f00004e410000564d00004f440000b8
:103c9400453a00002073000062530000656e000086
:103ca400644d0000657300007361000067650000e7
:103cb400004100006363000065700000746500004b
:103cc400642000004e610000762000004d6f00006b
:103cd4006465000020250000730a0000004900000c
:103ce400676e00006f72000065640000204e0000e3
:103cf40061760000204d00006f6400006520000024
:103d0400257300000a000000556e00006b6e000071
:103d14006f7700006e200000636f00006d6d00007f
:103d2400616e0000640a0000005500006e6b000024
:103d34006e6f0000776e0000206300006f6d00005e
:103d44006d6100006e6400003a20000073620000a0
:103d54004261000073690000635200006570000056
:103d64006c790000456e0000636f0000646500001c
:103d74000a000000534200005f5800005858000039
:103d8400583a00002073000062530000656e000082
:103d9400644d0000657300007361000067650000f6
:103da400000a00000d5500006e680000616e0000fe
:103db400646c000065640000206d00006573000001
:103dc4007361000067650000203c0000253000009e
:103dd400325800003e0a0000004d000073670000e6
:103de4002025000030320000583a00002045000031
:103df400727200006f720000206300006f640000a4
:103e040065200000256400000a0000004d730000d6
:103e14006720000025300000325800003a200000de
:103e2400737500006363000065730000730a00008b
:103e340000000000204d0000616e00002e200000f4
:103e4400466f00007263000065000000204d000012
:103e5400616e00002e2000004e6f00006e650000b1
:103e640020000000204d0000616e00002e200000a4
:103e7400506f00007320000020000000204d00005f
:103e8400616e00002e200000566500006c200000ca
:103e940020000000204d0000616e00002e20000074
:103ea400526500006c20000020000000204100004a
:103eb400757400006f200000466f000072630000fc
:103ec4006500000020410000757400006f200000b0
:103ed4004e6f00006e6500002000000020410000cd
:103ee400757400006f200000506f00007320000004
:103ef4002000000020410000757400006f200000c5
:103f0400566500006c2000002000000020410000e5
:103f1400757400006f200000526500006c200000e2
:103f240020000000436f00006e740000696e000002
:103f3400756f000075730000004f00006e200000d4
:103f44007265000071750000657300007400000064
:103f5400566500007274000069630000616c000023
:103f6400264800006f720000697a00006f6e00003e
:103f7400746100006c0000004e6f00006e6500006c
:103f8400005600006572000074690000636100005f
:103f94006c000000486f0000726900007a6f000036
:103fa4006e740000616c0000005200006177000034
:103fb400204300006f6e0000747200006f6c0000fc
:103fc400004900006e6300006f720000726500001b
:103fd40063740000204e000061760000204d000054
:103fe4006f64000065000000537400006f700000ef
:103ff40000490000646c000065000000546100008a
:104004006b650000204f000066660000004c000055
:10401400616e000064000000486f000076650000d7
:1040240072000000436f00006e740000726f0000a5
:104034006c6c00006564000000530000696e0000b1
:104044006b6900006e67000000000000256c000032
:10405400642d0000000000000000000000000000cb
:1040640000000000000000000a0a00000d480000e3
:10407400656c00006c6f00002c20000049270000d4
:104084006d2000006861000070700000792000005d
:1040940028530000455200002053000065700000c2
:1040a400203100003120000032300000303900009f
:1040b400290a0000000a00000a0d000048650000fb
:1040c4006c6c00006f2c000020490000276d00007c
:1040d4002068000061700000707900002028000052
:1040e400425400002053000065700000203100009d
:1040f400312000003230000030390000290a00006d
:10410400004400006562000075670000206600003e
:10411400756e000063740000696f00006e2000007b
:104124006973000020610000637400006976000078
:104134006174000065640000206f00006e200000c0
:104144007468000069730000206300006861000067
:104154006e6e0000656c00000a000000494d00000e
:10416400552000006e6f000074200000696e00008e
:1041740069740000696100006c69000073650000e7
:1041840064000000494d0000552000005265000005
:1041940061640000793a0000206200006f61000051
:1041a4007264000020250000730a0000000a000069
:1041b4004f730000636900006c6c000061740000c0
:1041c4006f72000020450000727200006f720000e0
:1041d4000a0a0000000a0000416400006472000042
:1041e400657300007320000045720000726f0000c8
:1041f400720a00000a0000000a5300007461000003
:10420400636b000020450000727200006f720000b2
:104214000a0a0000000a00004d61000074680000f2
:1042240020450000727200006f7200000a0a00004c
:104234000000000046610000696c00006564000035
:10424400207400006f200000656e0000636f0000a2
:104254006465000020680000656c000069200000af
:10426400737400006174000065200000300a0000cf
:1042740000460000616900006c65000064200000d5
:10428400746f0000206500006e6300006f6400001e
:1042940065200000686500006c6900002073000060
:1042a4007461000074650000203100000a00000001
:1042b400496e0000766100006c6900006420000013
:1042c400736f0000757200006365000020660000d3
:1042d4006f720000207300006574000050650000d8
:1042e400726900006f640000696300005374000089
:1042f40061740000650a000000000000536f0000b4
:1043040066740000776100007265000000490000d7
:104314006e760000616c00006964000000460000d5
:10432400726f00006d20000052430000004d000039
:104334006573000073610000676500003a200000a7
:10434400696400002025000030320000582f00006e
:10435400253000003258000020680000616e000023
:10436400646c000065200000256400002f25000017
:10437400642000006c6500006e20000025640000cd
:104384002f250000642000005b00000025300000a1
:1043940032580000200000005d200000435200005d
:1043a4004320000025300000325800000a000000bd
:1043b40000000000204100000ad70000233c000058
:1043c4003200000064000000e80300000200000066
:1043d4000400000010000000400000000001000084
:1043e400000000005365000070200000313100001f
:0c43f400203200003030000039000000d2
:020000040000fa
:10440000881f780000047800010078002c34070031
:104410000001eb0042849800328498006284980086
:104420005284980032149800421498008038210079
:1044300010149800803e2000201498006000b800fe
:10444000600c9800710c9800021498002001200064
:10445000400c980076004000300c9800300020009e
:10446000500c980010c0b30060449800020c780013
:10447000028c9800128c9800228c9800328c980044
:104480004f047800000006000f25b000889fbe0092
:104490008a9fbe008c9fbe008e1f7800800478002b
:1044a000010578000004eb004880980038809800ef
:1044b000688098005880980038109800481098003c
:1044c0008038210090149800803e2000a0149800ad
:1044d0006000b800e00c9800f10c98008814980077
:1044e000e2072000880078000a00780064f00700e6
:1044f0001910900060059800a910900051059800cf
:104500000855980018559800285598003855980077
:10451000485598005855980068559800085d9800cf
:10452000185d9800285d9800385d9800680d980027
:10453000780d9800081598001815980068159800cf
:1045400078159800081d9800181d980078059800a7
:10455000688744000e00780080330700ee86440030
:104560000d0078007d330700098990000200e0000b
:104570000300320021582900100020000200010031
:104580000081eb008081eb00e2b79f00f3b79f0052
:10459000a30220008381440083bf9f00690990002b
:1045a000f90990006fb29700ffb297000400510024
:1045b00085805900753e2000850f5000e08f58001f
:1045c00008003600e2b79f00f3b79f00098990000a
:1045d0000200e00003003200815929001000200091
:1045e000020001000a5190008280fb00706680008a
:1045f000808f500017003200024078009926070093
:1046000000047800ceccbf0096260700881f7800f3
:10461000801f7800405b2900801f780060f62f0023
:104620000f004000feef070009899000e687570061
:104630000200e00004003200c1f62f008f8040002d
:1046400010002000020001000a5090000080fb00d2
:1046500070668800e94090000104e000210032000b
:10466000398090000000e0001e0032005980900068
:104670000000e0001b003200098990000200e00009
:1046800003003200e15b290020002000020001004d
:10469000820c20008fb897000e007800241b0700c2
:1046a0000000e00008003200098990000200e000ec
:1046b00003003200115c29001000200002000100fc
:1046c0000e00780025330700598090008000e90033
:1046d000d18498000000eb00b084980042033200bf
:1046e000e9409000e1cf5000200032004980900066
:1046f0000000e0001d003200698090000000e00032
:104700001a003200098990000200e0000300320024
:10471000315c29002000200002000100820c2000f2
:104720008fb897000d007800011b07000000e00023
:1047300008003200098990000200e0000300320006
:10474000115c290010002000020001000d0078001b
:1047500002330700698090008000e900e18498003e
:104760000000eb00c08498004f00320011002000d0
:104770000e007800f53207000000e00052003a0019
:10478000098990000200e00003003200615c29000a
:104790002000200002000100830c200062e32f00b3
:1047a0000f0141008080eb000e0078008e1a070098
:1047b000000478000000e000e8023a000989900057
:1047c0000200e000ee023200215f290020002000fc
:1047d0000200010008067800ef7094000180fb00e1
:1047e000801f7800a2612900821f780080f62f00c8
:1047f0000f0040008aef070009899000e487570006
:104800000200e00004003200c1f62f008f8040005b
:1048100010002000020001006f70940080057800f5
:104820000b04b200f043b200e0779c000042eb00c2
:1048300043da2f0084f17f000080fb00010020009c
:1048400061005000e0805800f30f5000e08f5800e6
:1048500099023e0000600100360037006700370013
:1048600092003700aa003700d1003700f20037006d
:10487000ad0137009d013700f70137001f013700f8
:1048800039013700430137005d0137000b01370064
:1048900036023700c60137006d0237007901370054
:1048a000500237001c023700798190001000200070
:1048b00002000100110020000e007800a332070062
:1048c0000000e000aeff3200110020000d00780073
:1048d0009e3207000000e00030ff3a000989900096
:1048e0000200e00003003200516029002000200097
:1048f00002000100830c200062e32f000f01410041
:104900008080eb000d007800371a07000000e000ff
:104910009d023a00098990001c0020000200e0007e
:10492000adff3200215f29002000200002000100bd
:10493000a9ff37008042eb0044da2f0005f27f0028
:104940000004eb00b8149800098990000200e00010
:1049500003003200e18a290010002000020001005b
:104960006f7194000274a00043da2f008f81410020
:104970008840780020e92f000f0040000f19070041
:104980000000e000d0043200098990000200e0003d
:1049900003003200318c29000008200002000100d1
:1049a00044da2f0064c07f000004e0002e003200d3
:1049b0000080fb00801f7800cf7294000580fb0010
:1049c000801f7800f0ee2900801f780060f62f002d
:1049d0000f00400012ef070009899000e68757009a
:1049e0000200e000edfe3200c1f62f008f80400093
:1049f0000001200002000100e8fe37008040eb00cb
:104a000040da2f0001f07f006f7194000274a00063
:104a10008f01400020e92f000f004000e718070039
:104a20000000e000d6023200098990000200e00098
:104a3000dbff3200718f2900000820000200010016
:104a4000098990000200e000d5ff3200119329008f
:104a5000100020000200010044da2f0064c07f0033
:104a60000004e000d2ff3a00ef7094000180fb00e8
:104a7000801f780082f02900821f780080f62f00c6
:104a80000f004000e6ee070009899000e487570018
:104a90000200e000c1fe3200c1f62f008f8040000e
:104aa0001000200002000100bcfe37001901900038
:104ab000829f9d00a9019000939f9d0002db2f0023
:104ac0000f0141008040eb0020e92f000f00400063
:104ad000101907000000e000480232000989900028
:104ae0000200e000aeff32006185290000082000ce
:104af00002000100098990000200e000a8ff3200d6
:104b0000018929001000200002000100a4ff3700e5
:104b100051da2f008f80400060e32f000f0040002b
:104b20000e170700800078000000e000a3023200aa
:104b3000098990000200e00003003200419729003b
:104b40000008200002000100c0cfb30044da2f00ab
:104b500000f27f006f7194000274a00043da2f000e
:104b60008f8141008040eb0020e92f000f004000c2
:104b7000921807000000e000a002320009899000ae
:104b80000200e00086ff3200f198290000082000b2
:104b900002000100098990000200e00080ff32005d
:104ba000919c290010002000020001007cff3700ca
:104bb00021dc2f008f80400060e32f000f004000b9
:104bc000ef160700000478000000e000e902320060
:104bd000098990000200e00003003200b16f290053
:104be0000008200002000100c0cfb30042da2f000d
:104bf00000f17f006f7194000274a00043da2f006f
:104c00008f8141008040eb0020e92f000f00400021
:104c10006a1807000000e0000903320009899000cb
:104c20000200e0005eff32008175290000082000cc
:104c3000020001005aff370081db2f008f80400007
:104c400060e32f000f004000e21607000000e000c4
:104c5000b3023200098990000200e0000300320034
:104c600011c729000008200002000100c0cfb300d6
:104c700044da2f0000f27f006f7194000274a000ec
:104c800043da2f008f8141008040eb0020e92f00a4
:104c90000f004000491807000000e0001a0232002f
:104ca000098990000200e0003dff3200e1ca2900be
:104cb000000820000200010039ff370061df2f00eb
:104cc0008f80400060e32f000f0040006318070052
:104cd0000000e00032ff3a00d0779c000989900084
:104ce0000200e0002eff320061df2f008f804000c5
:104cf000100020000200010029ff37000a50900038
:104d0000e54f5000ff033200d0cfb30045da2f004b
:104d100080f27f000000eb00b01498000b00e00070
:104d20001fff32006f7194000274a00043da2f005d
:104d30008f8141008040780020e92f000f00400063
:104d40001e1807000000e00070043200098990007e
:104d50000200e00012ff320051d2290000082000ba
:104d6000020001000eff37000000eb00b0149800b5
:104d70000b00e000d2023a00098990000200e00036
:104d800007ff3200f16e2900100020000200010030
:104d900003ff37000a509000e74f50003502320001
:104da000d0cfb30045da2f0080f27f000000eb0087
:104db000b01498000b00e000f9fe32006f7194000f
:104dc0000274a00043da2f008f81410080407800f8
:104dd00020e92f000f004000f81707000000e00056
:104de000d8023200098990000200e000ecfe320097
:104df00061dc29000008200002000100e8fe370005
:104e000091da2f008f80400060e32f000f004000f8
:104e1000fd1607000000e00007023200098990003b
:104e20000200e0000300320091bf290000082000ca
:104e300002000100c0cfb30043da2f0080f17f00f1
:104e40006f7194000274a00043da2f008f8141003b
:104e50008040eb0020e92f000f004000d71707002b
:104e60000000e00074013200098990000200e000b7
:104e7000cbfe320051c329000008200002000100cf
:104e8000c7fe3700298990000200e000fd023200d1
:104e90000f7c94000804e000b9023a0061de2f00a4
:104ea0008f8040000000eb00020001008001eb0059
:104eb00062de2f000f0141008840780020e92f00ba
:104ec0000f0040002e1707000000e000de02320055
:104ed000098990000200e000b1fe320061b42900af
:104ee0000008200002000100adfe3700c1da2f00eb
:104ef0008f80400060e32f000f0040004316070042
:104f0000000478000000e0000f03320009899000df
:104f10000200e000a2fe3200d17829000008200043
:104f2000020001009efe370041db2f008f80400011
:104f300060e32f000f004000b9160700000478005e
:104f40000000e0004d043200098990000200e000fa
:104f500003003200819e29000008200002000100a9
:104f6000c0cfb30045da2f0080f27f006f7194004c
:104f70000274a00043da2f008f8141008040eb00d3
:104f800020e92f000f0040008c1707000000e00010
:104f900038013200098990000200e00080fe3200f2
:104fa00061a2290000082000020001007cfe3700f9
:104fb00071da2f008f80400060e32f000f00400067
:104fc000e9150700800078000000e00023043200ab
:104fd000098990000200e0000400320011622900fb
:104fe000000820000200010009899000c0cfb30032
:104ff00045da2f0080f27f001900e0001403320030
:105000000200e0000300320041642900100020008b
:10501000020001006f7194000274a00043da2f00b7
:105020008f8141008040eb0020e92f000f004000fd
:10503000621707000000e0001403320009899000a5
:105040000200e00056fe32008167290000082000bf
:105050000200010052fe37000a5490008041eb002c
:1050600042da2f0003f17f0061da2f008f804000c9
:1050700060e32f000f004000ef150700800078006c
:105080000000e0002e043200098990000200e000d8
:105090000300320021e02900000820000200010086
:1050a000c0cfb30044da2f0000f27f000000eb0015
:1050b000b01498000b00e000d7033a0045da2f0047
:1050c000e5c27f000504e00084023a0060da2f00a8
:1050d00060c07f0000559800e2230700801f780021
:1050e000b2e52900821f780080f62f000f004000f3
:1050f0004bed070009899000e48757000200e000ab
:1051000027fe3200c1f62f008f80400010002000e3
:105110000200010022fe37001a310700000178006a
:105120008040eb0020e92f000f00400053170700dc
:105130000000e000e5003200098990000200e00074
:1051400017fe320001802900000820000200010043
:10515000098990000200e00011fe3200c18329009d
:1051600010002000020001000dfe37008041eb001e
:1051700042da2f0003f17f006f7194000274a000e7
:1051800043da2f008f8141008040eb0020e92f009f
:105190000f004000091707000000e000c4003200c3
:1051a000098990000200e000090032009194290072
:1051b0000008200002000100098990000200e000c0
:1051c0000300320041962900100020000200010077
:1051d000198890000000e00001003200000001008a
:1051e000ffff37000a509000e54f50005f03320088
:1051f000d0cfb30045da2f0080f27f000000eb0033
:10520000b01498000b00e000e5fd32006f719400cf
:105210000274a00043da2f008f81410080407800a3
:1052200020e92f000f004000e41607000000e00016
:10523000c4003200098990000200e000d8fd32006d
:1052400051d229000008200002000100d4fd3700df
:10525000398990000200e000160332000f7c9400b0
:105260000804e000d2023a00c1db2f008f8040002a
:105270000000eb00020001008001eb00c2db2f0008
:105280000f0141008840780020e92f000f00400006
:10529000f01507000000e000f702320009899000d5
:1052a0000200e000befd320021a829000008200015
:1052b00002000100bafd3700098990000200e000f9
:1052c0000300320061e8290000082000020001000c
:1052d000e0cfb30045da2f0080f27f006f719400b9
:1052e0000274a0008f8142008040eb0020e92f0073
:1052f0000f004000b11607000000e0002b00320054
:10530000098990000200e0000300320071e92900e1
:1053100000082000020001006f7194000280fb0071
:10532000801f780033ed2900831f780080f62f005e
:105330000f004000baec070009899000e48757008d
:105340000200e00096fd3200c1f62f008f80400081
:10535000100020000200010091fd37000e007800cf
:10536000fe2f0700098990000200e00056fd320080
:10537000a15d2900000120000200010052fd37005c
:105380000206780014fd37000d007800f32f0700a7
:10539000098990000200e00080fc3200a15d290034
:1053a00000012000020001007cfc37006660b900ab
:1053b00000004700421f200021e92f008f8040009d
:1053c000db1707000000e000d3ff320009899000de
:1053d0000200e000d0ff3200c1eb290000082000ed
:1053e00002000100ccff37007981900001007800b5
:1053f00002000100e9409000bafc37006660b90085
:1054000000004700820c200021e92f008f8040001f
:10541000c71707000000e000b6fd320009899000c0
:105420000200e0005efd32006187290000082000d4
:1054300002000100affd37006660b90000004700c0
:10544000820c200021e92f008f804000b817070050
:105450000000e00052fd3200098990000200e000e7
:105460004ffd320061c52900000820000200010044
:105470004bfd37006660b90000004700820c200039
:1054800021e92f008f804000a91707000000e000ed
:1054900043fd3200098990000200e00040fd320027
:1054a00071a4290000082000020001003cfd370023
:1054b0006660b90000004700820c200021e92f003f
:1054c0008f8040009a1707003bff37006660b900e5
:1054d00000004700820c200021e92f008f8040004f
:1054e000931707000000e00019ff320009899000bf
:1054f0000200e0002afd320011822900000820008d
:105500000200010012ff37006660b900000047008a
:10551000820c200021e92f008f80400084170700b3
:105520000000e0001efd3200098990000200e0004a
:105530001bfd3200f1cc2900000820000200010010
:1055400017fd37006660b90000004700820c20009c
:1055500021e92f008f804000751707000000e00050
:105560000ffd3200098990000200e0000cfd3200be
:1055700061d42900000820000200010008fd370066
:105580006660b90000004700820c200021e92f006e
:105590008f804000661707000000e00028fd320001
:1055a000098990000200e000fdfc320071912900a1
:1055b000000820000200010021fd370052da2f0010
:1055c00062c07f00634060002055980043da2f00de
:1055d00081f17f006f7194000274a00043da2f0004
:1055e0008f8141008040eb0020e92f000f00400038
:1055f000f21507000000e00060fd3a006660b900a7
:1056000000004700820c200021e92f008f8040001d
:10561000471707000000e0005efd32000989900096
:105620000200e000defc3200f19a290000082000b0
:105630000200010057fd370095da2f00e5c27f0018
:1056400045fd9800a1da2f00e1c07f0051fd9800d0
:1056500042da2f0000f17f00098990000200e0008b
:10566000f7fd3200d1c12900100020000200010026
:10567000f3fd370021dd2f008f80400060e32f0015
:105680000f004000c71407000000e0000e003200c9
:10569000098990000200e00003003200f1d82900df
:1056a0000008200002000100c0cfb30042da2f0042
:1056b00000f17f000000eb00b01498000b00e00048
:1056c000b7fc3200bdfd37001faa950024159800d5
:1056d000afaa950035159800bfa895004115980010
:1056e0004fa9950052159800c014980043da2f0076
:1056f00080f17f00098990000200e000abfd3200dc
:1057000001db290010002000020001000000eb0076
:10571000b01498000b00e000a1fc3200a7fd370098
:1057200081db2f00e1c07f00015d980092db2f003c
:1057300062c17f00125d9800a3db2f00e3c17f00f0
:10574000235d9800b4db2f0064c27f00345d9800b5
:1057500045da2f0080f27f00098990000200e00006
:1057600045fd320021c9290010002000020001007f
:1057700041fd370024dc2f0064c07f0061416000e0
:1057800012559800e14f51003c003a0099009000fa
:105790003fa095000100600010059800a90090004e
:1057a0004fa09500010060002005980035dc2f0017
:1057b00065c07f000004e00002003a00024078006b
:1057c00082f27f000081fb0072059800813e20007c
:1057d000110009008200d8008000fd000c00460086
:1057e000090040002fa19500528098007981900017
:1057f0000c0078000200010043da2f0088f17f00de
:10580000098990000200e000fafc32005171290081
:1058100010002000020001006f7194000274a000cb
:1058200043da2f008f8141008040eb0020e92f00f8
:105830000f004000611507000000e000f7fc3a008f
:105840006660b90000004700820c200021e92f00ab
:105850008f804000b61607000000e00050fc3200c8
:10586000098990000200e0004dfc320051772900c8
:10587000000820000200010049fc37000c0046002f
:1058800009004000588098007805980079819000c0
:10589000880078000c0078000200010045da2f0033
:1058a00088f27f00098990000200e000d1fc3200fc
:1058b000717329001000200002000100cdfc3700a8
:1058c0008040780045da2f0080f27f006f719400ed
:1058d0000274a0008f81420020e92f000f004000d9
:1058e000361507000000e00007003200098990002b
:1058f0000200e0002afc3200616b29000008200051
:10590000020001001cfd37006660b900000047007e
:10591000820c200021e92f008f80400084160700b0
:105920000000e00014fd3200098990000200e00050
:105930001bfc3200516d290000082000020001000c
:105940000dfd37006660b90000004700820c2000a2
:1059500021e92f008f804000751607000000e0004d
:105960000ffc3200098990000200e0000cfc3200bc
:1059700071de2900000820000200010008fc370049
:1059800061de2f008f80400060e32f000f00400099
:10599000d91407000000e0001a00320009899000c5
:1059a0000200e00003003200c1b729000008200017
:1059b00002000100c0cfb30043da2f0080f17f0066
:1059c0006f7194000274a00043da2f008f814100b0
:1059d0008040eb0020e92f000f004000f714070083
:1059e0000000e0002e003200098990000200e00073
:1059f000ebfb3200a1bd29000008200002000100dd
:105a0000e7fb37002989900061de2f008f8040007e
:105a100010002000020001000000e0004100320000
:105a200000c0eb0045da2f0080f27f00098990006a
:105a30000200e000e2ff3200f1b92900000120007d
:105a400002000100deff37006660b9000000470079
:105a5000820c200021e92f008f80400034160700bf
:105a60000000e000cefb3200098990000200e00057
:105a7000cbfb320031b629000008200002000100f3
:105a8000c7fb3700098990000200e000c4fb320028
:105a9000d1b129000001200002000100c0fb370045
:105aa0006660b90000004700820c200021e92f0049
:105ab0008f8040001e1607000000e000b8fb320097
:105ac000098990000200e000b5fb320031b62900e0
:105ad0000008200002000100b1fb370063da2f004c
:105ae00063c07f005f210700801f780014e7290052
:105af000841f780080f62f000f004000c8ea0700de
:105b000009899000e48757000200e000a4fb3200fe
:105b1000c1f62f008f80400010002000020001001d
:105b20009ffb370041da2f0080f07f000989900049
:105b30000200e000a2ff3200b1bb290010002000eb
:105b4000020001009eff3700990090006f909500c1
:105b500001006000e0979d00a90090007f909500f3
:105b600001006000f0979d002908900000000100ee
:105b7000e1ee2f008f8040003e000900ba18780047
:105b8000e107b100ea07b100ef91950083bf9e00e5
:105b90007f92950094bf9e000101780088407800b4
:105ba00020e92f000f0040004c1f07000000e0001c
:105bb00018003200098990000200e0000300320062
:105bc000517a29000008200002000100ff92950090
:105bd000851f78005f909500801f7800e17d290087
:105be000811f780060f62f000f0040008cea07004c
:105bf00009899000e68757000200e00068fb320048
:105c0000c1f62f008f80400010002000020001002c
:105c100063fb37006660b90000004700820c20007b
:105c200021e92f008f804000c11507000000e0002f
:105c3000e6ff3200098990000200e000e3ff320035
:105c4000917c29000008200002000100dfff3700de
:105c50000200e000effc3200c165290000012000d5
:105c6000020001006f7194000274a00043da2f005b
:105c70008f8141008040eb0020e92f000f004000a1
:105c80004e1407000000e000ecfc3a006660b9002a
:105c900000004700820c200021e92f008f80400087
:105ca000a31507000000e0003dfb320009899000c9
:105cb0000200e0003afb3200a16929000008200040
:105cc0000200010036fb37006660b90000004700a3
:105cd000820c200021e92f008f80400094150700de
:105ce0000000e0002efb3200098990000200e00075
:105cf0002bfb3200018e2900000820000200010069
:105d000027fb3700a1dc2f008f80400060e32f00cd
:105d10000f0040000a1307000000e0000e003200f0
:105d2000098990000200e00003003200a1ce2900a2
:105d30000008200002000100c0cfb30042da2f00ab
:105d400000f17f000000eb00b01498000b00e000b1
:105d500013fb3200f3fb37005fa29500640d98003f
:105d6000efa29500750d9800ffa095000115980011
:105d70000fa9950012159800c014980043da2f005f
:105d800080f17f00098990000200e000e1fb320011
:105d9000b1d0290010002000020001000000eb003b
:105da000b01498000b00e000fdfa3200ddfb370074
:105db000c1db2f008f80400060e32f000f00400008
:105dc000561307000000e0001a0032000989900015
:105dd0000200e0000300320081ab2900000820002f
:105de00002000100c0cfb30043da2f0080f17f0032
:105df0006f7194000274a00043da2f008f8141007c
:105e00008040eb0020e92f000f004000eb1307005b
:105e10000000e0002e003200098990000200e0003e
:105e2000dffa3200e1af2900000820000200010083
:105e3000dbfa370039899000c1db2f008f804000ea
:105e400010002000020001000000e0003e003200cf
:105e500000c0eb0045da2f0080f27f000989900036
:105e60000200e000e2ff320051ad290000012000f5
:105e700002000100deff37006660b9000000470045
:105e8000820c200021e92f008f8040002815070098
:105e90000000e000c2fa3200098990000200e00030
:105ea000bffa3200f1a92900000820000200010019
:105eb000bbfa3700098990000200e000b8fa32000e
:105ec00021a629000001200002000100b4fa3700d9
:105ed0006660b90000004700820c200021e92f0015
:105ee0008f804000121507000000e000acfa32007d
:105ef000098990000200e000a9fa3200f1a9290006
:105f00000008200002000100a5fa37006660b90011
:105f100000004700820c200021e92f008f80400004
:105f2000031507000000e0009dfa32000989900087
:105f30000200e0009afa320061d429000008200033
:105f40000200010096fa370041da2f0080f07f004e
:105f5000098990000200e000a5ff320081ae29000f
:105f60001000200002000100a1ff3700a1dd2f007a
:105f70008f80400060e32f000f00400031120700c7
:105f80000000e0000e003200098990000200e000ed
:105f90000300320011d62900000820000200010091
:105fa000c0cfb30042da2f0000f17f000000eb0009
:105fb000b01498000b00e00079fa320093fc37002f
:105fc0005faa9500640d9800efaa9500750d9800e2
:105fd000ffa89500011598000fb1950012159800c3
:105fe000c014980043da2f0080f17f0009899000e7
:105ff0000200e00081fc3200b1d029001000200036
:10600000020001000000eb00b01498000b00e0005b
:1060100063fa32007dfc37006f7194000274a000b7
:1060200043da2f008f8141008040780020e92f0063
:106030000f004000611307000000e0003100320053
:10604000098990000200e0001cfc3200f1e1290007
:10605000000820000200010018fc370072da2f004f
:1060600062c17f000280fb00800c780043da2f00c1
:1060700081f17f0009899000dffb37002f989500a0
:106080000000e00001003200a01498003f98950045
:106090000000e000010032009014980019119000f7
:1060a00062059800a91190005305980044da2f006a
:1060b00008f27f006a009000801f7800da009000ec
:1060c000811f780092a02900821f780060f62f00bf
:1060d0000f00400052e9070009899000e687570049
:1060e0000200e00004003200c1f62f008f80400063
:1060f0001000200002000100b8149800c814980095
:106100009afb37006660b90000004700820c20004f
:1061100021e92f008f804000851407000000e00077
:10612000e6fb3200098990000200e000e3fb320048
:1061300001e429000008200002000100dffb370015
:1061400062da2f0062c07f00804f54006a00320084
:10615000e34f50003a0032002c003e00e14f500067
:106160001e00320013003600e14f540005003200db
:10617000e44f540003003200d0cfb30044da2f00c4
:1061800000f27f0089109000703e2000808f500048
:10619000c6fb3e00a0cfb30041da2f0080f07f00a5
:1061a0000000eb00b01498000b00e000c3fb3200cd
:1061b00099ff3700e14f5400bcfb3200d0cfb30051
:1061c00043da2f0080f17f000000eb00b01498004c
:1061d0000b00e000b9fb32008fff37000804e0003d
:1061e000b2fb3200e74f5400b0fb3200d0cfb30017
:1061f00045da2f0080f27f000000eb00b014980019
:106200000b00e000adfb320083ff3700e54f50008c
:106210002d00320024003900e74f500014003200f6
:10622000d0cfb30041da2f0080f07f000000eb00f8
:10623000b01498000b00e000a0fb320076ff37009e
:10624000e74f5400ddff3e008800fb0010002000f7
:106250000100dd00600fb200d8ff32000000eb004b
:10626000b01498000b00e00094fb32006aff370086
:10627000e14f540003003200d0cfb30042da2f00c8
:1062800000f17f0021159800311598004115980004
:10629000511598000000eb00b01498000b00e000ce
:1062a00086fb32005cff370065405400e14f500030
:1062b000ceff3e000000eb00b01498000b00e000a1
:1062c0007efb320054ff3700e64f540011003200cd
:1062d000e44f54000f003200d0cfb30042da2f0059
:1062e00000f17f000000eb00b01498000b00e0000c
:1062f00072fb320048ff370043da2f0081f17f0044
:106300000000eb00b01498000b00e0006bfb3200c3
:1063100041ff37008000eb00610d9800710d98007f
:1063200001159800111598002a589000e14f50006f
:1063300002003a004a1a9000041598003a5890005a
:10634000e24f500002003a008a2a9000151598008a
:10635000c11498000000eb00b01498000b00e0009e
:1063600056fb32002cff3700889fbe008a9fbe007c
:1063700080047800010478002008900000000100eb
:10638000885190000382fb00e3cf5100930032005c
:106390002a003600e5cf5100b20032008d003100f6
:1063a00099109000e18f40000300320039109000f6
:1063b000808f5000b10036000380fb00800f520038
:1063c000030032000000eb00801498008851900018
:1063d000285090008080fb000118a30024003200a8
:1063e000082890000000e900fa002000ed0f50009e
:1063f0001f003e006180600020003a0080057800a8
:1064000080027800e3cf51004b003200e3cf51000f
:106410005b003e00e1cf510079003e000040eb0000
:10642000605498003054980040549800505498009c
:106430004f05be004f04be0000000600e1cf510032
:10644000af003200e2cf5100dbff3a008002eb00e8
:10645000b514980039089000650050000829900094
:10646000800f5100be003c0088519000d2ff3700e1
:106470000085eb0061806000e0ff3200282a900078
:10648000382b9000c82b9000d82a90008400e90097
:106490008005eb0040092000808f500006003e0080
:1064a00062092000040051007400b90011000900c5
:1064b0000200d800800578000500e90044092000aa
:1064c000840f500006003e006209200005005100c4
:1064d0007400b900110009000200d8008085550041
:1064e0000600e9008002eb00840f500006003e0029
:1064f00062092000060051007400b9001100090073
:106500000200d8008002ea008700e900400920006c
:10651000808f5000bbff3e00620920000700510041
:106520007400b900110009000200d8008082420006
:10653000e3cf5100b5ff3a0020c0b300605498008b
:1065400010c0b30030549800405498005354980041
:1065500008289000d908900001005000101c9800f5
:106560000000eb006014980070149800001c980064
:106570004f05be004f04be0000000600afff37000d
:10658000e5cf5100400032002e00310010c0b300b2
:10659000305498004054980030c0b30050549800d4
:1065a0000a00e0009900340020c0b3006054980055
:1065b0001a1c9800651498007b1498000000eb00ea
:1065c000001c98004f05be004f04be0000000600ee
:1065d0009aff3700e6cf510077ff3a000000eb004a
:1065e000b01498008828900049089000808f5000cf
:1065f0009dff3c0013c0b300035498006eff3700aa
:1066000020c0b3006054980010c0b300305498000c
:106610004054980030c0b30050549800b90c90001a
:10662000191c98000000eb0060149800701498008a
:10663000001c98004f05be004f04be00000006007d
:106640007eff3700e6cf510052003200e7cf510005
:1066500072ff32004f05be004f04be00000006006e
:1066600076ff370099109000e18f40002d00320036
:1066700039109000808f50002a003e0063c0b300a4
:10668000035498004cff370028589000505498004d
:1066900008109000001c98000a00e000640034001c
:1066a00020c0b300605498001a1c9800085890004d
:1066b00030549800e14f5000500032000500e000d7
:1066c00023003a0068089000601498001858900061
:1066d00040549800e14f5000410032000b00e000b0
:1066e0002600320010c0b300405498007b1498007c
:1066f0004f05be004f04be00000006004fff3700ec
:1067000099109000e18f40002bff3200391090006b
:10671000808f500028ff3e008041eb00035498001a
:1067200025ff3700a9109000e18f400022ff3200c2
:1067300049109000808f50001fff3e0043c0b300ff
:106740000354980008289000101498001aff37008e
:1067500010c0b3003054980065149800dbff370078
:10676000335c98001214980043c0b300035498009f
:10677000b5149800885190000fff370078089000fa
:10678000701498004f05be004f04be0000000600c4
:106790002aff370020c0b3006054980010c0b30037
:1067a000305498004054980030c0b30050549800c2
:1067b00008289000d908900001005000101c980093
:1067c000651498007b1498000000eb00001c9800f2
:1067d0004f05be004f04be000000060017ff370043
:1067e0007808900000804500701498004f05be00a6
:1067f0004f04be000000060010ff3700680890003c
:106800000080420060149800b0ff370020c0b30041
:106810006054980018109000101c9800651498009f
:106820007b1498000000eb00001c980065ff370007
:10683000385890006054980018109000101c980070
:106840009aff370080017800f008900060089000ff
:1068500002004000e0804800e0099800f10998003b
:106860000310900000004100801198002310900058
:10687000e10f400003003200c3109000810f500070
:1068800009003e0093109000e18f400005003200a7
:1068900033109000808f500002003600000041004d
:1068a000b01198000000060001004100c0119800de
:1068b000f4ff37000000fa000000eb00607d880064
:1068c00010022000407d8800407d8000507d8800bf
:1068d00062cd20006000b8000089be0062cd2000bb
:1068e0006000b8002001980031019800e2cd20003e
:1068f0006000b8000089be00e2cd20006000b80052
:1069000020019800310198006000b800b072880042
:10691000c17288006000b800d0728800e1728800ff
:1069200082d420006000b800102998002129980026
:10693000e1ce20000000eb0080087800e1ce2000ce
:106940001000200090009800e2ce20006000b80007
:106950005011980061119800e2ce20006000b8004c
:106960003019980041199800e2ce20006000b8006c
:106970005001980061019800e2ce20006000b8004c
:106980001009980021099800e2ce20006000b800ac
:106990007019980001219800e2ce20006000b80034
:1069a0001021980021219800e2ce20006000b8005c
:1069b000302198004121980081d420000000eb0094
:1069c0008008780081d420001000200090009800fa
:1069d00081d420000000eb00a000980082d42000a9
:1069e0006000b800501198006111980082d4200016
:1069f0006000b800500998006109980082d4200016
:106a00006000b800700998000111980082d420003d
:106a10006000b800101198002111980082d4200065
:106a20006000b800301198004111980082d4200015
:106a30006000b800301998004119980082d42000f5
:106a40006000b800500198006101980082d42000d5
:106a50006000b800100998002109980082d4200035
:106a60006000b8007021980001299800e1ce200054
:106a70000000eb0080087800e1ce2000100020002c
:106a800090009800e2ce20006000b80050119800fd
:106a900061119800e2ce20006000b8005009980013
:106aa00061099800e2ce20006000b80070099800eb
:106ab00001119800e2ce20006000b800101198008b
:106ac00021119800e2ce20006000b800502198000b
:106ad00061219800e2ce20006000b80050199800b3
:106ae00061199800c1df20000000eb0080087800e9
:106af000c1df20001000200090009800c2df2000bd
:106b00006000b8005011980061119800c2df2000a9
:106b10006000b8005009980061099800c2df2000a9
:106b20006000b8007009980001119800c2df2000d1
:106b30006000b800101198002111980021da20009f
:106b40000000eb008008780021da2000100020000f
:106b50009000980022da20006000b80050119800e0
:106b60006111980022da20006000b80050099800f6
:106b70006109980022da20006000b80070099800ce
:106b80000111980022da20006000b800101198006e
:106b900021119800df2a07000000eb00b07c88007c
:106ba0000000eb00a07c88007a1807000080fa0043
:106bb000000006000c00fa00417d8000507d80003e
:106bc000808f50000a003a00707d80000000e800cd
:106bd000707d8800717d8000300f8500808f5000af
:106be00007003400300f8500707d880004003700f6
:106bf0000000eb00707d8800407d8000507d8800a3
:106c0000407d80006f006000e20f50000a003a00f3
:106c1000807d80000000e800807d8800817d80000c
:106c2000300f8500808f500005003400300f850044
:106c3000807d8800020037000000eb00807d880026
:106c40007018070010079800b07c80000000e0007a
:106c5000050032001e0090000000e00002003a0033
:106c600010002000100798001e00900050079800a8
:106c7000de009000e18f5000080032005e009000be
:106c8000e20f50000100320007003700caa2a8003e
:106c900010002000b07c8800a4003700caa2a80021
:106ca00010002000b07c88000000eb00000f78008e
:106cb000417d8000000f2000808060004107980027
:106cc00000022000ce009000808f500008003200ab
:106cd00000042000ce009000808f5000120032008f
:106ce0004e009000f00f50002800320034003700b2
:106cf000407a8000517a8000d2cc2c00c3f423006b
:106d0000efeb07000000e00001003c002c00370022
:106d1000407d8000ef0060000004200000807000d3
:106d2000407d880026003700717d8000200f85009f
:106d3000808f500010003d00407a8000517a800022
:106d4000d2cc2c00c3e42300dfeb07000000e000fe
:106d5000010035001a003700407d8000ef00600020
:106d60000002200000807000407d8800100020009c
:106d7000000f780012003700407d80006f00600037
:106d80000040a000407d88000d003700407a800060
:106d9000517a8000d2cc2c00c3e42300caeb070058
:106da0000000e0000100350005003700407d800054
:106db000ef0060000002200000807000407d88002d
:106dc0001e00e00026003200417d8000000f200000
:106dd0008080600000022000808f500020003a0078
:106de000407d80006f00600030079800be0090007a
:106df000e28f5000110032003e009000e20f500080
:106e000004003e00be009000e18f500008003200f8
:106e1000130037003e009000e40f50000e003200d7
:106e2000be009000e88f50000b0032000c003700cd
:106e300020022000407d880009003700817d80000d
:106e4000100f8500808f50000500340040022000a4
:106e5000407d88000200370020022000407d88002d
:106e6000417d800020022000808f500006003a0003
:106e7000817d8000300f8500808f500002003a0035
:106e800010022000407d8800407d8000010f20001e
:106e9000010060002007980000022000ae00900072
:106ea000808f50001500320000042000ae009000da
:106eb000808f5000110032002e009000f00f500023
:106ec000010032001900370081d42000100020009a
:106ed00080087800e1ce20001000200080087800b3
:106ee00021da20001000200080087800c1df200097
:106ef00010002000800878000c00370081d42000aa
:106f00000000eb0080087800e1ce20000000eb00dc
:106f10008008780021da20000000eb00800878006b
:106f2000c1df20000000eb00800878000080fa003c
:106f3000000006000c00fa00000f78001e00780028
:106f40006f0f6000407d8000010f20000100600095
:106f5000f00f5000030032000080eb002007980083
:106f600076003700407d80006f0060009e0f50006b
:106f700003003a000000eb00200798006f00370084
:106f8000b07c80000000e000160032001e00780097
:106f9000300798003e009000e40f500007003200d8
:106fa0003e009000e80f5000040032003e009000c8
:106fb000e20f5000040032000a0037000000eb002e
:106fc000200798005d003700407d80006f00600062
:106fd000e10f500003003a000000eb00200798008a
:106fe00056003700407d80006f0060001007980059
:106ff0001e009000e20f5000290032001e00900099
:10700000e20f500004003e001e009000e10f50000f
:1070100011003200440037001e009000e40f5000c1
:10702000380032001e009000e80f500001003200ce
:107030003d0037001e007800e10f500001003200d3
:107040000200370010012000407d88000080eb0026
:1070500020079800390037001e007800400798008c
:107060004e009000e20f5000040032004e009000ed
:10707000e80f500004003200060037002001200015
:10708000407d88002b00370080012000407d880073
:10709000280037000080eb00200798002700370009
:1070a0001e007800500798005e009000e10f50002d
:1070b000040032005e009000e40f50000400320033
:1070c0000d00370010012000407d880019003700b6
:1070d000817d8000100f8500808f500003003400f8
:1070e00040012000407d8800120037001000200081
:1070f00020079800110037000080eb00200798005f
:107100000e0037001e0078000000e900e10f50007b
:1071100002003e0020012000407d88000080eb003e
:1071200020079800050037000080eb00200798003a
:10713000020037000000eb00200798002e009000ae
:107140000080fa00000006000c00fa00889fbe00d4
:107150006000b80040079800510798000000200028
:1071600001fc230020079800310798000000200050
:1071700001082400008fbe0080d420002000900071
:107180000000e0002100320082d420006000b8003e
:10719000301998004119980082d420006000b8008e
:1071a000500198006101980082d420006000b8006e
:1071b000100998002109980080d420001000900048
:1071c0000000e00004003a0080d4200010007800a5
:1071d0000000e00006003a00c0798000d17980000c
:1071e00082d420005011980061119800dd00370012
:1071f00080d42000e010900050109000e2ce2000db
:107200001019980021199800d600370080d420006a
:10721000100090000000e00004003a0080d420003c
:10722000100078000000e0000a003a000000eb00c7
:10723000c07c8800c0798000d17980002e01900048
:10724000be01900049ea070082d420005011980046
:107250006111980080d42000e01090005010900040
:107260002e019000be01900095ea07000000e000aa
:1072700001003c000500370080d420002e01900062
:10728000be019000521098006310980080d4200036
:10729000e0109000501090004e019000de01900030
:1072a00089ea07000000e000010035000500370012
:1072b00080d420004e019000de0190005210980012
:1072c00063109800c17c8000d07c8000808f5000cb
:1072d0001200320082d420006000b80030199800fb
:1072e0004119980082d420006000b8005001980035
:1072f0006101980082d420006000b8001009980055
:107300002109980082d420006000b8007021980004
:1073100001299800c07c8000d07c8800c07c80005f
:107320000000e0000600320020e62000f01090008f
:1073300060109000b0728800c172880005003700ac
:1073400020e62000d010900040109000b07288001d
:10735000c1728800b0728000c17280001e01be0040
:1073600057ea07000000e00001003c00030037007e
:107370001e00be00b0728800c1728800b07280002a
:10738000c17280004e019000de0190004eea0700bd
:107390000000e00001003500040037004e019000bd
:1073a000de019000b2728800c372880080d4200091
:1073b000e010900050109000b2728000c372800004
:1073c0004ae9070082d4200030019800410198006a
:1073d000f40e8500050f850080d420003019900040
:1073e000c019900080d42000c000900030009000b0
:1073f000d6cc2c00c7dc23006201070082d4200019
:107400003001980041019800f40e8500050f8500b9
:1074100080d4200030199000c019900080d4200042
:10742000cb010700d4cc2c00c5dc2300d2cc2c002f
:10743000c3dc2b0080d42000e702070080d42000aa
:1074400050049000e004900080d42000301190009f
:10745000c01190000000200001f8230023e907007c
:107460000001be000800be0015ea07000000e000b1
:1074700001003c000900370080d42000301190004a
:10748000c01190000000200001f8230017e9070058
:1074900082d42000500198006101980080d420001f
:1074a000e0009000500090006011b80006ea07006c
:1074b0000000e000010035000400370082d4200005
:1074c0006000b800500198006101980080d420004d
:1074d00050029000e002900080d420003011900013
:1074e000c01190000400be0001e9070082d4200012
:1074f000500198006101980080d42000e0009000c5
:1075000050009000e2ce2000101998002119980038
:1075100080d42000c00090003000900082d4200071
:107520003019980041199800b0728000c172800033
:10753000d0728800e1728800c0f92000b00090008d
:1075400020009000c2f920004001980051019800ed
:10755000c0f920001000be00c2f9200020019800f0
:1075600031019800e0ce2000100090000000e00003
:1075700004003a00e0ce2000100078000000e00097
:107580001e003a00e0798000f1798000a29929007c
:1075900093f12b0075e90700e2ce2000501198000e
:1075a00061119800e0ce2000e01090005010900093
:1075b000f2282c0053df2b00c1e907000000e00097
:1075c00001003c000d003700e0ce2000e0109000ec
:1075d00050109000f2282c0053df2300bae9070076
:1075e0000000e0000100350004003700e2ce20007a
:1075f0006000b800501198006111980020e620004a
:10760000f018900060189000b07d8800c17d88005f
:10761000b07d8000c17d800002002000633924001d
:10762000a7e907000000e00001003c00040037006b
:107630000000200061392400b07d8800c17d8800f1
:10764000b07d8000c17d80000200200063392c00e5
:107650009de907000000e00001003500040037004c
:107660000000200061392c00b07d8800c17d8800b9
:10767000b07d8000c17d800023160700b07d8800aa
:10768000c17d880020e62000d000900040009000de
:107690001d160700e2ce2000701998000121980005
:1076a000e0ce2000e010900050109000b27d8000ed
:1076b000c37d80008de80700e2ce200030019800f5
:1076c00041019800e2ce20006000b800102198002f
:1076d00021219800f40e8500050f8500e0ce2000e2
:1076e00030199000c0199000e0ce2000b0010700d2
:1076f000f4282c0055d72300f2282c0053d72b0058
:10770000e0ce200034020700e0ce2000e000900030
:1077100050009000d2cc2c00c3ec230068e9070095
:107720000000e00001003c0005003700e2ce200030
:10773000d0cc2c00c1ec23005001980061019800ce
:10774000e0ce2000e000900050009000d2cc2c0051
:10775000c3ec2b005ce907000000e00001003500ed
:1077600005003700e2ce2000d0cc2c00c1ec2b006d
:107770005001980061019800e0ce2000c000900008
:1077800030009000e2ce2000301998004119980096
:10779000b07d8000c17d8000d07d8800e17d8800c3
:1077a000e0ce2000e000900050009000507e880065
:1077b000617e8800e0ce2000101c9000a01c90008c
:1077c000e0ce2000101a9000a01a9000e0ce200019
:1077d00050199000e01990000400be00e3e8070093
:1077e0000001be000800be0040e807000002be0025
:1077f000e0ce200050019000e00190000400be00a7
:107800003be8070062cd20000089be00e0ce2000ea
:10781000a01890001018900062cd20002001980060
:1078200031019800607a8000717a8000d2cc2c00ff
:10783000c3f4230022e907000000e00001003c003f
:10784000130037006011b8006000b8007924070009
:1078500020e62000d000900040009000aa1507000c
:10786000e2ce2000302198004121980082d42000ef
:107870006000b8001009980021099800e2ce2000ad
:107880006000b80010099800210998000600370030
:1078900060cd200020019000b001900060cd20005c
:1078a0001000be0063240700c0df2000100090001d
:1078b0000000e00004003a00c0df20001000780063
:1078c0000000e0000e003a00207a8000317a80004b
:1078d000d2cc2c00c3e42300a4e807000002be00c1
:1078e000a0798000b17980000001be000400be00d4
:1078f000ffe70700c2df20005011980061119800d7
:1079000020da2000100090000000e00004003a009f
:1079100020da2000100078000000e0000f003a009c
:10792000007a8000117a8000d2cc2c00c3e42300be
:107930008ee807000002be00807980009179800007
:107940000001be000400be00e9e7070001f0a2004c
:1079500022da2000501198006111980020da2000ee
:1079600050119000e0119000c0df2000e010900066
:1079700050109000702407004f04be000080fa00f1
:10798000000006001400fa00889fbe00200798003f
:107990003107980042079800530798006407980041
:1079a00075079800060f9800170f98006e01900059
:1079b000fe0190000e0890009e089000cce70700a2
:1079c0000001be006e009000fe00900025e8070058
:1079d000008fbe002e019000be0190001e00be0070
:1079e00062e807000004be001e01be000000200087
:1079f00001f82300bde707004e019000de01900072
:107a00005ae807000001be000800be00b8e7070002
:107a100020079800310798002e009000be009000cb
:107a20004f04be000080fa00000006000a00fa00c1
:107a3000889fbe00000f7800120798002307980067
:107a400034079800450798001e007800500a9000ff
:107a5000e00a90001e00780030019000c001900004
:107a60000400be0041e807001e0178007001980084
:107a7000010998001e007800100c9000a00c9000e6
:107a80001e00780030029000c00290001e007800b6
:107a900070099000801190000400be0033e80700d8
:107aa0000001be000800be0091e707001e0178003b
:107ab00010099800210998001e007800c00090006d
:107ac000300090001e019000ae01900087e7070093
:107ad0003e019000ce019000e2e707000002be00e8
:107ae0001e00780010119000a01190000400be004c
:107af0001ee807001e01780030099800410998002f
:107b00001e00780070029000800a90001e0078002d
:107b100010099000a00990000400be0074e707005f
:107b20000002be001e00780030099000c0099000dd
:107b30000400be006ee707001e01780050019800a7
:107b4000610198004f04be000080fa0000000600aa
:107b50000a00fa00889fbe00000f78001207980004
:107b60002307980034079800450798001e00780006
:107b7000500a9000e00a90001e007800300190004a
:107b8000c00190000400be00f8e707001e01780065
:107b90007001980001099800907d80000000e900c4
:107ba000907d8800a07d80000000e900a07d880015
:107bb000907d80000000e0002a003c001e0078005c
:107bc000c0009000300090006011b8003ce8070051
:107bd0000000e00001003c00220037001e00780099
:107be000c0009000300090006011b80034e8070039
:107bf0000000e00001003c00120037001e00780089
:107c0000100c9000a00c90001e0078003002900034
:107c1000c00290001e007800700990008011900052
:107c20000400be00d1e707000001be000800be004e
:107c30002fe707001e01780010099800210998001d
:107c4000060037001e007800a00890001008900081
:107c50001e017800100998002109980020002000da
:107c6000907d8800a07d80000000e0002a003c009c
:107c70001e007800c0009000300090006011b80035
:107c800011e807000000e000010035002200370085
:107c90001e007800c0009000300090006011b80015
:107ca00009e807000000e00001003500120037007d
:107cb0001e007800100c9000a00c90001e007800b0
:107cc00030029000c00290001e0078007009900001
:107cd000801190000400be00a4e707000001be0070
:107ce0000800be0002e707001e0178001009980096
:107cf00021099800060037001e007800a0089000b7
:107d0000100890001e0178001009980021099800c1
:107d100050002000a07d88001e007800c000900068
:107d2000300090001e019000ae019000efe60700c9
:107d30003e019000ce0190004ae707000002be001d
:107d40001e00780010119000a01190000400be00e9
:107d500086e707001e017800300998004109980065
:107d60001e00780070029000800a90001e007800cb
:107d700010099000a00990000400be00dce6070096
:107d80000002be001e00780030099000c00990007b
:107d90000400be00d6e607001e01780050019800de
:107da000610198004f04be000080fa000000060048
:107db0000a00fa00889fbe00000f780012079800a2
:107dc0002307980034079800450798001e007800a4
:107dd00050229000e02290001e00780010219000b8
:107de000a02190000400be0060e707001e0178009b
:107df00030299800412998001e007800100c90004e
:107e0000a00c90001e00780030029000c00290008c
:107e10001e00780070099000801190000400be00e0
:107e200052e707000001be000800be00b0e60700f0
:107e30001e01780010099800210998001e007800a2
:107e4000500a9000e00a90001e0078003001900077
:107e5000c00190000400be0044e707001e01780046
:107e600030099800410998001e007800302a9000df
:107e7000c02a90001e00780010099000a009900010
:107e80000400be009ae607000002be001e00780053
:107e900030099000c00990000400be0094e607007d
:107ea0001e01780050019800610198004f04be0047
:107eb0000080fa00000006001200fa00889fbe0051
:107ec00040079800520798006307980074079800cd
:107ed000050f98005e009000ee00900020079800cb
:107ee000310798007e0190008e099000028fbe003d
:107ef0004e009000e0009000500090001e01be0077
:107f00006fe707000000e00001003c0012003700ae
:107f10004e009000100c9000a00c90004e009000bd
:107f200050019000e00190001e00be006fe60700c7
:107f30000001be000800be006de607004e01900083
:107f400010099800210998004e0090001e01be0003
:107f500052009800630098004e009000e0009000ee
:107f6000500090002e019000be01900056e70700df
:107f70000000e00001003500140037004e009000c2
:107f8000100c9000a00c90004e009000500190004a
:107f9000e00190002e009000be00900053e6070024
:107fa0000001be000800be0051e607004e0190002f
:107fb00010099800210998004e0090002e019000b1
:107fc000be01900052009800630098004f04be006c
:107fd0000080fa00000006000a00fa00000f780096
:107fe0001207980023079800340798004507980067
:107ff0001e007800a0089000100890003e0190003c
:10800000ce0190002ee707000000e00001003c00d8
:10801000050037001e0078003e019000ce01900060
:1080200012089800230898001e007800a00890000d
:10803000100890001e019000ae01900022e707009a
:108040000000e00001003500050037001e00780048
:108050001e019000ae0190001208980023089800bd
:108060000080fa00000006000600fa00000f780009
:1080700012079800230798001e007800c0009000a7
:10808000300090001e019000ae0190000ce7070048
:108090000000e00001003c00060037001e007800f0
:1080a0001e019000ae01900032009800430098003d
:1080b000120037001e00780030029000c0029000cd
:1080c0001e009000ae0090000001be0003f0a20070
:1080d0000400be00fce607000000e00001003500df
:1080e000060037001e009000ae00900001f0a200d4
:1080f0001e01780030019800410198000080fa00cc
:10810000000006003600f800809fbe00829fbe007f
:10811000849fbe00869fbe003400f80000c0b300fc
:10812000a00188000200fa00d5c2bf0068406000cc
:108130000004e00012003200a0668000811e2a00c8
:1081400000004000610078000030a0003d0f0700f3
:10815000a06680000000e800a0668800a06680009d
:10816000811e2a0000004000610078000000e0004d
:1081700006003a000000eb00a0668800030037000c
:1081800010002000a07c8800caa2a80089fa07007d
:10819000407d80006f006000000f78001e007800b6
:1081a000e40f5000070032001e007800e80f500076
:1081b000060032001e007800e20f50000a00320074
:1081c00026003700e0fb070032003700407d8000ca
:1081d000010f200001006000f00f50002d00320060
:1081e000d9fb07002b003700607a8000717a80008d
:1081f000d2cc2c00c3f42300b1e607000000e0005d
:1082000001003c00040037006011b8006000b800b5
:108210000822070005003700a299290093e92300ee
:10822000a099290091e92300022207006011b800fb
:108230006000b8004022070020e62000d000900037
:10824000400090003013070001f0a200e2ce2000b1
:1082500030219800412198000e0037006011b800cd
:108260006000b800f32107006011b8006000b8009a
:108270003122070020e62000d0009000400090004e
:108280002113070001f0a200e2ce20003021980067
:10829000412198008760a9000080fa003400f900ad
:1082a0004f03be004f02be004f01be004f00be0094
:1082b0003600f900004006002000fa00881f780010
:1082c000a0ef2000100478006140b9005ce50700d1
:1082d000600f9800710f98000800e00007003d0053
:1082e00002002000037824006e089000fe08900031
:1082f0007fe50700600f9800710f9800a2702d00b5
:1083000033b223006e089000fe08900017e60700c5
:1083100042b6230073fa230074e5070080798800d1
:1083200091798800a0ef2000200490006140b900fe
:1083300043e50700400f9800510f98000800e00047
:1083400007003d0002002000037824004e08900042
:10835000de08900066e50700400f9800510f980076
:1083600022952400d3b123004e089000de0890002f
:10837000fee50700228e2500f3f923005be50700e8
:10838000a0798800b1798800a0ef20004004900017
:108390006140b9002ae50700200f9800310f9800ce
:1083a0000800e00007003d000200200003782400e0
:1083b0002e089000be0890004de50700200f9800a1
:1083c000310f9800324c2600a3aa23002e089000fb
:1083d000be089000e5e50700f2482e0023df2300e9
:1083e00042e50700c0798800d1798800a0ef20001d
:1083f000600490006140b90011e50700000f98008b
:10840000110f98000800e00007003d000200200066
:10841000037824000e0890009e08900034e50700c1
:10842000000f9800110f9800a2702d0033b22300a6
:108430000e0890009e089000cce5070082b720004f
:10844000c3fa230029e50700e0798800f179880064
:10845000a0ef2000100490006140b900f8e407008c
:1084600060079800710798000800e00007003d00d1
:1084700002002000037824006e009000fe009000af
:108480001be507006007980071079800324c260032
:10849000a3b223006e009000fe009000b3e5070039
:1084a000721b2d0003fb230010e50700007a8800f3
:1084b000117a8800a0ef2000300490006140b900dc
:1084c000dfe4070040079800510798000800e0002b
:1084d00007003d0002002000037824004e009000b9
:1084e000de00900002e50700400798005107980061
:1084f000a2702d0033b223004e009000de009000e9
:108500009ae5070092e4220073fa2300f7e40700db
:10851000207a8800317a8800a0ef20005004900073
:108520006140b900c6e407002007980031079800b1
:108530000800e00007003d0002002000037824004e
:108540002e009000be009000e9e40700200798008c
:1085500031079800324c2600a3aa23002e00900079
:10856000be00900081e50700a24e200043e32300f7
:10857000dee40700407a8800517a8800a0ef2000ee
:10858000700490006140b900ade40700008fbe00a8
:108590000800e00005003d000200200003782400f0
:1085a0001e00be00d2e40700008fbe00324c260041
:1085b000a3b223001e00be006ce50700a29b2400ae
:1085c000c3fa2300c9e40700607a8800717a880042
:1085d00080798000917980000200200003f8230058
:1085e000b7e507000000e00001003c00050037008f
:1085f0000000200001f8230080798800917988002c
:108600000c00370080798000917980000200200002
:1086100003f82b00ace507000000e0000100350086
:10862000040037000000200001f82b00807988004a
:1086300091798800a0798000b17980000200200043
:1086400003f823009ee507000000e00001003c0065
:10865000050037000000200001f82300a079880001
:10866000b17988000c003700a0798000b1798000d2
:108670000200200003f82b0093e507000000e00053
:1086800001003500040037000000200001f82b0035
:10869000a0798800b1798800c0798000d179800004
:1086a0000200200003f8230085e507000000e00039
:1086b00001003c00050037000000200001f8230005
:1086c000c0798800d17988000a003700c07980001d
:1086d000d17980006011b8007be507000000e00060
:1086e00001003500030037006000b800c079880041
:1086f000d1798800e0798000f179800002002000c3
:1087000003f823006ee507000000e00001003c00d4
:10871000050037000000200001f82300e079880000
:10872000f17988000c003700e0798000f179800051
:108730000200200003f82b0063e507000000e000c2
:1087400001003500040037000000200001f82b0074
:10875000e0798800f1798800007a8000117a800041
:108760000200200003f8230055e507000000e000a8
:1087700001003c00050037000000200001f8230044
:10878000007a8800117a88000c003700007a800097
:10879000117a80000200200003f82b004ae5070050
:1087a0000000e00001003500040037000000200058
:1087b00001f82b00007a8800117a8800207a800066
:1087c000317a80000200200003f823003ce5070016
:1087d0000000e00001003c00050037000000200020
:1087e00001f82300207a8800317a88000c003700d5
:1087f000207a8000317a80000200200003f82b00ec
:1088000031e507000000e0000100350004003700fa
:108810000000200001f82b00207a8800317a8800bf
:10882000407a8000517a80000200200003f8230083
:1088300023e507000000e00001003c0005003700d0
:108840000000200001f82300407a8800517a880057
:108850000a003700407a8000517a80006011b80029
:1088600019e507000000e0000100350003003700b3
:108870006000b800407a8800517a8800607a8000f1
:10888000717a80000200200003f823000ce5070045
:108890000000e00001003c0005003700000020005f
:1088a00001f82300607a8800717a88000c00370094
:1088b000607a8000717a80000200200003f82b00ab
:1088c00001e507000000e00001003500040037006a
:1088d0000000200001f82b00607a8800717a88007f
:1088e0004f0478000080fa00000006008400fa00bf
:1088f0000040eb0010479800d702a80000c42900f0
:108900000100200017240700d702a90000c4290095
:10891000010020001324070010c8b300204798006e
:1089200000c1b300104798009e4090002e40900078
:10893000d820070020c8b300204798000040eb0073
:10894000104798009e4090002e409000d1200700d4
:1089500030c8b30020479800f0c2b3001047980019
:108960009e4090002e409000ca20070060c8b300cf
:1089700020479800a0c4b300104798009e40900084
:108980002e409000c320070070c8b3002047980015
:108990000040eb00104798009e4090002e40900051
:1089a000bc200700b0c8b300204798000040eb008f
:1089b000104798009e4090002e409000b520070080
:1089c000c0c8b3002047980040c0b30010479800cb
:1089d0009e4090002e409000ae200700d0c8b3000b
:1089e0002047980010c4b300104798009e409000a4
:1089f0002e409000a7200700e0c8b3002047980051
:108a00000040eb00104798009e4090002e409000e0
:108a1000a020070000c9b30020479800e0ceb300b3
:108a2000104798009e4090002e409000992007002b
:108a3000b0c9b3002047980050c5b3001047980054
:108a40009e4090002e40900092200700c0c9b300c5
:108a50002047980050c0b300104798009e409000f7
:108a60002e4090008b200700d0c9b300204798000b
:108a700080c1b300104798009e4090002e409000a7
:108a80008420070020cbb30020479800c0c3b30068
:108a9000104798009e4090002e4090007d200700d7
:108aa00050cbb3002047980040c1b3001047980056
:108ab0009e4090002e40900076200700e0c9b30051
:108ac0002047980000c9b300104798009e409000ce
:108ad0002e4090006f200700f0c9b3002047980097
:108ae0000040eb00104798009e4090002e40900000
:108af00068200700f0c8b30020479800c0c2b30048
:108b0000104798009e4090002e4090006120070082
:108b100080cab3002047980020c0b30010479800d7
:108b20009e4090002e4090005a20070070cab3006b
:108b30002047980020c0b300104798009e40900046
:108b40002e4090005320070020cab3002047980011
:108b50008f87e80090c4b300e0ff9f0017ccb300fc
:108b6000f6cdb30025c6b30094c4b30003ccb30064
:108b700012cbb300f1cdb3002e409000552007007a
:108b80008f87e900f0c8b30020479800c0c0b30049
:108b9000104798009e4090002e4090003d20070016
:108ba00010c4b3002047980000c1b300004f780004
:108bb000e30047001e4178002e4090008820070007
:108bc000d0c5b3002047980030c0b300004f7800f4
:108bd000e30047001e4178002e40900080200700ef
:108be00060c6b3002047980030c0b300004f780043
:108bf000e30047001e4178002e40900078200700d7
:108c000020c7b3002047980010c0b300004f780081
:108c1000e30047001e4178002e40900070200700be
:108c200050c7b3002047980010c0b300004f780031
:108c3000e30047001e4178002e40900068200700a6
:108c40000000eb00b08188000000eb00c0818800cc
:108c50000080fa00000006006800fa000040eb0007
:108c600030479800f0c4b300004f78000040eb009c
:108c7000104798000040eb00204798000040eb00b0
:108c800050479800a1c0b30060c8b300012007009e
:108c90005b0037000040eb00104798000040eb00fd
:108ca0004047980053003700ce40900000c8b30002
:108cb000f81f070001c2b30090cab300f51f0700f8
:108cc000c1c2b300f0c8b300f21f0700e6004700be
:108cd00012c0b30090c0b300412007006e41900065
:108ce000e800470010c2b3003d200700c1c0b30038
:108cf000f0c8b300e71f07008040eb0090cab30044
:108d0000e41f0700e700470012c0b30070c0b300c3
:108d10003320070001c4b300d0c8b300dd1f070033
:108d200001c8b30050c8b300da1f07007106200065
:108d30008e80400012c0b30070c0b300282007002e
:108d40000b003700710620008e80400012c0b30077
:108d500070c0b3002220070000fa200001002000ac
:108d6000002307003e4090000040e8003047980094
:108d70007ee090000080fb004600de000000a200c4
:108d8000610060000004a2000004e00004003a005a
:108d9000be40900060c9b30080cf5000e9ff3600ac
:108da000e500470012c0b30030c1b3000c2007003b
:108db0000040eb00304798004e4090008080fb0060
:108dc0005e419000780047000100400002487800b2
:108dd0005e4090000004e00003003d001e40900053
:108de0000040e800104798004e4090000040e80026
:108df000404798004e4090009e4f5000aaff390017
:108e00001e409000e24f5000a2ff3600a1c4b30004
:108e100060c8b3009f1f070078004700104078002b
:108e2000704798000040eb0040479800140037005e
:108e30004e4090008080fb00780047000100400019
:108e4000904078007e40900080cf500009003900ab
:108e50004e4090008080fb007800470001004000f9
:108e60001040780070479800c0f22000ce4090007b
:108e7000014878004e4090000040e80040479800cc
:108e80004e4090009e4f5000e9ff3900c0f2200094
:108e9000104078008080fb0078004700810040008f
:108ea0000040eb00804878007800470010407800d0
:108eb000704798000040eb004047980014003700ce
:108ec0004e4090008080fb00780047000100400089
:108ed000904078007e40900080cf5000090039001b
:108ee0004e4090008080fb00780047000100400069
:108ef0001040780070479800c0f22000ce409000eb
:108f0000114098004e4090000040e8004047980013
:108f10004e4090009e4f5000e9ff3900c0f2200003
:108f2000104090008080fb007800470081004000e6
:108f30000040eb008048780078004700104078003f
:108f4000704798000040eb0040479800140037003d
:108f50004e4090008080fb007800470001004000f8
:108f6000904078007e40900080cf5000090039008a
:108f70004e4090008080fb007800470001004000d8
:108f80001040780070479800c0f22000ce4090005a
:108f9000214098004e4090000040e8004047980073
:108fa0004e4090009e4f5000e9ff3900c0f2200073
:108fb00090407800c0f220001040900080cf500018
:108fc0000a003600c0f22000104078007047980078
:108fd000c0f2200090409000c0f2200001487800cc
:108fe000fe409000c0f2200011409800c0f2200026
:108ff00090409000c0f220002040900080cf5000b0
:109000000a003600c0f2200010409000704798001f
:10901000c0f22000a0409000c0f220001140980053
:10902000fe409000c0f2200021409800c0f22000d5
:1090300090407800c0f220001040900080cf500097
:109040000a003600c0f220001040780070479800f7
:10905000c0f2200090409000c0f22000014878004b
:10906000fe409000c0f2200011409800c0f22000a5
:109070009040780000c8b300061f070001c2b3008b
:1090800090cab300031f0700c1c2b300f0c8b30009
:10909000001f0700e600470012c0b30090c0b300f5
:1090a0004f1f07006e419000e800470010c2b30058
:1090b0004b1f0700c1c0b300f0c8b300f51e070086
:1090c0008040eb0090cab300f21e0700e7004700a3
:1090d00012c0b30070c0b300411f070001c4b30049
:1090e000d0c8b300eb1e070001c8b30050c8b300de
:1090f000e81e07000080fa00000006000800fa00e1
:10910000a0ee2000404090000080fb001007980077
:109110001e009000000f7800a0ee200010407800a4
:109120000080fb0020079800a0ee20001040900077
:109130000080fb00300798009e009000000c20008b
:10914000008060004200dd0010079800000320004e
:109150001e0060004400dd00000f78009e009000bb
:109160002e00900080804000a0ef200001087800d1
:109170003e0090009e004000a0ef200011009800eb
:10918000a0ee2000404090000080fb0010079800f7
:109190009e009000010f7800a0ee2000204090007b
:1091a0000080fb0020079800a0ee200030409000d7
:1091b0000080fb00300798001e0090006c006000eb
:1091c0004600dd00100798009e0078006380600074
:1091d0004800dd00000f78009e0090002e009000f7
:1091e00080804000a0ef2000210098003e00900009
:1091f0009e004000a0ef200031009800a0ee20006b
:10920000104890000080fb00100798001e0090009e
:10921000000f7800a0ee2000504090000080fb007e
:1092200020079800a0ee2000604090000080fb0026
:10923000300798009e009000000c20000080600025
:109240004200dd0010079800000320001e006000af
:109250004400dd00000f78009e0090002e0090007a
:1092600080804000a0ef2000410098003e00900068
:109270009e004000a0ef200051009800a0ee2000ca
:10928000104890000080fb00100798009e0090009e
:10929000010f7800a0ee2000704090000080fb00dd
:1092a00020079800a0ee2000004890000080fb00fe
:1092b000300798001e0090006c0060004600dd0042
:1092c000100798009e007800638060004800dd0071
:1092d000000f78009e0090002e00900080804000db
:1092e000a0ef2000610098003e0090009e0040002a
:1092f000a0ef2000710098000080fa000000060036
:109300000800fa00881f78000040eb00004f78004a
:10931000440037001e80fb00300798001e80fb00d1
:10932000a1ef200000004000610478006140b90016
:1093300043e1070010079800210798000800e000ab
:1093400007003d0002002000037824001e0090006a
:10935000ae00900066e10700100798002107980012
:1093600002002000833424001e009000ae00900014
:109370005ee107000200200063412400b9e107001c
:109380000001be00a1f020003e0290004220dd005e
:10939000010040000288be001e80fb00a1f02000fa
:1093a0004200dd00008040001000be006011b800e7
:1093b00045e207000000e00001003500060037002c
:1093c0001e80fb00a1f020004200dd0001014000f2
:1093d0006000b8000089be001e80fb00a1f02000e4
:1093e0004200dd00008040001000be0002002000ae
:1093f00003f8230032e207000000e00001003c0017
:10940000070037001e80fb00a1f020004200dd00b5
:10941000010140000000200001f823000089be0087
:109420001e4fe80070c0b3009e4f1000b9ff360019
:109430004f0478000080fa00000006000000fa00e7
:10944000cf1e0700e41e0700d702a800e922a800eb
:109450000000eb005079880024fd0700fefd0700a6
:10946000d81e07000000eb000080fa000000060094
:109470003600f800809fbe00829fbe00849fbe0021
:10948000869fbe001200fa000040eb00004f7800fb
:109490000040eb00104798009460a9000040eb00ea
:1094a000104798000040eb00004f7800b08180002a
:1094b0000000e800b0818800c08180000000e80062
:1094c000c081880012c0b3008e00780070c0b30065
:1094d000431e07001e4078008080fb0050082000db
:1094e000008060000000e0001a00320001c2b300fa
:1094f00090cab300e71d0700c1c2b300f0c8b300b3
:10950000e41d07008e00e80012c0b30090c0b30055
:10951000331e07001e4190008e80e80010c2b30089
:109520002f1e0700c1c0b300f0c8b300d91d07004b
:109530008040eb0090cab300d61d070001c8b300fd
:1095400070c8b300d31d070021c8b30050c8b300d2
:10955000d01d07009e407800a0c3b30080cf50000c
:1095600022003a000000eb00b08188000000eb0010
:10957000c08188008e00e80012c0b30090c0b30024
:10958000171e07001e419000a1ee200010c2b3007c
:10959000131e0700a0ee2000404890000080fb0052
:1095a00063006000e30f50000d003a005079800026
:1095b0000000e8005079880050798000e30f5000e7
:1095c00002003a000000eb005079880050798000da
:1095d000c1f22000e140780000c8b300ad1d0700d3
:1095e00021c8b30050c8b300aa1d0700b181800094
:1095f000700c2000808f50001200360050798000df
:109600000000e90050798800507980000000e000f7
:1096100002003d0020002000507988005179800030
:10962000c0f22000e0c0780000c8b300991d070018
:1096300021c8b30050c8b300961d07000000eb001e
:10964000b0818800c1818000f07c2000808f5000b4
:1096500010003600d702a80000c429000100200035
:10966000c0200700d702a80000c429000100200084
:10967000bc2007000000eb00507988009bfc07002d
:1096800075fd07000000eb00b08188000000eb00d2
:10969000c081880099fe070007fb07008460a900cd
:1096a0009460a8000080fa004f03be004f02be0085
:1096b0004f01be004f00be003600f900004006001a
:1096c0000400fa00204798000040eb00004f7800ab
:1096d000ae40900000c1b300f11b0700004f7800be
:1096e0001e00fb000080fa00000006000400fa00e3
:1096f00020479800314798000040eb00004f780069
:109700003e419000ae40900000c1b3003c1c0700f9
:10971000004f78001e00fb000080fa0000000600e9
:109720000c00fa0010079800210798000000eb00d9
:10973000000f78002e0090000000e00003003a00c7
:10974000e0ff2f00500798001c0037001000200099
:10975000300798000a0037003e0090008000780033
:109760001e00900000804000104078000080fb0048
:109770001e0f40003e0090000000e80030079800f7
:10978000be0090002e009000808f5000f2ff390044
:10979000f00f20001e0f60001e00e00003003200ea
:1097a0000080eb0040079800020037000000eb004b
:1097b000400798004e009000500798005e0090000f
:1097c0000080fa00000006001800fa00200f980040
:1097d000e3004700a3c0b30042c7b30000c1b30019
:1097e000d31b0700204798002e4090000004e000a3
:1097f000040032002e4090000000fb00300f980063
:109800001d00370063004700a1002000c4ff0700cf
:10981000204798002e4090000004e0000400320031
:109820002e4090000000fb00300f9800120037001f
:109830000000eb00000f7800090037001e007800e0
:10984000800078002e089000008140009e00e80013
:109850006300470060c07800004978001e0fe800f0
:10986000700020009e0f1000f4ff34002e40900086
:109870000000fb00300f98003e0890000080fa00c6
:10988000000006000600fa00100798000040eb00f8
:10989000004f7800e3c0b300e2c0b3009e00900028
:1098a00000c1b300a21b0700004f78001e04e000b7
:1098b000030032001e00fb00200798000b00370059
:1098c0001e009000e100200095ff0700004f780087
:1098d0001e04e000030032001e00fb002007980079
:1098e000020037000000eb00200798002e009000d7
:1098f0000080fa00000006000600fa001007980039
:109900000040eb00004f7800e3c0b3000041eb00e3
:109910009e00900000c1b300851b0700004f780037
:109920001e04e000030032001e00fb002007980028
:109930000b0037001e009000e100200078ff0700b8
:10994000004f78001e04e000030032001e00fb0000
:1099500020079800020037000000eb002007980065
:109960002e0090000080fa00000006000600fa00b9
:10997000100798000040eb00004f7800e3c0b300f0
:10998000c2c1b3009e00900000c1b300681b070075
:10999000004f78001e04e000050032009e40780071
:1099a0006ac050000000fb00200798000d0037003f
:1099b0001e009000e100200059ff0700004f7800d2
:1099c0001e04e00005003200e0ccb3001e40400061
:1099d0000000fb0020079800020037000000eb00a9
:1099e000200798002e0090000080fa00000006007a
:1099f0000600fa00100798000040eb00004f7800c6
:109a0000e3c0b300a2c2b3009e00900000c1b30047
:109a1000471b0700004f78001e04e00003003200df
:109a20001e00fb00200798000b0037001e0090006e
:109a3000e10020003aff0700004f78001e04e0001c
:109a4000030032001e00fb002007980002003700d0
:109a50000000eb00200798002e0090000080fa0024
:109a6000000006000600fa00100798000040eb0016
:109a7000004f7800e3c0b30082c3b3009e009000a3
:109a800000c1b3002a1b0700004f78001e04e0004d
:109a9000030032001e00fb00200798000b00370077
:109aa0001e009000e10020001dff0700004f78001d
:109ab0001e04e000030032001e00fb002007980097
:109ac000020037000000eb00200798002e009000f5
:109ad0000080fa00000006000600fa001007980057
:109ae0000040eb00004f780063c0b30062c4b300d5
:109af0009e00900000c1b3000d1b0700004f7800ce
:109b00001e04e000030032001e00fb002007980046
:109b10000b0037001e0090006100200000ff0700ce
:109b2000004f78001e04e000030032001e00fb001e
:109b300020079800020037000000eb002007980083
:109b40002e0090000080fa00000006000600fa00d7
:109b5000100798000040eb00004f780063c0b3008e
:109b6000c2c4b3009e00900000c1b300f01a070009
:109b7000004f78001e04e000030032001e00fb00ce
:109b8000200798000b0037001e00900061002000a5
:109b9000e3fe0700004f78001e04e00003003200df
:109ba0001e00fb0020079800020037000000eb00b9
:109bb000200798002e0090000080fa0000000600a8
:109bc0000600fa00100798000040eb00004f7800f4
:109bd00043c1b30002c6b3009e00900000c1b300b1
:109be000d31a0700004f78001e04e0000500320081
:109bf0009e4078006ac050000000fb0020079800db
:109c00000d0037001e00900041012000c4fe070037
:109c1000004f78001e04e00005003200e0ccb300e5
:109c20001e4040000000fb002007980002003700a3
:109c30000000eb00200798002e0090000080fa0042
:109c4000000006000600fa00100798000040eb0034
:109c5000004f7800e3c0b30022c5b3009e0090001f
:109c600000c1b300b21a0700004f78001e04e000e4
:109c7000030032001e00fb00200798000b00370095
:109c80001e009000e1002000a5fe0700004f7800b4
:109c90001e04e000030032001e00fb0020079800b5
:109ca000020037000000eb00200798002e00900013
:109cb0000080fa00000006000600fa001007980075
:109cc0000040eb00004f780023c1b30062c6b30030
:109cd0009e00900000c1b300951a0700004f780065
:109ce0001e04e000030032001e00fb002007980065
:109cf0000b0037001e0090002101200088fe0700a5
:109d0000004f78001e04e000030032001e00fb003c
:109d100020079800020037000000eb0020079800a1
:109d20002e0090000080fa00000006000200fa00f9
:109d3000000f7800e0c0b30061fe070080407800ab
:109d40001e007800014878001e0fe800f0c0b30044
:109d50005bfe0700804078001e0078000148780014
:109d60001e0fe80000c1b30055fe070080407800d8
:109d70001e007800014878001e0fe80010c1b300f3
:109d80004ffe0700804078001e00780001487800f0
:109d90001e0fe80020c1b30049fe07008040780094
:109da0001e007800014878001e0fe80030c1b300a3
:109db00043fe0700804078001e00780001487800cc
:109dc0001e0fe80040c1b3003dfe07008040780050
:109dd0001e007800014878001e0fe80050c1b30053
:109de00037fe0700804078001e00780001487800a8
:109df0001e0fe80060c1b30031fe0700804078000c
:109e00001e007800014878001e0fe80070c1b30002
:109e10002bfe0700804078001e0078000148780083
:109e20001e0fe80080c1b30025fe070080407800c7
:109e30001e007800014878001e0fe80090c1b300b2
:109e40001ffe0700804078001e007800014878005f
:109e50001e0fe800a0c1b30019fe07008040780083
:109e60001e007800014878001e0fe800b0c1b30062
:109e700013fe0700804078001e007800014878003b
:109e80000080fa0000000600cc00fa0050a79800fd
:109e90000000eb00000f78005ea090006100600001
:109ea0000004e0002d0032000e80e80075fe07007f
:109eb0000000fb001e0f70000e80e80010419000b3
:109ec0000e80e800204290000e80e800b040900034
:109ed0000e80e80040409000824178000441780004
:109ee000e70b070022e620000089be000e80e80094
:109ef000504190000e80e800604290000e80e80023
:109f0000f04090000e80e800004890008241780008
:109f100004417800da0b070022e6200020019800b7
:109f2000310198000e80e800104990000e80e80092
:109f3000204a90000e80e800b04890000e80e800b3
:109f4000404890008241780004417800cc0b070023
:109f500022e6200040019800510198005ea0900088
:109f60004800de00610060000004e0002e003200c6
:109f70000e80e80060fe07000000fb001e0f70006e
:109f80000e80e800104190000e80e8002042900012
:109f90000e80e800b04090000e80e8004040900045
:109fa0008241780004417800b50b070022e62000ca
:109fb00060019800710198000e80e8005041900007
:109fc0000e80e800604290000e80e800f0409000b3
:109fd0000e80e8000048900082417800044178003b
:109fe000a70b070022e6200000099800110998003d
:109ff0000e80e800104990000e80e800204a900092
:10a000000e80e800b04890000e80e80040489000c4
:10a010008241780004417800990b070022e6200075
:10a0200020099800310998005ea090000000d1003e
:10a03000610060000004e0002e0032000e80e800a5
:10a040004afe07000000fb001e0f70000e80e800b3
:10a05000104190000e80e800204290000e80e80041
:10a06000b04090000e80e8004040900082417800af
:10a0700004417800820b070022e620004009980086
:10a08000510998000e80e800504190000e80e800d1
:10a09000604290000e80e800f04090000e80e800e2
:10a0a000004890008241780004417800740b07005a
:10a0b00022e6200060099800710998000e80e800ef
:10a0c000104990000e80e800204a90000e80e800c1
:10a0d000b04890000e80e80040489000824178002f
:10a0e00004417800660b070022e62000001198006a
:10a0f000111198005ea090004200de006100600037
:10a100000004e0002e0032000e80e80038fe070058
:10a110000000fb001e0f70000e80e8001041900050
:10a120000e80e800204290000e80e800b0409000d1
:10a130000e80e800404090008241780004417800a1
:10a140004f0b070022e620002019980031199800d3
:10a150000e80e800504190000e80e80060429000c0
:10a160000e80e800f04090000e80e800004890006b
:10a170008241780004417800410b070022e620006c
:10a1800040199800511998000e80e800104990007d
:10a190000e80e800204a90000e80e800b048900051
:10a1a0000e80e80040489000824178000441780029
:10a1b000330b070022e620006019980071199800ff
:10a1c0005ea090004300de00610060000004e0003b
:10a1d0002e0032000e80e8009afe07000000fb000f
:10a1e0001e0f70000e80e800104190000e80e80005
:10a1f000204290000e80e800b04090000e80e80001
:10a200004040900082417800044178001c0b070018
:10a2100022e6200040119800511198000e80e800bd
:10a22000504190000e80e800604290000e80e800ef
:10a23000f04090000e80e8000048900082417800d5
:10a24000044178000e0b070022e6200060199800f8
:10a25000711998000e80e800104990000e80e80007
:10a26000204a90000e80e800b04890000e80e80080
:10a27000404890008241780004417800000b0700bc
:10a2800022e6200020099800310998005ea0900085
:10a290004400de00610060000004e0002e00320097
:10a2a0000e80e800effd07000000fb001e0f7000ad
:10a2b0000e80e800104190000e80e80020429000df
:10a2c0000e80e800b04090000e80e8004040900012
:10a2d0008241780004417800e90a070022e6200064
:10a2e00060219800712198000e80e8005041900094
:10a2f0000e80e800604290000e80e800f040900080
:10a300000e80e80000489000824178000441780007
:10a31000db0a070022e62000002998001129980096
:10a320000e80e800104990000e80e800204a90005e
:10a330000e80e800b04890000e80e8004048900091
:10a340008241780004417800cd0a070022e620000f
:10a3500020299800312998005ea090004500de0079
:10a36000610060000004e000120032000e80e8008e
:10a37000f6fd07000000fb001e0f70000e80e800d5
:10a38000104190000e80e800204290000e80e8000e
:10a39000b04090000e80e80040409000824178007c
:10a3a00004417800b60a070022e620004011980018
:10a3b000511198005ea090004600de006100600030
:10a3c0000004e000120032000e80e800c2fd070029
:10a3d0000000fb001e0f70000e80e800104190008e
:10a3e0000e80e800204290000e80e800b04090000f
:10a3f0000e80e800404090008241780004417800df
:10a400009f0a070022e62000402998005129980061
:10a410005ea090004700de00610060000004e000e4
:10a420003c0032000e80e80023fe07000000fb0025
:10a430001e0f70000e80e800104190000e80e800b2
:10a44000204290000e80e800b04090000e80e800ae
:10a45000404090008241780004417800880a07005b
:10a4600022e6200060299800712998000e80e800fb
:10a47000504190000e80e800604290000e80e8009d
:10a48000f04090000e80e800004890008241780083
:10a49000044178007a0a070022e620000031980083
:10a4a000113198000e80e800104990000e80e800fd
:10a4b000204a90000e80e800b04890000e80e8002e
:10a4c0004048900082417800044178006c0a0700ff
:10a4d00022e6200020319800313198000e80e800fb
:10a4e000504990000e80e800604a90000e80e8001d
:10a4f000f04890000e80e800005090008241780003
:10a50000044178005e0a070022e6200040319800ee
:10a51000513198001e0078000080fa00000006000b
:10a520000e00fa0040079800510798004e00900076
:10a530000000e800300798000000eb0010079800ca
:10a540004e00900047fd07000000fb00000f780060
:10a550001e00e0000400320080f32f001e004000c7
:10a56000600798002d0037004e00900010407800e2
:10a57000e14f500003003e000000eb006007980030
:10a58000260037004e009000104078000080fb004d
:10a590000080e9000080d100100798000000eb0067
:10a5a00020079800170037003e0090001040780008
:10a5b0008081fb003e0090000000e800300798001a
:10a5c0003e009000104078000081fb003e009000ab
:10a5d0000000e800300798002e00900000004000c6
:10a5e000800078005e009000808040004810dd0010
:10a5f00003007000800878002e0090000000e80042
:10a6000020079800ae0090001e009000808f500040
:10a61000e5ff39001e009000600798006e00900072
:10a620000080fa0000000600a04090008180fb003e
:10a6300063834000e303400020c4b300c049e3004b
:10a64000180032000600e00003003a0006407800df
:10a650000080fb00000006000041eb000000eb0062
:10a6600080007800059c2000674078000140680069
:10a670000080fb0060c07a000080fb00c808dd009d
:10a68000810068000241e8000280fb00860f500054
:10a69000f5ff3900014078000080fb000000060053
:10a6a000edff37000001eb00059c200083cdb300d7
:10a6b0000410200002407800810020000004e00027
:10a6c0000a003500004040008100e900fbff3a002d
:10a6d00000f17a000201e800840f5100d9ff320036
:10a6e0000240780081002000f4ff37000040d000d5
:10a6f000034068008100e900f0ff3a00f4ff3700f2
:10a7000001487800124098008040eb0021409800fa
:10a7100000000500889fbe0080047800104078008b
:10a72000b044980019409000c0449800294090001f
:10a73000d04498000084fb006304440009007800c2
:10a74000b9ff0700b0dc980088804400b040980052
:10a750000000eb004f04be000000060060409000c7
:10a760008048780000000500630040003041900000
:10a77000824878004040900090409800000005001a
:10a7800063004000304190008248780040419000d2
:10a7900092409800d04190008381fb00604190007e
:10a7a0004811dd0082817100b30098007041900073
:10a7b0000281fb00a2009800004990000281fb008a
:10a7c000104890004800dd000001710092009800e0
:10a7d000000005006601400092417800efc861006a
:10a7e0001281fb004411de00924098006700400097
:10a7f000904178006fc16100a24098001080fb007a
:10a800004400de00b04098000000050063004000f6
:10a81000b04190008381fb00404190004811dd0071
:10a820008281710093009800504090000080fb00ee
:10a8300080087800000005006040900080487800a3
:10a840000000050063004000b04190008381fb00e0
:10a85000404190004811dd0082887100d041900095
:10a860008381fb00604190004811dd00828171000e
:10a8700093009800f04190008381fb000049900014
:10a880004811dd0082817100a3009800904990007a
:10a890008381fb00204990004811dd008281710016
:10a8a000b3009800604990000281fb000300200083
:10a8b000c2009800d3009800c819dd000280fd0096
:10a8c000824178000041eb00504a90000482fb0076
:10a8d000050020000401710085817100c20098000c
:10a8e000d3009800c819dd000280fd008241780085
:10a8f0000041eb00404a90000482fb00050020006c
:10a900000401710085817100c2009800d300980095
:10a91000c819dd000280fd00824178000041eb0093
:10a92000304a90000482fb00050020000401710001
:10a9300085817100c2009800d300980000000500d6
:10a9400063004000b04190008381fb0040419000d3
:10a950004811dd0082887100d04190008381fb00a6
:10a96000604190004811dd008281710093009800e1
:10a97000f04190008381fb00004990004811dd0008
:10a9800082817100a3009800104990000281fb00b1
:10a99000204890004800dd0000017100b2009800de
:10a9a0000000050063004000b04190008381fb007f
:10a9b000404190004811dd0082887100d041900034
:10a9c0008381fb00604190004811dd0082817100ad
:10a9d00093009800f04190008381fb0000499000b3
:10a9e0004811dd0082817100a30098001049900099
:10a9f0000281fb00204890004800dd00000171004a
:10aa0000b200980000000500630040003041900053
:10aa10008248780040409000904098000000050077
:10aa200063004000b04190008381fb0040419000f2
:10aa30004811dd0082887100504190000281fb00c6
:10aa4000604090004800dd00000171009200980015
:10aa500000000500889fbe008a9fbe0000057800a8
:10aa60000140780002047800e3044500e605450053
:10aa700011c5b3000300e00013003200004178006c
:10aa80000a0078001eff0700984d780028409000cb
:10aa9000c044980038409000d0449800484090004e
:10aaa000e044980058449000f844980050c0b30027
:10aab000204598000a00780016ff07004f05be00e9
:10aac0004f04be000000060011c9b3000041780029
:10aad0000a0078000aff0700984d7800284090008f
:10aae000c044980038409000d044980048409000fe
:10aaf000e044980058449000f844980050c0b300d7
:10ab0000204598000a00780002ff07004f05be00ac
:10ab10004f04be0000000600ebff3700630040005a
:10ab20003041900082487800c04190008381fb0052
:10ab3000504190004811dd0082817100930098001f
:10ab4000604190000281fb00704090004800dd00f1
:10ab500000017100a20098000000050011192a00f0
:10ab60000004e0000400320001182a00e14f500008
:10ab70000100320091182a00010078000000060050
:10ab8000889fbe008a9fbe000005780001407800c3
:10ab900002047800e3044500e605450021c5b30042
:10aba0000300e00029003200004178000a0078002c
:10abb000d3fe0700984d780018409000c0449800dc
:10abc00028409000d044980038409000e04498001d
:10abd00048409000f044980058409000804c980005
:10abe00068409000904c980078409000a04c9800ed
:10abf00008489000b04c980018489000c04c98004d
:10ac000028489000d04c980038489000e04c9800bc
:10ac100048489000f04c98005848900080549800a4
:10ac20006848900090549800784c9000a854980080
:10ac300000c1b300204598000a007800b5fe070067
:10ac40004f05be004f04be000000060021c9b3003e
:10ac5000004178000a007800a9fe0700984d7800ae
:10ac600018409000c044980028409000d0449800bc
:10ac700038409000e044980048409000f04498002c
:10ac800058409000804c980068409000904c98008c
:10ac900078409000a04c980008489000b04c980074
:10aca00018489000c04c980028489000d04c98005c
:10acb00038489000e04c980048489000f04c9800cc
:10acc000584890008054980068489000905498002c
:10acd000784c9000a854980000c1b300204598001b
:10ace0000a0078008bfe07004f05be004f04be002f
:10acf00000000600d5ff370063004000b04190001f
:10ad00008381fb00404190004811dd008288710082
:10ad1000d04190008381fb00604190004811dd002c
:10ad20008281710093009800f04190008381fb00c4
:10ad3000004990004811dd0082817100a300980055
:10ad4000904990008381fb00204990004811dd006c
:10ad500082817100b3009800b04990008381fb00ac
:10ad6000404990004811dd0082817100c3009800c5
:10ad7000d04990008381fb00604990004811dd00bc
:10ad800082817100d3009800f04990008381fb001c
:10ad9000005190004811dd0082817100e3009800ad
:10ada000105190000281fb00205090004800dd000f
:10adb00000017100f200980000000500889fbe00ad
:10adc0000004780002407800830478000074a0003a
:10add00001417800804078000800780048fe0700b4
:10ade000994478006944980010c0b300204498004a
:10adf0000800780047fe07004f04be000000060070
:10ae0000889fbe008a1f7800000578000204780041
:10ae1000e604450001417800e1c0b3000a00780073
:10ae200037fe0700080178000000eb000104200055
:10ae300032f07c000000e800810f5000fcff3a0077
:10ae400000042000204598000a00780031fe070029
:10ae50004f0578004f04be00000006006600400069
:10ae60000001eb0003042000e05879000201e80033
:10ae7000830f5100fcff3a0000000500889fbe00d0
:10ae80008a1f78000005780002047800e30445007a
:10ae90000141780041c9b3000a00780018fe07009c
:10aea00018407800b044980018409000c0449800c2
:10aeb00028409000d044980038409000e04498002a
:10aec0006a014500f40044000000eb003171780095
:10aed0000000e800f00f5000fcff3a0077814400ca
:10aee000e40044000000eb00317178000000e8004d
:10aef000f00f5000fcff3a007440400020459800dd
:10af00000a00780003fe07004f0578004f04be00da
:10af100000000600889fbe008a1f780000057800a8
:10af200082047800630445000141780031c8b30011
:10af30000a007800f2fd0700294090003044980094
:10af400039409000404498001940780050449800df
:10af5000994490006944980040c0b300204598008f
:10af60000a007800ebfd07004f0578004f04be0093
:10af700000000600881f780000047800aafd070082
:10af800080417800a8409000d2ff2f0040c5b30058
:10af900080cf500003003600020078004f04780094
:10afa000000006000180fb0064004000e2ff2f006b
:10afb00071052000810f5000f7ff3c0038d8900049
:10afc00000c069000080fb000001ea004f91de0034
:10afd000020078004f04780000000600f1ff3700ff
:10afe00010417800e54f5100120032000900360090
:10aff000e84f51001a0032000f003600e94f5100af
:10b0000019003200ea4f5100160032000080eb00b8
:10b0100000000600e24f51000c003200090036002b
:10b02000e34f510009003200e44f5100f7ff3a00ae
:10b03000cafd3700d2fd3700e64f5100f3ff3a005a
:10b04000e4fd3700e14f5100f0ff3a005b000900da
:10b05000b0587800c105b100c005b100000005007e
:10b06000eafd370036fe3700f3fd37008000fa00b6
:10b07000889fbe008a9fbe00800578000204780089
:10b0800042062000b9180700584090000080fb00dd
:10b09000801f7800284090000080fb00801f78000f
:10b0a000484090000080fb00801f7800184090000e
:10b0b0000080fb00801f7800384090000080fb007b
:10b0c000801f78001880fb00801f780090192a00ec
:10b0d000801f7800a0f62f000f00400050d5070019
:10b0e00042062000a1f62f008f8040000b00780060
:10b0f0009e180700ee875700284090000004e000eb
:10b1000012003a0038d890000080fb00801f7800c1
:10b11000e01c2a00801f780040f72f000f0040003d
:10b120003fd507004206200041f72f008f804000e6
:10b130000b0078008d180700e48757004f05be000c
:10b140004f04be000080fa000000060066054400bf
:10b150008004eb003a80fb00801f7800801c2a00ee
:10b16000801f780040f72f000f0040002cd507000b
:10b170004206200041f72f008f8040000b0078002e
:10b180007a1807008904e800284090000080fb003e
:10b19000e4875700808f5400daff31003a80fb00cb
:10b1a000801f7800801c2a00801f780040f72f0045
:10b1b0000f0040001ad507004206200041f72f007b
:10b1c0008f8040000b007800681807008904e800b1
:10b1d000284090000080fb00e4875700808f5400d7
:10b1e000dcff3900c7ff3700889fbe008a9fbe0082
:10b1f0008c1f780000057800010678008204780032
:10b200008305780063044100320020008800780044
:10b210004a1807008081eb000000e00005003200c2
:10b22000030078004f0678004f05be004f04be00b3
:10b2300000000600984c7800494090009044980027
:10b24000d9409000a14498000141e800b3ff2f00cd
:10b2500040c5b30080cf5000f1ff3e000281fb00eb
:10b26000e68044008b0178000a007800331807005c
:10b27000e3ff2f000000e000e9ff3a0029409000c2
:10b280000080fb000900400060409000b0dc9800a6
:10b290000900780037ff0700d3ff2f000000e0000f
:10b2a000dfff3a000c00e000040035001980fb00cd
:10b2b000c3ff2f00800f5600d9ff3a000000200086
:10b2c0004f0678004f05be004f04be000000060088
:10b2d000d8ff37005c00fa00881f7800020478006d
:10b2e0008180fb0022fa2f000f014100beff070002
:10b2f0008080eb000000e0000400320001007800d4
:10b300004f0478000080fa000000060088007800f2
:10b3100020fa2f000f00400031ff070000007800e6
:10b320004f0478000080fa0000000600f7ff3700a5
:10b3300082017800214190000281fb0064014100fc
:10b34000e3804000f91737000c00fa00100798005e
:10b35000210798000000eb00000f78002e009000fd
:10b360000000e00003003a00e0ff2f0050079800c3
:10b370001c00370010002000300798000a0037003a
:10b380003e009000800078001e0090000080400089
:10b39000104078000080fb001e0f40003e0090002f
:10b3a0000000e80030079800be0090002e009000da
:10b3b000808f5000f2ff3900f00f20001e0f600058
:10b3c0001e00e000030032000080eb004007980000
:10b3d000020037000000eb00400798004e0090008c
:10b3e000500798005e0090000080fa000000060000
:10b3f0000a00fa0010079800210798003207980009
:10b400000040eb00004f78003e0090008041780043
:10b410002e0090008040780000c8b30000c04000bb
:10b42000004178009e00900000c1b300c0140700e6
:10b43000004f78001e04e0000500320000c8b30091
:10b440001e4070000000fb00400798000d00370010
:10b45000be0090001e009000bbff0700004f780068
:10b460001e04e0000500320000c4b3001e4070005e
:10b470000000fb0040079800020037000000eb00ce
:10b48000400798004e0090000080fa00000006007f
:10b490000600fa00200798002e009000630040008c
:10b4a000104078000080fb0001002000008fbe00eb
:10b4b0001e00be004809dd00c801de0083017100e6
:10b4c0004801dd002e0090000080e8001040780068
:10b4d0000080fb0001002000001f4100019749008f
:10b4e0001e00be004809dd00c801de0083017100b6
:10b4f0004801dd002e0090000000e80010407800b8
:10b500000080fb0001002000001f4100019749005e
:10b510001e00be004809dd00c801de008301710085
:10b520004801dd002e009000104078000080fb00f4
:10b5300001002000001f4100019749001e00be00cd
:10b540000080fa00000006001000fa00881f780052
:10b5500050079800610798000040eb00004f78000a
:10b560006e0090000000e000060032000e00e800cf
:10b57000820020008000eb009dff0700004f780054
:10b58000050037000e00e800820020008100200046
:10b5900097ff0700004f78001e04e0000300320010
:10b5a0001e00fb0070079800310037000e00e80015
:10b5b000204090000080fb00c800dd000e00e80085
:10b5c000104090000080fb0000807000cf80de0003
:10b5d0009bd807000200200043bb230063d907006b
:10b5e0005e0190000089be005e009000640440008f
:10b5f0000e00e800404090000080fb00c800dd0025
:10b600000e00e800304090000080fb0000807000d9
:10b61000cf80de008ad807000200200043bb230051
:10b6200052d90700008cbe005e0090006804400004
:10b630000e00e800604090000080fb00c800dd00c4
:10b640000e00e800504090000080fb000080700079
:10b65000cf80de007ad807000200200043bb230021
:10b6600042d90700008cbe000000eb007007980074
:10b670007e0090004f0478000080fa000000060071
:10b680000e00fa00881f7800500798000040eb0079
:10b69000004f78000e00e800820020000101200029
:10b6a00053ff0700004f78001e04e0000300320043
:10b6b0001e00fb0060079800310037000e00e80014
:10b6c000204090000080fb00c800dd000e00e80074
:10b6d000104090000080fb0000807000cf80de00f2
:10b6e00057d807000200200003202400ddd80700ff
:10b6f0005e0190000089be005e009000640440007e
:10b700000e00e800404090000080fb00c800dd0013
:10b710000e00e800304090000080fb0000807000c8
:10b72000cf80de0046d8070002002000032024005e
:10b73000ccd80700008cbe005e009000680440007a
:10b740000e00e800604090000080fb00c800dd00b3
:10b750000e00e800504090000080fb000080700068
:10b76000cf80de0036d8070002002000032024002e
:10b77000bcd80700008cbe000000eb0060079800fa
:10b780006e0090004f0478000080fa000000060070
:10b790000e00fa00881f7800500798000040eb0068
:10b7a000004f78000e00e800820020008101200098
:10b7b0000fff0700004f78001e04e0000300320076
:10b7c0001e00fb0060079800310037000e00e80003
:10b7d000204090000080fb00c800dd000e00e80063
:10b7e000104090000080fb0000807000cf80de00e1
:10b7f00013d807000200200043cb2300dbd807004a
:10b800005e0190000089be005e009000640440006c
:10b810000e00e800404090000080fb00c800dd0002
:10b820000e00e800304090000080fb0000807000b7
:10b83000cf80de0002d807000200200043cb2300a7
:10b84000cad80700008cbe005e009000680440006b
:10b850000e00e800604090000080fb00c800dd00a2
:10b860000e00e800504090000080fb000080700057
:10b87000cf80de00f2d707000200200043cb230078
:10b88000bad80700008cbe000000eb0060079800eb
:10b890006e0090004f0478000080fa00000006005f
:10b8a0000e00fa00881f7800500798000040eb0057
:10b8b000004f78000e00e800820020000102200006
:10b8c000cbfe0700004f78001e04e00003003200aa
:10b8d0001e00fb0060079800310037000e00e800f2
:10b8e000204090000080fb00c800dd000e00e80052
:10b8f000104090000080fb0000807000cf80de00d0
:10b90000cfd70700020020000370240055d807009d
:10b910005e0190000089be005e009000640440005b
:10b920000e00e800404090000080fb00c800dd00f1
:10b930000e00e800304090000080fb0000807000a6
:10b94000cf80de00bed70700020020000370240075
:10b9500044d80700008cbe005e00900068044000e0
:10b960000e00e800604090000080fb00c800dd0091
:10b970000e00e800504090000080fb000080700046
:10b98000cf80de00aed70700020020000370240045
:10b9900034d80700008cbe000000eb006007980060
:10b9a0006e0090004f0478000080fa00000006004e
:10b9b0001800fa00881f7800200f98000040eb0064
:10b9c000004f78000e00e80022012000c103200093
:10b9d00087fe0700004f78001e04e00003003200dd
:10b9e0001e00fb00300f9800290037000e00e80011
:10b9f0000000e800a6fe070091d707000200200023
:10ba00000370240017d807002e0990000089be009b
:10ba10002e089000640440000e00e800650040001d
:10ba20009bfe070086d70700020020000370240059
:10ba30000cd80700008cbe002e089000680440005f
:10ba40000e00e8006900400091fe07007cd7070067
:10ba5000020020000370240002d80700008cbe0002
:10ba60002e0890006c0440000e00e8006d004000bd
:10ba700087fe070072d70700020020000370240031
:10ba8000f8d70700008cbe000000eb00300f9800d4
:10ba90003e0890004f0478000080fa000000060085
:10baa0001400fa00881f7800000f98000040eb0097
:10bab000004f78000e00e800e2002000e1042000c2
:10bac0004bfe0700004f78001e04e0000300320028
:10bad0001e00fb00100f9800310037000e00e80038
:10bae0000000e8006afe070055d7070002002000aa
:10baf000433324001dd807000200200003702400f7
:10bb0000d8d707000200200003682400d5d707001b
:10bb10000e0990000089be000e08900064044000e9
:10bb20000e00e8006500400059fe070044d70700fa
:10bb300002002000433324000cd80700020020003c
:10bb400003702400c7d70700020020000368240008
:10bb5000c4d70700008cbe000e08900068044000a7
:10bb60000e00e8006900400049fe070034d70700d6
:10bb70000200200043332400fcd70700020020000d
:10bb800003702400b7d707000200200003682400d8
:10bb9000b4d70700008cbe000000eb00100f980027
:10bba0001e0890004f0478000080fa000000060094
:10bbb0000a00fa00300798000040eb00004f7800c0
:10bbc0000e00e800420020008102200008fe07006d
:10bbd000004f78001e04e000030032001e00fb004e
:10bbe000400798000e0037000e00e800204090004b
:10bbf0000080fb00c800dd000e00e800104090004f
:10bc00000080fb0000807000cf80de000cd70700b2
:10bc10003e0190000089be000000eb004007980044
:10bc20004e0090000080fa00000006000e00fa00ae
:10bc3000881f7800500798000040eb00004f780004
:10bc40000e00e80082002000c1022000e8fd07008d
:10bc5000004f78001e04e000030032001e00fb00cd
:10bc600060079800310037000e00e8002040900087
:10bc70000080fb00c800dd000e00e80010409000ce
:10bc80000080fb0000807000cf80de00ecd6070053
:10bc9000020020000348240072d707005e019000d4
:10bca0000089be005e009000640440000e00e800c1
:10bcb000404090000080fb00c800dd000e00e8005e
:10bcc000304090000080fb0000807000cf80de00dc
:10bcd000dbd60700020020000348240061d70700dc
:10bce000008cbe005e009000680440000e00e8007a
:10bcf000604090000080fb00c800dd000e00e800fe
:10bd0000504090000080fb0000807000cf80de007b
:10bd1000cbd60700020020000348240051d70700bb
:10bd2000008cbe000000eb00600798006e009000e1
:10bd30004f0478000080fa00000006001200fa00ac
:10bd40005007980061079800720798000040eb00c8
:10bd5000004f78000e00e800820020004103200020
:10bd6000a3fd0700004f78001e04e000030032002e
:10bd70001e00fb00000f98002f0037000e00e800a7
:10bd8000204090000080fb00c800dd000e00e800ad
:10bd9000104090000080fb0000807000cf80de002b
:10bda000a7d6070002002000034824002dd7070073
:10bdb0005e0190000089be000e00e8004040900047
:10bdc0000080fb00c800dd000e00e800304090005d
:10bdd0000080fb0000807000cf80de0098d6070056
:10bde0000200200043cb230060d707006e019000c3
:10bdf0000089be000e00e800604090000080fb005b
:10be0000c800dd000e00e800504090000080fb00fc
:10be100000807000cf80de0089d60700020020007d
:10be2000034824000fd707007e0190000089be0060
:10be30000000eb00000f98000e0890000080fa0050
:10be4000000006001000fa00700798000000eb00e8
:10be5000000f78007e009000610060000004e000a8
:10be6000050032008000eb0020e62000b6fd070050
:10be70000000fb001e0f70007e0090004800de00f6
:10be8000610060000004e0000500320011002000a5
:10be9000e0e62000acfd07000000fb001e0f700074
:10bea0007e0090000000d100610060000004e0000e
:10beb00004003200a0e72000f1fd07000000fb00b5
:10bec0001e0f70007e0090004200de0061006000e6
:10bed0000004e0000400320060e920002cfe0700ae
:10bee0000000fb001e0f70007e0090004300de008b
:10bef000610060000004e00006003200e1e920007b
:10bf0000e2e82000a0e820008cff07000000fb0012
:10bf10001e0f70007e0090004400de006100600093
:10bf20000004e00004003200e0ea20005cfe0700ac
:10bf30000000fb001e0f70007e0090004500de0038
:10bf4000610060000004e000150032000e80e8008f
:10bf500036ff07000000fb001e0f70000e80e80097
:10bf60001000be0022e620004011980051119800f8
:10bf70000e80e800b00090002000900022e6200033
:10bf800060119800711198000e80e800d0009000b8
:10bf90004000900022e62000001998001119980036
:10bfa0007e0090004600de00610060000004e000ba
:10bfb00004003200a0eb2000fdfe07000000fb00a3
:10bfc0001e0f70007e0090004900de0061006000de
:10bfd0000004e00004003200e0ec200074fe0700e2
:10bfe0000000fb001e0f70007e0090004a00de0083
:10bff000610060000004e00004003200e0ed200079
:10c00000a7fe07000000fb001e0f70001e00780056
:10c010000080fa00000006001000fa00881f780077
:10c020000001780001047800f00f50005100320048
:10c0300005003e00e10f50006d003200e20f50009d
:10c04000ad003a008b00370000082000800f51003f
:10c0500025003200f00f2000800f5100a6003a00aa
:10c060006166800061409000e14f40001a0032009c
:10c0700061099000f1099000829fbe0083022a00ae
:10c08000831f78007880570065d1070061668000c3
:10c09000e88140006140900062c0b3000440bc00f1
:10c0a0000280410042062000f8805700af140700cc
:10c0b00061668000e88140006140900062c0b3008a
:10c0c0000440bc0002804100420620008800780045
:10c0d000a6140700e6875700caa2a80010c0b30044
:10c0e000c70207008400370061668000614090004d
:10c0f000e14f40001a00320061099000f109900000
:10c10000829fbe0083022a00831f78007880570038
:10c1100043d1070061668000e881400061409000e3
:10c1200062c0b3000440bc0002804100420620000f
:10c13000f88057008d14070061668000e881400098
:10c140006140900062c0b3000440bc000280410026
:10c15000420620008800780084140700e687570014
:10c16000caa2a80010c0b300a5020700caa2a90075
:10c17000610037006166800061409000e14f40003f
:10c180005d00320061099000f1099000829fbe00bd
:10c1900083022a00831f78007880570020d107008f
:10c1a00061668000e88140006140900062c0b30099
:10c1b0000440bc000280410042062000f880570085
:10c1c0006a14070061668000e881400061409000c9
:10c1d00062c0b3000440bc0002804100420620005f
:10c1e0008800780061140700e68757004200370096
:10c1f000616680001100e0003f0032006140900065
:10c20000e14f40003c00320061099000f1099000cc
:10c21000829fbe0083022a00831f78007880570027
:10c22000ffd0070061668000e88140006140900017
:10c2300062c0b3000440bc000280410042062000fe
:10c24000f88057004914070061668000e8814000cb
:10c250006140900062c0b3000440bc000280410015
:10c26000420620008800780040140700e687570047
:10c27000210037006166800012002000910f11003c
:10c280001d00360061409000e14f40001a0032006e
:10c2900061099000f1099000829fbe0083022a008c
:10c2a000831f780078805700ddd00700616680002a
:10c2b000e88140006140900062c0b3000440bc00cf
:10c2c0000280410042062000f88057002714070032
:10c2d00061668000e88140006140900062c0b30068
:10c2e0000440bc0002804100420620008800780023
:10c2f0001e140700e68757004f0478000080fa00fc
:10c30000000006000000fe0000000600889fbe003e
:10c31000810478000000e0004b003200110490001e
:10c320006140b90046d507000800e00003003d0069
:10c3300002002000037824006dd5070002002000d1
:10c34000a3472400c7d507004069880051698800c9
:10c3500059009000cf80de0039d507000200200090
:10c36000a3472400bfd507004068880051688800b3
:10c3700069009000cf80de0031d507000200200068
:10c38000a3472400b7d5070060688800716888005b
:10c3900079009000cf80de0029d507000200200040
:10c3a000a3472400afd50700806888009168880003
:10c3b000190490006140b90021d507000800e00091
:10c3c00003003d00020020000378240048d5070048
:10c3d00002002000a3472400a2d50700106c8800ab
:10c3e000216c880029009000cf80de0014d5070062
:10c3f00002002000a34724009ad50700106b880094
:10c40000216b880039009000cf80de000cd507003a
:10c4100002002000a347240092d50700306b88005b
:10c42000416b880049009000cf80de0004d50700f2
:10c4300002002000a34724008ad50700506b880023
:10c44000616b88003800370002002000a3472400f9
:10c450004069800051698000c4d50700f7d5070006
:10c460009004980002002000a3472400706b800015
:10c47000816b8000bdd50700f0d50700800c7800e7
:10c4800002002000a3472400106b8000216b800075
:10c49000b6d50700e9d50700a004980002002000e7
:10c4a000a3472400306b8000416b8000afd50700ac
:10c4b000e2d50700b004980002002000a347240042
:10c4c000506b8000616b8000a8d50700dbd50700aa
:10c4d000c004980002002000a347240040688000a8
:10c4e00051688000a1d50700d4d50700d00498007a
:10c4f00002002000a347240060688000716880006b
:10c500009ad50700cdd50700e0049800020020006e
:10c51000a3472400806880009168800093d50700bd
:10c52000c6d50700f00498000000eb004f04be00e1
:10c5300000000600889fbe008a1f78000105780071
:10c540000000e0001200320021009000cf80de00e9
:10c55000bbd4070002002400c361240041d50700ba
:10c560000004be001a009000cf80de00b4d40700a3
:10c5700002002400c36124003ad507000001be0078
:10c580001a80fb000802be007b0a0700100037007b
:10c59000810a0700004d78000080fb00800a070038
:10c5a00002002400c361240070d50700a3d5070052
:10c5b000100598001a80fb00860a0700020024007c
:10c5c000c361240069d507009cd5070020059800a9
:10c5d0000000eb004f0578004f04be00000006008d
:10c5e0005a00fa00889fbe00d0022a000800090005
:10c5f000305f78009e00b1009000b1003712070054
:10c6000000482800e1012000d6140700c5140700e7
:10c61000e11007006011b8000200be00051107001c
:10c620006011b8000200be00431107005e1307004e
:10c630008a110700cc100700cf100700004828001f
:10c64000e1012000c71407000040eb00200a0700aa
:10c6500098e8070010c0b3006901070077f30700ee
:10c66000ca22a800caa2a90000202100a107200018
:10c67000bc140700d5c2bf000038a30004003a0074
:10c6800092140700d5c2bf000038a300fcff32009f
:10c690000e0078004cf407000040eb00004f9800bb
:10c6a0000e007800a213070030c0b3005401070049
:10c6b000ca22a900d00e8500e10e85006312070092
:10c6c000fd0d07000110200000ac20004cdf07002a
:10c6d000c0d62700a0568800e0f22700705a8800d4
:10c6e000c0002600805a880020182600905a880032
:10c6f00060182600a05a8800a0292600b05a880099
:10c700001000200000568800c6eab7000004eb00c5
:10c71000b8568800a9002000c9568800d056880065
:10c7200020ac2000c00c07008900780080cd2800d4
:10c73000f60d070088007800e0ec2700f30d0700f5
:10c7400088007800e0ef2700f00d0700411f20006f
:10c7500040802700ed0d070080ac2000be120700ce
:10c7600080ac2000e1120700421f200061032a0074
:10c7700080ac2000fd120700e0ac2000c1120700d1
:10c78000e0ac2000d9120700421f2000d1052a008a
:10c79000e0ac2000f5120700616680006140900067
:10c7a000e14f40001b00320069044700610990001e
:10c7b000f1099000829fbe0083022a00831f780047
:10c7c0000800780096cf070061668000e88140008d
:10c7d0006140900062c0b3000440bc000280410090
:10c7e0004206200088007800e012070061668000a1
:10c7f000e88140006140900062c0b3000440bc008a
:10c80000028041004206200031082a00d7120700aa
:10c81000e68757001e04e00004003a00010b2a00de
:10c82000f00f2000fcfd070026003700f904470048
:10c830008e1f7800410c2a00811f780009007800c3
:10c8400077cf070061668000e48757006140900061
:10c85000e14f40001b00320069044700610990006d
:10c86000f1099000829fbe0083022a00831f780096
:10c87000080078006acf070061668000e881400008
:10c880006140900062c0b3000440bc0002804100df
:10c890004206200088007800b4120700616680001c
:10c8a000e88140006140900062c0b3000440bc00d9
:10c8b000028041004206200089007800ab12070088
:10c8c000e687570081b5200000ac2000eede0700af
:10c8d00080ac200076120700e0ac20007412070044
:10c8e0000000eb004f04be000080fa0000000600cc
:10c8f0003600f800809fbe00829fbe00849fbe006d
:10c90000869fbe003400f80000c0b300a00188007c
:10c910001000fa008020a90061668000614090004c
:10c92000e14f40001a00320061099000f1099000c7
:10c93000829fbe0083022a00831f78007680570002
:10c9400037cf070061668000e881400061409000b9
:10c9500062c0b3000440bc000280410042062000d7
:10c96000f68057008112070061668000e881400070
:10c970006140900062c0b3000440bc0002804100ee
:10c9800042062000910d2a0078120700e687570022
:10c990000000fe000080fa003400f9004f03be00e2
:10c9a0004f02be004f01be004f00be003600f9002e
:10c9b000004006003600f800809fbe00829fbe0047
:10c9c000849fbe00869fbe003400f80000c0b30004
:10c9d000a00188001000fa008060a9006166800054
:10c9e00061409000e14f40001a0032006109900060
:10c9f000f1099000829fbe0083022a00831f780005
:10ca00007680570006cf070061668000e88140000d
:10ca10006140900062c0b3000440bc00028041004d
:10ca200042062000f6805700501207006166800021
:10ca3000e88140006140900062c0b3000440bc0047
:10ca40000280410042062000d10e2a004712070052
:10ca5000e68757000000fe000080fa003400f9006d
:10ca60004f03be004f02be004f01be004f00be008c
:10ca70003600f900004006003600f800809fbe0036
:10ca8000829fbe00849fbe00869fbe003400f800d7
:10ca900000c0b300a00188001000fa008040a90087
:10caa0006166800061409000e14f40001a00320052
:10cab00061099000f1099000829fbe0083022a0064
:10cac000831f780076805700d5ce0700616680000e
:10cad000e88140006140900062c0b3000440bc00a7
:10cae0000280410042062000f68057001f12070016
:10caf00061668000e88140006140900062c0b30040
:10cb00000440bc000280410042062000e10f2a00e0
:10cb100016120700e68757000000fe000080fa00aa
:10cb20003400f9004f03be004f02be004f01be00ab
:10cb30004f00be003600f900004006003600f80045
:10cb4000809fbe00829fbe00849fbe00869fbe0065
:10cb50003400f80000c0b300a00188001000fa0003
:10cb60008080a9006166800061409000e14f400034
:10cb70001a00320061099000f1099000829fbe0006
:10cb800083022a00831f780076805700a4ce070016
:10cb900061668000e88140006140900062c0b3009f
:10cba0000440bc000280410042062000f68057008d
:10cbb000ee11070061668000e8814000614090004e
:10cbc00062c0b3000440bc00028041004206200065
:10cbd000d1102a00e5110700e68757000000fe008b
:10cbe0000080fa003400f9004f03be004f02be007f
:10cbf0004f01be004f00be003600f90000400600a5
:10cc00000600fa00404798004e409000004f780020
:10cc10001a003700803e20001007980010003700ef
:10cc2000cbc2bf00624060000004e00005003a0093
:10cc3000cb22a80000f421000100200049130700c6
:10cc400004003700cb22a90000f4210001002000dd
:10cc5000441307001e0090000000e9001007980030
:10cc60001e0090000000e000edff3a000090200060
:10cc7000d10320003b1307001e4fe9001e04e00013
:10cc8000e4ff3a000080fa00000006000400fa0009
:10cc900000d4200031002000008fbe0011003700ba
:10cca000cbc2bf00624060000004e00005003a0013
:10ccb000cb22a80000f42100010020002913070066
:10ccc00004003700cb22a90000f42100010020005d
:10ccd000241307000080eb008080eb001e0f400053
:10cce0005e9748001e00be00e00f5000e08f580025
:10ccf000ebff3a000080fa00000006000000fa0096
:10cd0000cbc2bf000080fa00000006000200fa005b
:10cd1000000f78001e0078006101b80000c42900ef
:10cd20000012b8006010b90005037800000343004a
:10cd300000c429000098b90000034300860278006f
:10cd40000400be00071307000080fa000000060080
:10cd50000200fa00000f78001e0078006101b800a0
:10cd6000800220000012b8006010b90005037800ae
:10cd700000034300800220000098b9000003430034
:10cd8000860278000400be00f61207000080fa0058
:10cd9000000006000400fa00881f78000000eb0085
:10cda000a111070020818800288180006140b9001e
:10cdb000a3d20700008fbe000800e00005003d0080
:10cdc00002002000037824001e00be00c8d2070025
:10cdd000008fbe0092282d00e3b523001e00be0088
:10cde00062d3070082612200b3fc2300bfd2070098
:10cdf00030818800418188004f0478000080fa006b
:10ce0000000006000200fa003081800041818000ad
:10ce10000200200083122400a9d307000000e000d4
:10ce200001003c0004003700caa2a9000000eb008a
:10ce3000000f78000f0037003081800041818000b2
:10ce400032332300331224009fd307000000e00098
:10ce50000100350004003700caa2a800200020000d
:10ce6000000f780003003700caa2a80010002000bd
:10ce7000000f78001e0078000080fa000000060015
:10ce80000a00fa006047980071479800024f980026
:10ce9000134f98000e8fe8001e0078009e48900007
:10cea000014878001e00e8008e4890000148780094
:10ceb0001e80e800fe409000014878009e00780047
:10cec00063804000ee409000014878001e00900012
:10ced000ae0090000080fa00000006000400fa0096
:10cee000008fbe001e00be00b2fd2000930424008f
:10cef000dcd2070002002000433324001bd30700cc
:10cf00000080fa00000006000400fa00008fbe0056
:10cf10001e00be00b2fd20009304240013d30700be
:10cf20000200200043332400ced207000080fa0024
:10cf3000000006001000fa00200798003107980052
:10cf400042079800530798006407980075079800f7
:10cf50004e019000de0190002e009000be00900077
:10cf600057d307000000e00001003c001c00370020
:10cf70006e019000fe0190002e009000be00900017
:10cf800051d307000000e000010035000400370025
:10cf90002e009000be009000008fbe002b003700d6
:10cfa0004e019000de0190006e009000fe009000a7
:10cfb00043d307000000e00001003c0004003700fc
:10cfc0006e009000fe009000008fbe001f00370032
:10cfd0004e009000de009000008fbe001b00370066
:10cfe0006e019000fe0190002e009000be009000a7
:10cff00033d307000000e00001003c0004003700cc
:10d000002e009000be009000008fbe000f00370081
:10d010004e019000de0190006e009000fe00900036
:10d0200029d307000000e0000100350004003700ac
:10d030006e009000fe009000008fbe0003003700dd
:10d040004e009000de009000008fbe001e00be006b
:10d050000080fa00000006000800fa00100798009f
:10d0600021079800320798009e0090002e00900043
:10d07000808f5000110036009e0090003e0090000e
:10d08000808f5000030031001e009000000f7800d8
:10d090001a003700be0090002e009000808f5000d4
:10d0a000030036003e009000000f780013003700a8
:10d0b0002e009000000f7800100037009e009000b6
:10d0c0003e009000808f5000030036001e0090004c
:10d0d000000f780009003700be0090002e0090007d
:10d0e000808f5000030031003e009000000f780058
:10d0f000020037002e009000000f78001e0078001c
:10d100000080fa00000006000c00fa0010079800ea
:10d1100021079800320798004307980054079800a9
:10d120009e0090002e009000808f5000480031003b
:10d130009e0090003e009000808f5000440031001f
:10d140009e0090004e009000808f50004000310003
:10d150009e0090005e009000808f50003c003100e7
:10d16000de0090004e009000808f50000e003600d0
:10d17000de0090003e009000808f50000a003600d4
:10d18000de0090002e009000808f500006003600d8
:10d190004e019000be0090002e009000aeff0700f0
:10d1a000000f780049013700ce0090005e0090002b
:10d1b000808f50000e003600ce0090003e009000a0
:10d1c000808f50000a003600ce0090002e009000a4
:10d1d000808f5000060036005e019000be00900077
:10d1e0002e0090009cff0700000f780037013700e9
:10d1f000be0090005e009000808f50000e00360050
:10d20000be0090004e009000808f50000a00360053
:10d21000be0090002e009000808f50000600360067
:10d220005e019000ce0090002e0090008aff070063
:10d23000000f7800250137005e019000ce009000bd
:10d240003e00900084ff0700000f78001f013700a8
:10d25000ae0090001e009000808f5000480031000a
:10d26000ae0090003e009000808f500044003100de
:10d27000ae0090004e009000808f500040003100c2
:10d28000ae0090005e009000808f50003c003100a6
:10d29000de0090004e009000808f50000e0036009f
:10d2a000de0090003e009000808f50000a003600a3
:10d2b000de0090001e009000808f500006003600b7
:10d2c0004e019000be0090001e00900062ff07001b
:10d2d000000f7800fd003700ce0090005e00900047
:10d2e000808f50000e003600ce0090003e0090006f
:10d2f000808f50000a003600ce0090001e00900083
:10d30000808f5000060036005e019000be00900045
:10d310001e00900050ff0700000f7800eb00370060
:10d32000be0090005e009000808f50000e0036001e
:10d33000be0090004e009000808f50000a00360022
:10d34000be0090001e009000808f50000600360046
:10d350005e019000ce0090001e0090003eff07008e
:10d36000000f7800d90037005e019000ce009000d9
:10d370003e00900038ff0700000f7800d300370010
:10d38000be0090001e009000808f500048003100c9
:10d39000be0090002e009000808f500044003100ad
:10d3a000be0090004e009000808f50004000310081
:10d3b000be0090005e009000808f50003c00310065
:10d3c000de0090004e009000808f50000e0036006e
:10d3d000de0090002e009000808f50000a00360082
:10d3e000de0090001e009000808f50000600360086
:10d3f0004e019000ae0090001e00900016ff070046
:10d40000000f7800b1003700ce0090005e00900061
:10d41000808f50000e003600ce0090002e0090004d
:10d42000808f50000a003600ce0090001e00900051
:10d43000808f5000060036005e019000ae00900024
:10d440001e00900004ff0700000f78009f003700c7
:10d45000ae0090005e009000808f50000e003600fd
:10d46000ae0090004e009000808f50000a00360001
:10d47000ae0090001e009000808f50000600360025
:10d480005e019000ce0090001e009000f2fe0700aa
:10d49000000f78008d0037005e019000ce009000f4
:10d4a0002e009000ecfe0700000f78008700370088
:10d4b000ce0090001e009000808f50004800310088
:10d4c000ce0090002e009000808f5000440031006c
:10d4d000ce0090003e009000808f50004000310050
:10d4e000ce0090005e009000808f50003c00310024
:10d4f000de0090003e009000808f50000e0036004d
:10d50000de0090002e009000808f50000a00360050
:10d51000de0090001e009000808f50000600360054
:10d520003e019000ae0090001e009000cafe070071
:10d53000000f780065003700be0090005e0090008c
:10d54000808f50000e003600be0090002e0090002c
:10d55000808f50000a003600be0090001e00900030
:10d56000808f5000060036005e019000ae009000f3
:10d570001e009000b8fe0700000f7800530037002f
:10d58000ae0090005e009000808f50000e003600cc
:10d59000ae0090003e009000808f50000a003600e0
:10d5a000ae0090001e009000808f500006003600f4
:10d5b0005e019000be0090001e009000a6fe0700d5
:10d5c000000f7800410037005e019000be0090001f
:10d5d0002e009000a0fe0700000f78003b003700ef
:10d5e000ce0090003e009000808f50000e0036006c
:10d5f000ce0090002e009000808f50000a00360070
:10d60000ce0090001e009000808f50000600360073
:10d610003e019000ae0090001e0090008efe0700bc
:10d62000000f780029003700be0090004e009000e7
:10d63000808f50000e003600be0090002e0090003b
:10d64000808f50000a003600be0090001e0090003f
:10d65000808f5000060036004e019000ae00900012
:10d660001e0090007cfe0700000f780017003700b6
:10d67000ae0090004e009000808f50000e003600eb
:10d68000ae0090003e009000808f50000a003600ef
:10d69000ae0090001e009000808f50000600360003
:10d6a0004e019000be0090001e0090006afe070030
:10d6b000000f7800050037004e019000be0090007a
:10d6c0002e00900064fe0700000f78001e00780016
:10d6d0000080fa00000006000800fa002007980009
:10d6e000310798006011b8002e009000be00900035
:10d6f00075d107000000e00001003500050037008b
:10d700002e009000be00900001f0a200008fbe002d
:10d71000030037002e009000be009000008fbe0076
:10d720001e00be000080fa00000006000600fa009d
:10d73000200798002e009000100798000e8fe80038
:10d740001e007800104078000080fb000080fa0086
:10d75000000006000600fa00200798002e00900046
:10d76000100798000e8fe8001e00e80010407800b7
:10d770000080fb000080fa00000006000001780035
:10d780006e08b9008000780064004000038020002b
:10d79000608079001200600005003a006680400059
:10d7a00092009000608079000080600001003200eb
:10d7b00010002000000006006e09b9008201780008
:10d7c000e400410002802000e100790090807000b8
:10d7d00001187800e6804100e100790010887000af
:10d7e000000005001082fb00b001900082717a00f9
:10d7f0001082fb00b0019000848141004811de00de
:10d800009241980010c8e8000080e800eaff370065
:10d810009082fb003002900002f27a009082fb00be
:10d8200030029000050242004811de0012429800ca
:10d830001082fb0030019000040141002341980058
:10d840001082fb003001900004014100c819de0085
:10d850003341980010417800644841000080e8009e
:10d86000d5ff37001083fb00b002900082727b006e
:10d870001083fb00b0029000868242004811de0057
:10d88000924298009082fb00300190000501410017
:10d89000234198009082fb00300190000501410077
:10d8a000c819de00334198009081fb0030019000e0
:10d8b00003014100444198009081fb003001900039
:10d8c000030141004822de005441980010417800d5
:10d8d000664841000080e800b7ff37000800fa0002
:10d8e000889fbe008a1f7800000578000204780037
:10d8f00040c0b300a0f79f008004eb00a9bf9f00c9
:10d90000b9bf9f00c9bf9f000141780081c8b30023
:10d910000a0078007af3070066004500c0bf9f0048
:10d9200018487800c8409000114098005841900075
:10d9300022409800a8409000314098009800900044
:10d94000224080000100610077003a00280090002a
:10d950000608b60074003a009240800001006100a1
:10d960009e003a00280090001408b6009b003a0080
:10d970000241800001006100a3003a0028009000ed
:10d980002208b600a0003a00724180000100610048
:10d9900084003a00280090003008b60081003a0068
:10d9a000e241800001006100a1003a0028009000df
:10d9b0003e08b6009e003a0052428000010061001d
:10d9c000a5003a00280090004c08b600a2003a00da
:10d9d000c242800001006100ab003a0028009000c4
:10d9e0005a08b600a8003a003243800001006100e6
:10d9f000ad003a00280090006808b600aa003a007e
:10da0000a243800001006100b0003a0028009000ad
:10da10007608b600ad003a001244800001006100b3
:10da2000b2003a00280090008408b600af003a0027
:10da30008244800001006100e5003a002800900067
:10da40009208b600e2003a00f24480000100610052
:10da5000e8003a0028009000a008b600e5003a006f
:10da60006245800001006100ea003a002800900051
:10da7000ae08b600e7003a00d24580000100610020
:10da8000ed003a0028009000bc08b600ea003a0019
:10da90004246800001006100f1003a002800900039
:10daa000ca08b600ee003a00b246800001006100ec
:10dab000f3003a0028009000d808b600f0003a00c1
:10dac0002247800001006100f5003a002800900024
:10dad000e608b600f2003a009247800001006100bb
:10dae000f8003a0028009000f408b600f5003a006b
:10daf0000248800001006100fb003a00280090000d
:10db00000209b600f8003a00aff0970021459800ee
:10db10000a007800fff207004f0578004f04be00ae
:10db20000080fa0000000600b8519000e781610013
:10db300048509000670060004300dd008081710064
:10db400058509000670060004600dd008081710041
:10db5000e8509000e7806000c908dd00085190009f
:10db60006f01610018509000610060004400dd000a
:10db70000001710028509000630060004500dd0046
:10db80000001710081817100890078006e8057006a
:10db90001fff07000000e0000a003a009800900014
:10dba0006dff370058199000781a9000e81990001e
:10dbb000310020006e8057002aff07000000e000bf
:10dbc0002f0032000080eb004f0578004f04be00ac
:10dbd0000080fa0000000600d3ff370038009000f4
:10dbe000c800900081017800000178001100200039
:10dbf0006e80570006ff07000000e000f1ff3a00ca
:10dc0000980090005aff370028199000481a900099
:10dc1000b8199000210020006e80570011ff070006
:10dc20000000e000e7ff3a009800900056ff370040
:10dc300008219000282290009821900041002000a7
:10dc40006e80570007ff07000000e000ddff3a008c
:10dc50009800900058ff370038219000582290001b
:10dc6000c8219000510020006e805700fdfe070083
:10dc70000000e000d3ff3a009800900054ff370006
:10dc80009800900046ff3700682190006100200056
:10dc90006e805700d3fe07000000e000c9ff3a0085
:10dca0009800900050ff37000829900098299000b4
:10dcb000710020006e805700d5fe07000000e000d4
:10dcc000c0ff3a00980090004dff37007821900087
:10dcd000810020006e805700c2fe07000000e000b7
:10dce000b8ff3a00980090004bff3700d82a900008
:10dcf000482a9000b8299000a82890002ff097009b
:10dd00000081fb004fb89700017079002ff0970059
:10dd10000081fb004fb8970002004000c808de00f9
:10dd2000114098002ff197008280fb004fb89700b8
:10dd300001004000234098002ff097008080fb00f6
:10dd40004fb8970001004000c819de00334098002a
:10dd50002ff197008280fb004fb897000100400030
:10dd6000444098002ff097008080fb004fb8970048
:10dd7000010040004822de00544098002ff1970037
:10dd80008280fb004fb8970001004000654098007a
:10dd90002ff097008080fb004fb8970001004000f3
:10dda000c82ade0075409800aff09700e8c0400038
:10ddb000a1f79f00910020006c8057007efe0700b5
:10ddc0000000e0007fff3a009800900018ff370045
:10ddd00068299000f8299000a10020006e8057006b
:10dde0008bfe07000000e00076ff3a0098009000ec
:10ddf00015ff370008319000b10020006e805700f9
:10de000078fe07000000e0006eff3a0098009000e6
:10de100013ff370058019000e8019000c100200076
:10de20006e8057007afe07000000e00065ff3a00b0
:10de30009800900010ff37001831900038329000a1
:10de4000a8319000d10020006e80570085fe0700a9
:10de50000000e0005bff3a00980090000cff3700e4
:10de600048319000e10020006e8057005dfe070001
:10de70000000e00053ff3a00980090000aff3700ce
:10de800058319000f10020006e80570055fe0700c9
:10de90000000e0004bff3a009800900008ff3700b8
:10dea00068319000f8319000010120006e80570029
:10deb00057fe07000000e00042ff3a009800900083
:10dec00005ff3700083990009839900011012000b3
:10ded0006e8057004efe07000000e00039ff3a0058
:10dee0009800900002ff370042072000080141001f
:10def0002ff097008080fb004fb897008080400093
:10df000080002000b25878000000e900fdff3a00d0
:10df1000210120006c80570027fe07000000e00070
:10df200028ff3a00aff09700214598000a007800da
:10df3000f8f10700f8fe37000080fb000038a3006e
:10df40000e00320067006000c1f42900e20f5000ab
:10df5000080032001600340001f42900e30f5000dd
:10df600004003200c1f12900e40f5000010032002a
:10df70008000eb00010078000000060067006000f0
:10df800081f82900e20f5000faff3200100034003f
:10df9000c1f72900e30f5000f6ff320081f5290098
:10dfa000e40f5000f3ff32008000eb00f1ff370078
:10dfb00081f229000000e000eeff3200e10f500086
:10dfc000ebff3a0040f3290000000600ebff3700aa
:10dfd00041f629000000e000e6ff3200e10f5000aa
:10dfe000e3ff3a0000f7290000000600e3ff3700d6
:10dff00061006000f1f929000400320041f92900b4
:10e00000e10f5000010032008000eb0001007800b9
:10e010000000060063006000c1fc2900e10f500011
:10e02000080032000900340031fc2900e20f5000e2
:10e0300004003200a1fa2900e30f50000100320071
:10e040008000eb000100780000000600e1fb2900e1
:10e050000000e000faff3a0001007800000006002e
:10e06000faff37006700600091002a00e30f5000bc
:10e07000060032000700340041012a00e50f50007d
:10e0800002003200e1002a000e003d00010078008d
:10e0900000000600b1ff2900e10f5000fbff320035
:10e0a00001002a00f9ff3c0061ff29000000e000a8
:10e0b000f6ff320031fe2900010078000000060062
:10e0c000f4ff3700f1012a00e60f5000efff3200a5
:10e0d00071fd2900e70f5000ecff320031fe2900ee
:04e0e000f5ff370011
:020000040000fa
:10e0e400b00c00000a00000000000000580b000003
:10e0f4007e00000000000000ca0c000002000000c6
:10e104000200000000000000cc0c0000020000002f
:10e1140002000000c00a0000c00a000098000000cd
:10e12400000000008c0c000024000000020000002d
:10e1340000010000000000000000000000000000da
:10e1440000000000000000000000000000000000cb
:10e1540000000000000000000000000000000000bb
:10e16400ce0c00000200000002000000ffff0000cf
:10e1740000080000c00100000200000000000000d0
:10e184000000000001000000000000000200010087
:10e194000000000000000200000000000100020076
:10e1a4000002000000000000000400000000030062
:10e1b400000300000300000000000000080000004d
:10e1c400000700000300040000000000000010002d
:10e1d400000000000f000300000500000000000024
:10e1e4000020000000001f000003000006000000e3
:10e1f4000000000040000000003f00000100070094
:10e204000000000000008000000000007f00020009
:10e214000008000000000000000001000000ff00f2
:10e2240000010000090000000000000000020000de
:10e2340000ff010004000a000000000000000000cc
:10e2440004000000ff030200000b000000000000b7
:10e25400000008000000ff00070100000c0000009f
:10e26400000000000010000000ff0f0002000d007d
:10e27400000000000000000020000000ff1f030059
:10e28400000e000000000000000040000000ff003d
:10e294003f0100000f0000000000000000800000ab
:10e2a40000ff7f00010010000001000001000000d9
:10e2b40000000000ffff0200001100000100020046
:10e2c400000000000100ff00ff0200001200010036
:10e2d400000400000000030000ffff00040013001e
:10e2e400000100000800000000070000ffff00001c
:10e2f4000014000001001000000000000f00ff00e7
:10e30400ff000000150001000020000000001f00b5
:10e3140000ffff00000016000001000040000000a4
:10e32400003f0000ffff0000001700000100800014
:10e33400000000007f00ff00ff0000001800010043
:10e34400000000000000ff00ffffff0000001900b4
:10e35400000100000000000000ffff00ffff0000bc
:10e36400001a00000100000000000000ffffff0091
:10e37400ff0000001b00000000070000ffffff007b
:10e38400ffffff0000001c000000000000007c00f4
:10e3940000ffff00ffff0000001d00000000000060
:10e3a40000800200ffffff00ff0000001e000000cd
:10e3b400000000008001ff00ffffff0000001f00bd
:10e3c4000000000003000000e0ffff00ffff00006a
:10e3d40000000000620c00002a000000020000009f
:10e3e400640c8e007a8a7a008c7ad2007bda7b0005
:10e3f400fa7b54007cc67c00067d78000c8e7a0083
:10e404008a7a8c007a907a00987ab8007a127b0023
:10e41400847bc4007b010000d00c000002000000db
:10e4240000000000c009000000010000020000001c
:10e434004200000000000000000000000000000096
:10e4440000000000000000000000000000000000c8
:10e4540000000000000000000000000000000000b8
:10e4640000000000000000000000000000000000a8
:10e474000000000000000000000000000000000098
:10e484000000000000000000000000000000000088
:10e494000000000000000000000000000000000078
:10e4a4000000000000000000000000000000000068
:10e4b4000000000000000000000000000000000058
:10e4c4000000000000000000000000000000000048
:10e4d4000000000000000000000000000000000038
:10e4e4000000000000000000000000000000000028
:10e4f4000000000000000000000000000000000018
:10e504000000000000000000000000000000000007
:10e5140000000000000000000000000000000000f7
:10e5240000000000000000000000000000000000e7
:10e5340000000000000000000000000000000000d7
:10e5440000000000000000000000000000000000c7
:10e5540000000000000000000000000000000000b7
:10e5640000000000000000000000000000000000a7
:10e574000000000000000000000000000000000097
:10e58400000000000000000024100000060000004d
:10e59400020000000000000000000000940f0000d2
:10e5a4003a0000000200000000000000000000002b
:10e5b4000000000000000000000000000000000057
:10e5c40000000000000000000000ff00ffffff004b
:10e5d4000200050000000000000000000000000030
:10e5e4000000000000000000000000000000000027
:10e5f4000000000000000000d40c00008e010000a8
:10e60400000000003a1000000200000000000000ba
:10e61400ea0e000066000000020000000000000096
:10e6240000000000000000000000000000000000e6
:10e6340000000000000000000000000000000000d6
:10e6440000000000000000000000000000000000c6
:10e6540000000000000000000000000000000000b6
:10e6640000000000000000000000000000000000a6
:10e6740000000000ffffff00000000000000000099
:10e684000000000000000000000000000000000086
:10e694000000000000000000000000000000000076
:10e6a400000000003610000004000000000000001c
:10e6b400620e000088000000000000003c10000012
:10e6c4000200000000000000f00f00001200000033
:10e6d400000000001410000008000000000000000a
:10e6e400ba0c000008000000020000000000000056
:10e6f4000000000000000000d60b000046000000ef
:10e704000200000000000000000000000000000003
:10e7140000000000000000000000000000000000f5
:10e7240000000000000000000000000000000000e5
:10e7340000000000000000000000000000000000d5
:10e7440000000000000000000000000000000000c5
:10e7540000000000000000000000000000000000b5
:10e7640000000000c20c00000800000002000000cd
:10e774000000000000000000000000001c0c00006d
:10e78400460000000200000000000000000000003d
:10e794000000000000000000000000000000000075
:10e7a4000000000000000000000000000000000065
:10e7b4000000000000000000000000000000000055
:10e7c4000000000000000000000000000000000045
:10e7d4000000000000000000000000000000000035
:10e7e40000000000000000003e10000002000000d5
:10e7f40002000000000000002a10000006000000d3
:10e8040002000000040000000000000030100000be
:10e814000600000002000000220050000f22000049
:10e82400500f00004400000000000000021000002f
:10e8340012000000020000000100020000040000b9
:10e844000800100000000000202b2d0023300000e1
:10e854001c1000000800000002000000686a6c0040
:10e86400747a4c0000000000ce0f0000220000006b
:10e8740002000000303132003334350036373800be
:10e884003961620063646500660030003132330030
:10e894003435360037383900414243004445460098
:10e8a40000000000d20c0000020000000000000084
:04e8b4000000000060
:020000040000fa
:10e8b8000000fa000000370006c2bf006140600097
:10e8c8000004e000fcff3a0006c2bf00644060009c
:10e8d8000004e000f8ff3a0006c2bf00684060008c
:10e8e8000004e000f4ff3a0006c2bf007040600078
:10e8f8000004e000f0ff3a0009c2bf000044b20083
:10e908000004e000ecff3a000080fa000000060076
:10e918000000fa0007e2a90007a2a9000782a800e0
:10e928000762a9000742a9000722a8000702a90058
:10e9380006e2a90006c2a90006a2a9000682a9004b
:10e948000662a9000642a9000622a9000602a9003b
:10e95800f005200020108800c10a200091407800ae
:10e96800f0c8b30000c0600001c5b30001407000ea
:10e97800ace0b70008c2a9009600a90007e2a80009
:10e9880000a8210061002000f40b070010002000ff
:10e998000080fa00000006000000fa0007e2a90063
:10e9a8008620a9008600a9009600a900d8ff0700c4
:10e9b8000600070000fa200001002000e70b07000e
:10e9c800100020000080fa00000006000000fa0095
:10e9d8008620a9009620a80000322000010020000f
:10e9e800de0b0700100020000080fa00000006007f
:10e9f8000000fa008620a9009620a9001000200037
:10ea08000080fa00000006000600fa000000370047
:10ea180016c2bf00614060000004e000fcff3a003d
:10ea280016c2bf00644060000004e000f8ff3a002e
:10ea380016c2bf00684060000004e000f4ff3a001e
:10ea480016c2bf00704060000004e000f0ff3a000a
:10ea580016c2bf00624060000004e000ecff3a000c
:10ea6800a103210010c0b3008048780008c2bf008d
:10ea7800704060000004e000170032000602a800a1
:10ea88000071220001002000008fbe000b0037003b
:10ea9800a0032100104078000004e00003003a00c1
:10eaa80010002000200798000d0037000080eb00c0
:10eab8008080eb001e0f40005e9748001e00be00dd
:10eac800e00f5000e08f5800f1ff3a008000eb00a3
:10ead80021079800020037000000eb00200798008b
:10eae8002e0090000080fa00000006000600fa00e0
:10eaf800a103210060c0b3008048780008c2bf00ad
:10eb0800684060000004e000170032000622a800f8
:10eb18000071220001002000008fbe000b003700aa
:10eb2800a0032100104078000004e00003003a0030
:10eb380010002000200798000d0037000080eb002f
:10eb48008080eb001e0f40005e9748001e00be004c
:10eb5800e00f5000e08f5800f1ff3a008000eb0012
:10eb680021079800020037000000eb0020079800fa
:10eb78002e0090000080fa00000006000200fa0053
:10eb8800a103210030c0b3008048780006c2bf004e
:10eb9800614060000004e00010003a0006c2bf00b7
:10eba800644060000004e0000c003a0006c2bf00a8
:10ebb800684060000004e00008003a0006c2bf0098
:10ebc800704060000004e00004003a0006c2bf0084
:10ebd800624060000004e000030032000000eb0027
:10ebe800000f78000b00370006a2a9000682a800d3
:10ebf800a0032100104078000004e00003003a0060
:10ec080010002000000f7800020037000000eb0021
:10ec1800000f78001e0078000080fa00000006004f
:10ec28000600fa00a103210030c0b3008048780034
:10ec380006c2bf00614060000004e00010003a0016
:10ec480006c2bf00644060000004e0000c003a0007
:10ec580006c2bf00684060000004e00008003a00f7
:10ec680006c2bf00704060000004e00004003a00e3
:10ec780006c2bf00624060000004e00003003200ea
:10ec88000000eb00200798001700370006a2a80034
:10ec98000682a8000071220001002000008fbe003b
:10eca8000b003700a0032100104078000004e000aa
:10ecb80003003a0011002000210798000a003700dd
:10ecc8000080eb008080eb001e0f40005e9748003c
:10ecd8001e00be00e00f5000e08f5800f1ff3a0020
:10ece8008000eb00210798002e0090000080fa00b9
:10ecf800000006000a00fa003007980000712200a0
:10ed08000100200010079800210798000040eb0040
:10ed1800004f7800a103210040c0b300804878006c
:10ed280000712200010020001007980021079800b8
:10ed38001d00370006c2bf00614060000004e0000b
:10ed480013003a0006c2bf00644060000004e000ff
:10ed58000f003a0006c2bf00684060000004e000ef
:10ed68000b003a0006c2bf00704060000004e000db
:10ed780007003a0009c2bf000044b2000004e000e6
:10ed880003003a0010c0b300004f78000b003700b2
:10ed98001e009000ae00900061005000e080580016
:10eda80010079800210798001e009000ae00900000
:10edb800e00f5000e08f5800deff3a001e04e0002c
:10edc80003003a000000eb00400798001e003700df
:10edd8000662a800006a28001100200010079800a9
:10ede8002107980011003700a00321001040780087
:10edf8000004e00007003a0000108000804078001e
:10ee08003e0090000148780010002000400798005c
:10ee18000d0037001e009000ae0090006100500009
:10ee2800e080580010079800210798001e00900005
:10ee3800ae009000e00f5000e08f5800eaff3a0063
:10ee48000000eb00400798004e0090000080fa0098
:10ee5800000006000600fa00a103210050c0b3001c
:10ee6800804878000642a8000071220001002000b6
:10ee7800008fbe000b003700a0032100104078006f
:10ee88000004e00003003a0010002000200798006a
:10ee98000a0037000080eb008080eb001e0f400066
:10eea8005e9748001e00be00e00f5000e08f58003b
:10eeb800f1ff3a008000eb00210798002e00900037
:10eec8000080fa00000006000800fa004047980099
:10eed800a103210020c0b300804878004e40900074
:10eee8000000fb00101088000602a8000071220034
:10eef80001002000008fbe000b003700a003210096
:10ef0800104078000004e00003003a0010002000e0
:10ef1800300798000a0037000080eb008080eb0083
:10ef28001e0f40005e9748001e00be00e00f500014
:10ef3800e08f5800f1ff3a008000eb00310798009d
:10ef48003e0090000080fa0000000600809fbe008e
:10ef58000000fa008620a900a10321000040eb0070
:10ef6800804878000080fa004f00be00004006008c
:10ef780080658800e10f500004003a00926588001f
:10ef8800a3658800b4658800c56588000000060090
:10ef98008065800000000600000178000000e000a5
:10efa800040032006000b800e10f510006003a008a
:10efb80003003700207a8000317a80000200370091
:10efc80090658000a16580000000060000017800bf
:10efd8000000e000040032006000b800e10f5100ba
:10efe80006003a0003003700007a8000117a80009a
:10eff80002003700b0658000c1658000000006008f
:10f00800889fbe008a1f780081b5200000ac2000d0
:10f01800d3dc070068cbbf00e14f50001b00320073
:10f0280017003900e74f50001b003a00800020000d
:10f03800bedf0700f05b8000cf80de00fec907005e
:10f048000004be00e05b8000cf80de00fac9070044
:10f058000801be0075060700105c8000cf80de0046
:10f06800f5c907000004be00005c8000cf80de0008
:10f07800f1c907000801be00ad06070012013700fc
:10f0880010002000a9df07000f0137002000200032
:10f09800a6df07000c01370040002000a3df0700af
:10f0a8000000eb00f05b8800e05b8800105c8800e3
:10f0b800005c88006bcbbf000038a300030032005f
:10f0c80010002000f06f88001a0037006700600009
:10f0d800e10f500013003a00fe2def00205c800085
:10f0e800cf80de00d4c9070002002000a347240017
:10f0f8005aca07000004be0080658000a6ff07000a
:10f10800d2cc2c00c3e4230096ca07000001be003d
:10f118000800be00f4c907003071880041718800fa
:10f128000400370010002000f06f8800262eef0042
:10f13800282eef006ccbbf000038a300030032007c
:10f1480010002000206d88001b0037006700600059
:10f15800e10f500014003a00a42def00305c80004d
:10f16800cf80de00b4c9070002002000a3472400b6
:10f178003aca07000004be008065800093ff0700bc
:10f18800d2cc2c00c3e4230076ca07000001be00dd
:10f198000800be00d4c9070001f0a200606e880014
:10f1a800716e88000400370010002000206d880070
:10f1b800cc2def00ce2def006dcbbf000038a300a3
:10f1c8000300320010002000806788006b003700c1
:10f1d80067006000e10f50000f003200e30f50009d
:10f1e80060003a00f02cef00405c8000cf80de0029
:10f1f80091c90700b2fd20009304240059ca0700f2
:10f2080002002000134e240014ca0700c0688800ba
:10f21800d168880059003700f02cef00805c80002e
:10f22800880bb500cf80de0083c9070002002000ec
:10f238000312240009ca07000004be0016003700a4
:10f2480002002000433324000800be009aca0700c9
:10f258000000e0000500340002002000433b2400c9
:10f268000800be009fc907000004be00020020007d
:10f2780043332c000800be0091ca07000000e000dc
:10f2880005003d0002002000433b24000800be00aa
:10f2980095c907000004be006011b8000800be0050
:10f2a80087ca07000000e00009003d000045eb00a8
:10f2b8000200200043332c000800be0080ca07006b
:10f2c8000000e0000a003d001ac0b3000800370043
:10f2d8000045eb0002002000433324000800be0074
:10f2e80075ca07000000e000010034001ac0b3002e
:10f2f8000a04e000d2ff3a000200200003122400b2
:10f308000800be006cca07000000e00003003400db
:10f31800080020000912240008003700020020001d
:10f3280003122c000800be0065ca07000000e000b8
:10f3380002003d000800200009122c00d2cc2c004d
:10f34800c3dc23000800be0006ca07000200200034
:10f3580003122400c1c90700c0688800d16888006a
:10f3680006003700f02cef00805c8000cf80de00c4
:10f3780031c90700c0688800d1688800e1b620005c
:10f38800914078000180fb000038a3001000320093
:10f3980067006000e40f500004003a0010002000ed
:10f3a800606a8800506a8800470037004c2def00db
:10f3b80010002000506a8800405d8000cf80de0089
:10f3c8001dc90700906b8800a16b88003e003700bc
:10f3d80067806000e20f50002600320003003c0006
:10f3e800e10f500030003a0014003700e30f5000de
:10f3f8000e003200e40f50002b003a0010002000ed
:10f40800606a88004a2def00505c8000cf80de00e3
:10f4180009c9070002002000832c24008fc90700b7
:10f42800906b8800a16b8800270037004a2def00f9
:10f43800722def00742def00230037000000eb0061
:10f44800606a8800506a880010002000c07c88002c
:10f45800505c8000cf80de00f7c807000200200063
:10f46800832c24007dc90700906b8800a16b88005d
:10f47800150037000000eb00606a8800506a8800b9
:10f48800c07c8800505c8000cf80de00eac807009e
:10f4980002002000832c240070c90700906b8800ac
:10f4a800a16b8800080037000000eb00606a880044
:10f4b800506a8800405d8000cf80de00dec807000b
:10f4c800906b8800a16b88004f0578004f04be0040
:10f4d80000000600d02cec00000006008a0ce200b8
:10f4e80002003a008a2cef00000006008000eb00c2
:10f4f800e0a6270083020700fe06070001070700b1
:10f508008a2cef0000000600f8ff37000000050015
:10f518000000050000000500010078008200780066
:10f528003b08070000000500889fbe000104780022
:10f538008004eb0008007800b50807000000e00030
:10f54800060032000804e8008904e8000800780092
:10f55800af0807000000e000faff3a000900780051
:10f568004f04be0000000600889fbe008a1f780076
:10f57800010578000204be000300e00009003a001b
:10f58800820078000a007800210807002c0807008c
:10f598000000e000fdff3a004f0578004f04be0070
:10f5a80000000600d02cef00a1002000e0a62700f4
:10f5b800ac020700880078000a00780014080700e9
:10f5c8001f080700000478000000e0000b0032006c
:10f5d80080668000808f5400f9ff31008000eb00c6
:10f5e800e0a627009f0207000080eb004f05780087
:10f5f8004f04be0000000600eaff370080007800d4
:10f60800e0a6270097020700080078004f05780059
:10f618004f04be0000000600e2ff3700889fbe00ce
:10f628008a9fbe00010478000205780083047800f0
:10f638000300e0000e003a000200e000080032007b
:10f6480008007800720807000000e000fcff3200a4
:10f658000804e8008904e800890f5500f8ff3a001b
:10f668000000eb004f05be004f04be00000006007e
:10f67800d02cef00a1002000e0a6270079020700a7
:10f688000a00e0000b003a008a0578008000eb00d1
:10f69800e0a62700730207000080eb008a8f550060
:10f6a800efff32004f05be004f04be000000060009
:10f6b800efff37008005eb000800780054080700ca
:10f6c8000000e000020032000804e8008b05e800b2
:10f6d80080668000808f5400ecff39008a8f5500c7
:10f6e800f5ff39008000eb00e0a627005d02070067
:10f6f8000080eb008a8f5500eaff3a00d8ff3700f8
:10f70800881f7800010478000100e00006003a0034
:10f718003b0807000000e000fdff32000000eb009e
:10f728004f04780000000600d02cef00a100200054
:10f73800e0a627004b02070080668000800f540077
:10f74800080036002e0807000000e000faff32002b
:10f758008000eb00e0a62700420207000000eb0053
:10f76800efff37008000eb00e0a627003d0207000e
:10f778000080eb004f04780000000600eaff370025
:10f788000200fa000f80e900210807000000e000ed
:10f79800fcff3a000080fa00000006000100780033
:10f7a80082007800cb07070000000500889fbe0094
:10f7b800010478008004eb00080078003308070093
:10f7c8000000e000060032000804e8008904e800b0
:10f7d800080078002d0807000000e000faff3a0052
:10f7e800090078004f04be0000000600889fbe0094
:10f7f8008a1f7800010578000204be000300e000bb
:10f8080009003a00820078000a007800b107070072
:10f81800bc0707000000e000fdff3a004f05780034
:10f828004f04be0000000600d02cef00a10020000d
:10f83800e0a627000b020700880078000a0078007d
:10f84800a4070700af070700000478000000e000e5
:10f858000b00320080668000808f5400f9ff310071
:10f868008000eb00e0a62700fe0107000080eb0007
:10f878004f0578004f04be0000000600eaff37007d
:10f8880080007800e0a62700f6010700080078004d
:10f898004f0578004f04be0000000600e2ff370065
:10f8a800889fbe008a9fbe00010478000205780088
:10f8b800830478000300e0000e003a000200e00034
:10f8c8000800320008007800f00707000000e00098
:10f8d800fcff32000804e8008904e800890f55009d
:10f8e800f8ff3a000000eb004f05be004f04be00d1
:10f8f80000000600d02cef00a1002000e0a62700a1
:10f90800d80107000a00e0000b003a008a057800d9
:10f918008000eb00e0a62700d20107000080eb0082
:10f928008a8f5500efff32004f05be004f04be001e
:10f9380000000600efff37008005eb0008007800a4
:10f94800d20707000000e000020032000804e800c7
:10f958008b05e80080668000808f5400ecff39003a
:10f968008a8f5500f5ff39008000eb00e0a62700dc
:10f97800bc0107000080eb008a8f5500eaff3a00bf
:10f98800d8ff3700881f7800010478000100e000e4
:10f9980006003a00b90707000000e000fdff32004a
:10f9a8000000eb004f04780000000600d02cef00a8
:10f9b800a1002000e0a62700aa01070080668000b9
:10f9c800800f540008003600ac0707000000e00074
:10f9d800faff32008000eb00e0a62700a101070033
:10f9e8000000eb00efff37008000eb00e0a62700e7
:10f9f8009c0107000080eb004f047800000006001f
:10fa0800eaff37000200fa000f80e9009f070700ad
:10fa18000000e000fcff3a000080fa000000060049
:10fa2800881f7800000478008000eb000108780047
:10fa3800110098005ef70700110020000800780008
:10fa48005bf70700210020000800780058f707003e
:10fa5800310020000800780055f707004100200019
:10fa68000800780052f707005100200008007800cd
:10fa78004ff7070081002000080078004cf70700c6
:10fa8800c10020000800780049f707007100200035
:10fa98000800780046f70700910020000800780069
:10faa80043f70700b10020000800780040f707007e
:10fab80021012000080078003df70700e100200040
:10fac800080078003af707004f04780000000600a5
:10fad800881f7800b07c800000404000944fb70039
:10fae80058ebb700e0568000f1568000f05a8800c5
:10faf800015b880021578000115b88001057800047
:10fb0800205b88000200200003122400707380002c
:10fb18008173800013c8070046c80700605c88002e
:10fb2800020020000312240090738000a17380005b
:10fb38000cc807003fc80700705c8800020020005e
:10fb480003122400b0738000c173800005c8070049
:10fb580038c80700805c88000200200003122400d7
:10fb6800b0748000c1748000fec7070031c8070068
:10fb7800905c88000200200003122400d0748000ea
:10fb8800e1748000f7c707002ac80700a05c880056
:10fb98000200200003122400f07480000175800028
:10fba800f0c7070023c80700b05c880002002000e7
:10fbb800a3472400d0738000e1738000e9c70700e1
:10fbc8001cc80700c05c880002002000a34724006e
:10fbd800f073800001748000e2c7070015c80700b1
:10fbe800d05c880002002000a34724001074800025
:10fbf80021748000dbc707000ec80700e05c88009e
:10fc080002002000a34724007075800081758000e1
:10fc1800d4c7070007c80700f05c8800020020006e
:10fc2800a347240090758000a1758000cdc7070008
:10fc380000c80700005d880002002000a3472400d8
:10fc4800b0758000c1758000c6c70700f9c70700f6
:10fc5800105d8800a42bef0002002000832c2400f4
:10fc68005074800061748000bec70700f1c70700a8
:10fc7800405d880002002000832c240070748000fe
:10fc880081748000b7c70700eac70700505d880085
:10fc9800d0758000e1758000e6c70700305d8800f8
:10fca8009501070002002000832c2400b07f80000b
:10fcb800c17f8000abc70700dec70700605d880012
:10fcc800d701070002002000832c2400d07f800089
:10fcd800e17f8000a3c70700d6c70700705d8800d2
:10fce8001e02070002002000832c2400f07f800001
:10fcf800018080009bc70700cec70700805d880091
:10fd0800b2abef0021f4070002002000832c24008e
:10fd1800308180004181800092c70700c5c7070075
:10fd2800c05d8800d8ea2d00a85d8800b85d88000d
:10fd3800b0ab2a00d05d8800d0cd2c00e05d8800f3
:10fd4800f0ef2e00f05d880002002000832c2400d4
:10fd5800006980001169800082c70700b5c70700e5
:10fd6800005e8800185e8800285e8800385e88007b
:10fd7800485e880040232100505e8800c1bc2000f6
:10fd8800a0ef200007000900b05878004f04780061
:10fd980000000600460be20015003a00480be2009e
:10fda8000300320010002000305a8800100037008d
:10fdb80082b520008040eb00a0ae2000c5f6070009
:10fdc8000000e000080032006066800000899000b2
:10fdd8000200e00006003200c1112a0000082000dd
:10fde800020001000200370010002000305a88008d
:10fdf80000000600480be20015003a00460be2003e
:10fe08000300320010002000405a8800100037001c
:10fe180082b520008040eb00a0ae2000adf60700c0
:10fe28000000e00008003200606680000089900051
:10fe38000200e00006003200b1132a00000820008a
:10fe4800020001000200370010002000405a88001c
:10fe5800000006000000e00003003200e10f50003f
:10fe68000b003a00050037006a08b90080007800e6
:10fe7800e0ec27007b0007000c0037006a08b90097
:10fe880080007800e0ef27007600070007003700c1
:10fe980060668000008990000200e00003003200e4
:10fea800a1152a0000082000020001000000060039
:10feb8000000fa000000eb00800888000111200013
:10fec80091407800f0ccb30000c0600010e1b700aa
:10fed8000000eb003008880000fa20006008880065
:10fee80084e0a90094e0a80011e1a8000080fa00cd
:10fef800000006000000fa0011e1a9000080fa00e5
:10ff0800000006000800fa00100798002107980072
:10ff1800e0818000000f78000b0037001e00780099
:10ff2800b00090001e009000808f500003003a003f
:10ff380011002000310798001f0037001e007800cc
:10ff4800c0009000010f78001e00e000f3ff3a00a7
:10ff5800a0002000cfc10700000f78001e00e000bd
:10ff680002003a00100020001cc20700ae009000fa
:10ff78001e007800010878009e0078000000eb0061
:10ff8800900098009e00780010c0b300c040980010
:10ff98001e0078009e00900031009800e1818000ea
:10ffa8001e007800410098001e007800e08188005b
:10ffb80011002000310798003e0090000080fa00f0
:10ffc800000006000800fa00200798000000eb0077
:10ffd80010079800e0818000000f78001a003700b1
:10ffe8001e007800b00090002e009000808f500016
:10fff80010003a001e0090000000e00005003200ea
:020000040001f9
:100008001e007800c00090001e009000410098007b
:10001800030037001e00780040009000e08188004f
:100028001e007800ffc1070011002000310798006a
:10003800090037001e007800100798001e0078009d
:10004800c0009000010f78001e00e000e4ff3a00b5
:1000580020002000300798003e0090000080fa0041
:10006800000006000800fa00100798002107980011
:10007800e0818000000f78000e0037001e00780035
:10008800b00090001e009000808f500006003a00db
:10009800ae0090001e0078000108780011002000d2
:1000a80031079800070037001e007800c000900054
:1000b800010f78001e00e000f0ff3a002000200049
:1000c800300798003e0090000080fa00000006000b
:1000d8000600fa0010079800e0818000000f780001
:1000e8000e0037001e007800b00090001e0090003f
:1000f800808f500006003a009e0078000000eb0058
:100108009000980011002000210798000700370090
:100118001e007800c0009000010f78001e00e0006b
:10012800f0ff3a0020002000200798002e009000e1
:100138000080fa00000006000600fa001007980088
:10014800e0818000000f78000e0037001e00780064
:10015800b00090001e009000808f500006003a000a
:100168009e0078000040eb00c0409800110020007d
:1001780021079800070037001e007800c000900093
:10018800010f78001e00e000f0ff3a002000200078
:10019800200798002e0090000080fa00000006005a
:1001a8000600fa0010079800e0818000000f780030
:1001b8000e0037001e007800b00090001e0090006e
:1001c800808f500006003a009e00780010c0b300ef
:1001d800c040980011002000210798000700370050
:1001e8001e007800c0009000010f78001e00e0009b
:1001f800f0ff3a0020002000200798002e00900011
:100208000080fa00000006003600f800809fbe005b
:10021800829fbe00849fbe00869fbe003400f80007
:1002280000c0b300a00188000200fa00cac2bf00e3
:10023800624060000004e00002003a00ca22a80000
:1002480001003700ca22a900e0818000000f780071
:1002580084e0a9001e0037001e007800404090008e
:10026800e14f500017003a001e0078001000780097
:100278000000e000130032001e007800100090001b
:100288008000e8001e007800110098001e00780029
:1002980010009000800078001e00780010007800a0
:1002a8000000e900808f5000060036001e0078002c
:1002b80030009000000001009e0078000000eb0074
:1002c800900098001e007800c0009000010f780090
:1002d8001e00e000e0ff3a000080fa003400f90058
:1002e8004f03be004f02be004f01be004f00be00cc
:1002f8003600f900004006000800fa00889fbe009a
:10030800c0002000460407008000780000ff20009d
:100318000108780000ff2000100478006140b9004f
:1003280045c5070020079800310798000800e0003d
:1003380007003d0002002000037824002e009000f2
:10034800be00900068c50700200798003107980094
:100358002e009000be009000008fbe00020020001a
:10036800030a24001e00be00fec507001e01be00d1
:10037800fcc507000004be0002002000034a240058
:100388001e00be00f7c507000001be000800be0041
:1003980055c507000200200003a3240052c507002a
:1003a8000001be000000200001aa2400abc5070020
:1003b80062ff20000089be0060ff20001000be0020
:1003c8006011b8003ec607000000e00001003500db
:1003d8000400370062ff20006000b8000089be00fa
:1003e8000c00370060ff20001000be000200200053
:1003f8000300240030c607000000e00001003c00b4
:100408000400370062ff20000000200001002400e3
:100418000089be004f04be000080fa0000000600fc
:100428000800fa00889fbe00b0002000fc03070007
:100438008000780000ff20001100980000ff2000d5
:10044800100490006140b900fbc407002007980021
:10045800310798000800e00007003d000200200076
:10046800037824002e009000be0090001ec50700ef
:1004780020079800310798002e009000be009000d9
:10048800008fbe0002002000030a24001e00be00e8
:10049800b4c507001e01be00b2c507000004be00b7
:1004a80002002000034a24001e00be00adc507005c
:1004b8000001be000800be000bc5070002002000b6
:1004c80003a3240008c507000001be0000002000a7
:1004d80001aa240061c5070062ff200020019800de
:1004e8003101980060ff2000b000900020009000cb
:1004f8006011b800f2c507000000e00001003500f7
:100508000500370062ff20006000b8002001980055
:10051800310198000e00370060ff2000b000900005
:10052800200090000200200003002400e2c507001c
:100538000000e00001003c000500370062ff2000d9
:1005480000002000010024002001980031019800db
:100558004f04be000080fa00000006000800fa0000
:10056800889fbe00a0002000ad030700800078002f
:1005780000ff20002100980000ff200020049000c8
:100588006140b900acc40700200798003107980003
:100598000800e00007003d00020020000378240066
:1005a8002e009000be009000cfc4070020079800de
:1005b800310798002e009000be009000008fbe000a
:1005c80002002000030a24001e00be0065c50700c3
:1005d8001e01be0063c507000004be000200200023
:1005e800034a24001e00be005ec507000001be00cd
:1005f8000800be00bcc407000200200003a32400ba
:10060800b9c407000001be000000200001aa2400b0
:1006180012c5070062ff20004001980051019800b0
:1006280060ff2000d0009000400090006011b800ea
:10063800a3c507000000e0000100350005003700f1
:1006480062ff20006000b800400198005101980046
:100658000e00370060ff2000d0009000400090009e
:10066800020020000300240093c507000000e000fa
:1006780001003c000500370062ff20000000200058
:100688000100240040019800510198004f04be0069
:100698000080fa00000006000400fa0020479800d5
:1006a800314798000040eb00004f780018003700f1
:1006b80010c0b300004f7800d3f807001e4f600049
:1006c8002e40900000fa07001e4f60003e40900048
:1006d800fdf907001e4f600004f907001e4f600077
:1006e8002e4090000040e800f7f907001e4f600018
:1006f8000e00e8007ff907001e4f600048f9070068
:10070800d4f907001e04e00003003a00a2f807002d
:100718001e04e000e6ff32001e4090000000fb00cf
:100728000080fa00000006000800fa002047980040
:100738002107980062479800734798000040eb0033
:10074800004f780010c0b300004f7800aef80700e3
:100758001e4f60002e409000dbf907001e4f60001e
:100768006e409000d8f907001e4f6000dff80700c0
:100778001e4f60002e4090000040e800d2f90700ac
:100788001e4f6000150037002e00900059f9070031
:100798001e4f60002e0090000000e800200798001f
:1007a8007e4090000040e900704798007e4090002d
:1007b8000004e00003003a0019f907001e4f60002a
:1007c80002003700edf807001e4f600006c2bf00a8
:1007d800704060000004e000fcff3a007e4090009a
:1007e8000004e000e8ff3a009af907001e00fb0049
:1007f8000080fa00000006000600fa002047980072
:1008080031479800424798000040eb00004f7800bd
:100818001200370010c0b300004f78007af80700c4
:100828001e4f60002e409000a7f907001e4f600081
:100838003e409000a4f907001e4f60004e40900013
:10084800a1f907001e4f600082f907001e4f6000e3
:100858001e04e00003003a004ff807001e04e00001
:10086800ecff32001e00fb000080fa0000000600ca
:100878000400fa00100798000040eb00004f7800d1
:100888000040eb00104798001600370010c0b30076
:10089800004f78005cf807001e4f600000c1b300ed
:1008a80089f907001e4f600010c0b30086f90700e1
:1008b8001e4f60008df807001e4f600010c1b30086
:1008c80081f907001e4f60000e00e80009f90700d3
:1008d8001e4f6000d2f807001e4f60005df9070048
:1008e8001e4f60001e04e000e8ff32001e4090002a
:1008f8000000fb000080fa00000006000600fa0075
:1009080010079800414798000040eb00004f78001e
:100918000f00370010c0b300004f78003af8070006
:100928001e4f600000c1b30067f907001e4f60004a
:100938000040eb0064f907001e4f600050c0b30090
:1009480061f907001e4f600042f907001e4f600062
:100958001e04e000efff32000080fa0000000600ed
:100968000000fa00eaf707000080fa00000006001d
:100978000000fa0015f807000080fa0000000600e1
:100988000000fa001af807000080fa0000000600cc
:100998000000fa000000eb00200c88000000eb00cb
:1009a800100c880010272000000c8800e0002000b0
:1009b800200c88000000eb00500c88000000eb00c1
:1009c800400c880010272000300c8800e000200030
:1009d800500c88000000eb00800c88000000eb0041
:1009e800700c88000000eb00600c8800e00020001c
:1009f800800c88000000eb00b00c88000000eb00c1
:100a0800a00c88000000eb00900c8800e00020009b
:100a1800b00c8800a0862100700888000002280019
:100a2800900888000080fa00000006000800fa001c
:100a3800008fbe00220798003307980002002000ac
:100a480003f823001e00be009bc407000000e0005e
:100a580001003c00030037000000200001f82300db
:100a6800008fbe006011b8001e00be0094c40700cd
:100a78000000e00001003500020037006000b80007
:100a8800008fbe000200200003f823002e00900013
:100a9800be00900088c407000000e00001003c0090
:100aa800040037000000200001f823002007980008
:100ab800310798006011b8002e009000be00900029
:100ac8007fc407000000e000010035000300370084
:100ad8006000b80020079800310798000200240041
:100ae800c34124001e00be001ec4070002002400eb
:100af800c34124007cc3070073c40700000c8800ae
:100b080002002400c34124002e009000be00900083
:100b180014c4070002002400c341240072c3070064
:100b280069c40700300c88000080fa000000060045
:100b38000800fa00008fbe002207980033079800cb
:100b48000200200003f823001e00be005ac407005c
:100b58000000e00001003c00030037000000200016
:100b680001f82300008fbe000200200003f82b00cc
:100b78001e00be0052c407000000e000010035005e
:100b8800030037000000200001f82b00008fbe0092
:100b98000200200003f823002e009000be00900001
:100ba80045c407000000e00001003c0004003700d5
:100bb8000000200001f82300200798003107980062
:100bc8000200200003f82b002e009000be009000c9
:100bd8003bc407000000e0000100350004003700b6
:100be8000000200001f82b0020079800310798002a
:100bf80002002400c33924001e00be00d9c3070028
:100c080002002600a346240037c307002ec40700ad
:100c1800600c880002002400c33924002e009000d4
:100c2800be009000cfc3070002002600a3462400a0
:100c38002dc3070024c40700900c88000080fa0028
:100c4800000006000000fa008500a9000080fa00f4
:100c5800004006000000fa00410b20009140780097
:100c6800f0c8b30000c0600001c6b30001407000c6
:100c7800b4e0b700901220001013880060c2a900e9
:100c880061e2a8000080fa00000006000200fa00f5
:100c9800004f780011479800e922a9001e80fb0048
:100ca800350007001e4090000080fb00320007005e
:100cb800e922a8006022a900800720000100200086
:100cc800260307000080fa00000006000800fa006a
:100cd800004f780011479800224798003347980042
:100ce800444798005547980066479800774798000a
:100cf800e922a9001e80fb001f0007001e4090008b
:100d08000080fb001c0007002e4090000080fb00c4
:100d1800190007003e4090000080fb001600070005
:100d28004e4090000080fb00130007005e409000da
:100d38000080fb00100007006e4090000080fb0060
:100d48000d0007007e4090000080fb000a000700ad
:100d58000ef897000080fb0007000700e922a800b2
:100d68006022a9008007200001002000fb02070084
:100d78000080fa00000006000200fa00000f780068
:100d880063c2bf00644060000004e000030032005a
:100d98001e0078004013880003003700f00f200081
:100da8001e0060004013880060c2bf0062406000ff
:100db8000004e000fcff3a0060c2bf006140600030
:100dc8000004e000fcff320040138000000f7800b0
:100dd8000080fa00000006000600fa00004f7800c4
:100de8001107980042479800e922a9001e80fb00dd
:100df800e1ff0700ce4090001e00900006000700ab
:100e0800e922a8008007200001002000d302070083
:100e18000080fa00000006000400fa00000f7800c5
:100e280021479800080037000c0007008040780030
:100e38001e007800014878001e0fe8002e40900040
:100e48000040e900204798002e4090000004e00090
:100e5800f5ff3a000080fa00000006000200fa00e0
:100e680060c2a9000000eb004013880060c2bf0008
:100e7800614060000004e000fcff320060c2bf0077
:100e8800614060000004e0000d00320060c2a9006b
:100e980063c2bf00644060000004e0000300320049
:100ea80040138000000f78000700370041138000ce
:100eb800f00f200080806000010f780002003700ea
:100ec8000080eb00000f78001e0078000080fa0018
:100ed800000006000000fa004174200091407800ec
:100ee80000ceb30000c060003040b30044e7b70054
:100ef80044c7bf00f043b20044e7b700e001200058
:100f0800303a88000000eb00403a880040a7a9006a
:100f18003200200081072000a0092000337420003f
:100f280081497800804978008249780012002000c1
:100f38006104200070052000237420008149780096
:100f4800804978008249780043c7bf0002c7b300d0
:100f58008240600000c3b30080cf5000faff3a001f
:100f680042c7bf000042b2000004e000fcff3200ac
:100f78000080fa00000006000000fa000000eb0004
:100f8800200888008460a900510a20009140780058
:100f9800f0c8b30000c0600001c5b3000140700094
:100fa800a5e0b7000000eb000008880000c4290095
:100fb800100888000080fa00000006000000fa000f
:100fc8009460a80005e1a8000080fa00000006006f
:100fd8000000fa009460a90005e1a9000080fa0069
:100fe800000006000000fa000000eb0090088800ee
:100ff8008500a900810a20009140780080cfb300c5
:1010080000c060005040b300a8e0b7000000eb004b
:10101800500888000080fa00000006000000fa006e
:101028009500a80013e1a8000080fa00000006005f
:101038000000fa009500a90013e1a9000080fa0059
:10104800000006000400fa00008fbe001e00be006b
:1010580002002400c3312400c2c207001ac30700db
:10106800d008880000032800f0088800110b200031
:1010780091407800f0c8b30000c060000044a000b0
:10108800b1e0b7008760a9009760a8000080fa0067
:10109800000006000600fa00fdc4070070052000e5
:1010a8002007980060ac2800a0808800a0be280017
:1010b800b0808800f0fd2f0005c5070080c02c0017
:1010c80010079800d0752900000f78002e019000b5
:1010d8009e0078001e009000d8c507000000eb00b5
:1010e800b06088000000eb00c06088000080fa0053
:1010f800000006000000fa00e6ff07000080fa0082
:10110800000006000000fa00020007000080fa0054
:10111800000006000600fa00e5c40700700520007c
:101128002007980080b22800c080880080c228006c
:10113800d0808800f0fd2f001ac5070080602c00c1
:1011480010079800d0752900000f78002e01900034
:101158009e0078001e009000c4c507000000eb0048
:10116800e06288000000eb00f06288000080fa006e
:10117800000006000c00fa007005200050079800d7
:101188007005200040079800f0fd2f00d0c407002c
:1011980080c02c0030079800910a20009140780008
:1011a800f0c8b30000c0600001c2b3000140700085
:1011b800a9e0b700a10a20009140780080cfb300d1
:1011c80000c060000014a000aae0b70080802c00d6
:1011d80030079800005028002007980090fb2f0047
:1011e800f0c40700310b20009140780080cfb30095
:1011f80000c060003040b300b3e0b700310b2000fe
:1012080091407800f0c8b30000c0600001c3b3008b
:1012180001407000b3e0b70080602c001007980010
:10122800d0752900000f78005e019000ae00900094
:101238003e00900081c507004e0190009e00780096
:101248001e00900089c507000080fa000000060013
:10125800881f78007100200001087800b1638000c1
:10126800210098000004eb00180098009bf8070084
:10127800080078004f04780000000600881f7800f6
:101288008100200001087800116380002100980087
:101298000004eb001800980090f807000800780098
:1012a8004f04780000000600881f780000047800ca
:1012b800a00090000100e00007003200100090003c
:1012c8009100780001000100800078000000eb0028
:1012d8001004980020049800010078004f0478005a
:1012e80000000600a00090001000900091009000ff
:1012f80001400100a000900010009000a1009000a3
:1013080001400100a001900010009000b30190007e
:1013180003400100a001900010009000c30190005c
:101328000340010020029000100090005402900039
:101338000440010020029000100090006402900018
:1013480004400100200190001000900072019000fc
:1013580002400100a0009000100090008108900059
:1013680001400100889fbe008a1f780000057800b0
:10137800810478000204780001007800b7bc0700f7
:101388000001780088017800890078000a00780058
:10139800e4ff07004f0578004f04be000000060078
:1013a8000000fa0021e3a90021a3a9002143a80015
:1013b8001132200091407800c0cfb30000c0600017
:1013c80021e3b700013220009140780000ceb3003d
:1013d80000c0700020e3b7002043a9002023a90023
:1013e8002003a90023c3bf007f40600023e3b700a8
:1013f8002223a9002203a90025e3a90025c3bf00d1
:10140800f041b30025e3b700f0c3b30024e3b7000d
:101418000080eb00501988000080fa0000000600e8
:101428000400fa001007980028e3a9001e009000a5
:101438007f4060007f416000813220009140780049
:1014480000ceb30000c060000240700028e3b7007f
:101458000000eb0070198800110020001e009000a9
:101468000008dd00801988000080eb005019880012
:10147800110020001e0090000008dd000080ea0036
:101488006019880021e3a8002023a80020c3bf001a
:10149800614060000004e000fcff3200001880009a
:1014a800000f78002023a90021e3a9001e0078007e
:1014b8000080fa0000000600706488008000eb00dd
:1014c800421f2a0003ca2000124078000004e000ee
:1014d8000a00320080f079008100e8000201e8008b
:1014e800f08f5000f8ff3a0000c920000058eb00c8
:1014f800808f5100fdff3a000000060000ca20005e
:10150800008040000058eb008100e800ef8f500099
:10151800f5ff3e000058eb008100e800ef8f500017
:10152800f8ff3600f0ff37000001eb0003c9200088
:10153800e04079000104e0000500320001f1790083
:101548000201e800f00f5100f9ff3a000000060020
:1015580000c92000000041000058eb000201e8002b
:10156800ef0f5100f9ff3e000058eb000201e800c0
:10157800ef0f5100f8ff3600f4ff3700c0c8200015
:10158800000006008580a900809fbe00821f7800a9
:10159800ba2cec00c00ce20015003200bc0ce200d2
:1015a80016003200be0ce20014003200e165800033
:1015b800420020002322af00feff3700f0658000c4
:1015c8000000e000070032000000e900beacb700f0
:1015d8003140780024e2b7000201e900f5ff3a0043
:1015e80002003700bc2cef0001003700e1658800dd
:1015f8004f0178004f00be000040060000002000a8
:10160800006688004f0178004f00be0000400600c9
:10161800c00ce200feff3a009580a9008100e900b5
:10162800f1658800b040780021118800e0658800e5
:1016380011002000016688009580a80000000600bf
:10164800006680000000060087e0a900809fbe00b9
:10165800821f7800c22cec00c80ce2001500320092
:10166800c40ce20016003200c60ce200140032007e
:1016780021668000420020003322af00feff3700c1
:10168800306680000000e000070032000000e9003a
:10169800c6acb7003140780034e2b7000201e90077
:1016a800f5ff3a0002003700c42cef0001003700b4
:1016b800216688004f0178004f00be0000400600f8
:1016c80000002000406688004f0178004f00be00ef
:1016d80000400600c80ce200feff3a0097e0a900af
:1016e8008100e90031668800b0407800a1118800c7
:1016f80020668800110020004166880097e0a80055
:101708000000060040668000000006000000fa00a5
:10171800e2ce2000f0282c0051cf23005019980069
:1017280061199800e2ce200070b5250011d323007e
:101738005009980061099800e2ce2000e05320008b
:1017480001bc23007009980001119800e2ce200026
:101758006000b8001011980021119800e2ce200016
:10176800a0702d0031c223005021980061219800fb
:1017780082d42000d0cc2c00c1e42300500998006a
:101788006109980082d42000a0702d0031c2230086
:10179800700998000111980082d42000d0cc2c0048
:1017a800c1dc2300101198002111980082d4200078
:1017b80080eb210051f0230030119800411198006e
:1017c8000000eb000080fa0000000600809fbe00c9
:1017d8008560a9001a2cec00b0608000f003b2000c
:1017e80061bd2000810040000000eb0026c2bf0060
:1017f80080487800162cec004f00be000040060020
:10180800b0608000c1608000010050000000060048
:10181800b1608000c26080000208e1000800320068
:10182800f203b20061bd20000281400092407800be
:1018380001487800182cec00100020000000060079
:101848000000eb0000000600809fbe0087c0a900d2
:10185800602cec00e0628000f003b200c1c12000ff
:10186800810040000000eb0036c2bf0080487800cd
:101878005c2cec004f00be0000400600e0628000d7
:10188800f16280000100500000000600e162800063
:10189800f26280000208e10008003200f203b200a0
:1018a800c1c12000028140009240780001487800c0
:1018b8005e2cec0010002000000006000000eb0089
:1018c800000006000000fa00ca22a8000024240034
:1018d800f100200021000700ca22a90000242400ea
:1018e800f10020001d0007000080fa00000006003b
:1018f8000000fa00caa2a80000242400f100200079
:1019080016000700caa2a90000242400f100200044
:10191800120007000080fa00000006000000fa002c
:10192800ca22a900c622a900caa2a900c6a2a90063
:10193800e4c2a900e4e2a800e502a900e522a900a2
:10194800d302a900c602a800cb22a900c722a90079
:10195800d362a8000080fa0000000600f03fb10042
:101968000180b10006003500ee0309000000000008
:10197800403fb1000180b100fbff3d001000b00006
:10198800203fb00002003500008009000000000080
:1019980000000600ca2cef000000e0000100320041
:1019a800ffff370000000600ca2cec0012002000e0
:1019b80081b5200000ac2000a0d30700000006007d
:020000040000fa
:020000040001f9
:0419c8000000fe001d
:00000001FF
